:100000000C9449180C947A180C947A180C947A1859
:100010000C947A180C947A180C947A180C947A1818
:100020000C947A180C947A180C947A180C947A1808
:100030000C942F210C947A180C947A180C947A183A
:100040000C947A180C947A180C947A180C947A18E8
:100050000C947A180C947A180C947A180C946626DE
:100060000C947A180C943A250C9411250C947A1857
:100070000C947A180C947A180C947A180C947A18B8
:100080000C947A180C947A180C947A180C947A18A8
:100090000C947A180C947A180C947A180C94B02654
:1000A0000C947A180C947A180C947A180C947A1888
:1000B0000C947A180C947A180C947A180C947A1878
:1000C0000C947A180C947A180C947A180C947A1868
:1000D0000C947A180C947A180C947A180C947A1858
:1000E0000C947A18E954EB54ED54EF54F154F35452
:1000F000F554015593229622852289228F22CD2202
:100100009A229E22A422A822AC22B222B622BA228D
:10011000CD22C022C422C822E829EE29F129F729DC
:10012000022A0A2A0D2A172A36503B5040504A50BC
:100130005450CD505E5066506E50785082508C5066
:100140009B50A550CD50AF50B950C35000407A10CD
:10015000F35A00A0724E18090010A5D4E80000E878
:100160007648170000E40B54020000CA9A3B0000D6
:1001700000E1F505000080969800000040420F0065
:100180000000A08601000000102700000000E80326
:10019000000000006400000000000A0000000000F1
:1001A0000100000000002C76D888DC674F0823DFB0
:1001B000C1DFAE59E1B1B796E5E3E453C63AE65183
:1001C000997696E8E6C28426EB898C9B62ED407CAA
:1001D0006FFCEFBC9C9F40F2BAA56FA5F490055A46
:1001E0002AF75C936B6CF9676DC11BFCE0E40D476B
:1001F000FEF520E6B500D0ED902E0300943577058E
:100200000080841E080000204E0A000000C80C3345
:100210003333330F986E12831141EF8D2114893BD4
:10022000E65516CFFEE6DB18D1844B381BF77C1D54
:10023000901DA4BBE424203284725E228100C9F1A7
:1002400024ECA1E53D2700002100240027002A001E
:100250002D003000330001010000040107010A01F4
:1002600015EF03038002CF0300C130ED04640312D5
:1002700081E803850078CB05392C003402F7012092
:10028000EA020000C00123C10110C5023E28C701D7
:10029000863601483A0155B1020018B60308822794
:1002A000F20100260101E00F0F312B0C0E084EF178
:1002B000370710030E0900E10F000E140311073178
:1002C000C148080F0C31360F11807829007F1F823A
:1002D00007840684068407827F18820784068406C2
:1002E0008407827F20278E0F900D920D9001800849
:1002F00081018E01820683108404850E8504850E9B
:100300008504850E8504850E8504850E8504850E7D
:100310008504850E8504850E8504850E8504850E6D
:100320008504850E8504850E8504850E850484105C
:10033000840482028E028204800292028006960960
:10034000940C9002811B83198519851985198519CB
:1003500085198519851985198519851985198519AD
:100360008519851A830B8E01810B900D920D900FCC
:100370008E28278E0F900D920D9001800881018E9E
:1003800001820683108404850E8504850E8504850C
:100390000E8504850E8504850E8504850E850485ED
:1003A0000E8504850E8504850E8504850E850485DD
:1003B0000E8504850E8504850E85048410840482D0
:1003C000028E0282048002920280069606800194C8
:1003D0000782019002810484118304850E850485BF
:1003E0000E8504850E8504850E8504850E8504859D
:1003F0000E8504850E8504850E8504850E8504858D
:100400000E8504850E8504850E8504850E8504857C
:100410000E85058310830781018E01810B900D925B
:100420000D900F8E28278E0F900D920D9001800C4D
:100430008E01821B841985198519851985198519DD
:100440008519851985198519851985198519851ABB
:10045000841C821E805D811B83198519851985196D
:10046000851985198519851985198519851985199C
:1004700085198519851A831C817F24278E0F900D7D
:10048000920D900B81018E0B831A851985198519A0
:10049000851985198519851985198519851985196C
:1004A00085198519841A82028E0A8002920A96069C
:1004B0008001940782019002810484118304850ED7
:1004C0008504850E8504850E8504850E8504850EBC
:1004D0008504850E8504850E8504850E8504850EAC
:1004E0008504850E8504850E8504850E8504850E9C
:1004F0008504850E85058310830781018E01810B9C
:10050000900D920D900F8E28278E0F900D920D90CA
:100510000B81018E0B831A8519851985198519851B
:1005200019851985198519851985198519851985DB
:1005300019841A82028E0A8002920A9609940C90FB
:1005400002811B83198519851985198519851985D6
:1005500019851985198519851985198519851985AB
:100560001A830B8E01810B900D920D900F8E287FB8
:100570001980088112820683108404850E85048503
:100580000E8504850E8504850E8504850E850485FB
:100590000E8504850E8504850E8504850E850485EB
:1005A0000E8504850E8504850E8504850E850484DC
:1005B00010840482028E02820480029202800696D7
:1005C00009940C9002811B83198519851985198559
:1005D000198519851985198519851985198519852B
:1005E000198519851A831C817F24278E0F900D92FF
:1005F0000D9001800C8E01821B8419851985198547
:1006000019851985198519851985198519851985FA
:10061000198519851A840A8E02820892028006962C
:1006200009940C9002811B831985198519851985F8
:1006300019851985198519851985198519851985CA
:10064000198519851A830B8E01810B900D920D90DF
:100650000F8E28278E0F900D920D9001800C8E0129
:10066000821B84198519851985198519851985199C
:10067000851985198519851985198519851A840A99
:100680008E028208920280069606800194078201FB
:100690009009841A8519851985198519851985196F
:1006A0008519851985198519851985198519851A59
:1006B000831C81018E0F900D920D900F8E287F1953
:1006C000801D821B8419851985198519851985193D
:1006D0008519851985198519851985198519851B28
:1006E000831D811E805D811B8319851985198519DC
:1006F000851985198519851985198519851985190A
:1007000085198519851A831C817F24278E0F900DEA
:10071000920D9001800881018E018206831084046D
:10072000850E8504850E8504850E8504850E850459
:10073000850E8504850E8504850E8504850E850449
:10074000850E8504850E8504850E8504850E850439
:10075000850E850484108404821482048018802409
:10076000801E8215810484118304850E8504850E04
:100770008504850E8504850E8504850E8504850E09
:100780008504850E8504850E8504850E8504850EF9
:100790008504850E8504850E8504850E8504850EE9
:1007A00085058310830781018E01810B900D920DC9
:1007B000900F8E287F7F7F7B8207840684068407C4
:1007C00082107F7F7F7F3F7F7F10860C83028B09A3
:1007D00083018D0883008F078805860686098406B5
:1007E000850B8405840D8305840D8305840D8404A5
:1007F000830F8304830F8304830F8304830F830495
:10080000830F8304830F8304830F8304830F830484
:10081000830E8404840D8305840C8405850B840574
:10082000860984068805860683008F0783018D0864
:1008300083028B098304860C83188318831883181A
:100840008318831883188318831883327F7F7F056A
:100850008607860A830289048A0883008C028C0733
:1008600083008D008E068705890584068508860825
:100870008405840A840A8305840A840A8305830B19
:10088000830B8305830B830B8305830B830B83050A
:10089000830B830B8305830B830B8305830B830BF4
:1008A0008305830B830B8305830B830B8305830BEA
:1008B000830B8305830B830B8305830B830B8305DA
:1008C000830B830B8305830B830B8305830B830BC4
:1008D0008305830B830B8305830B830B8305830BBA
:1008E000830B8305830B830B8305830B830B837F30
:1008F0007F7F7A7F7B880F8D0A9009910785068517
:1009000006840A8405830C8305830C8305830C838A
:10091000168315840E8B09900792068D0183058836
:10092000078305840B8304840C8304830D83048371
:100930000D8304830C8404830B8504840986058459
:10094000068A038F0184048D0284058A0583078645
:100950007F7F357F1A8409840984098409847F3D57
:100960008409840984098409847F7422880F8C0C8B
:100970008F0991078605860585098405840B840403
:10098000830D8303840D8303830F8302830F83020C
:10099000830F8302830F8302830F8302840D8403FA
:1009A000830D8403840B85048409860486058805E9
:1009B00094068E0083078B02830A860483168315B0
:1009C00083168303830E8303830D8403840C8305C2
:1009D000830B84058409850685058608900A8E0C9C
:1009E0008B11867F7F332485118B0C8F09910786AD
:1009F00005860684098405840B8404840B8404839F
:100A00000D8304830D8304830D8304840B84058389
:100A10000B830684098407850585098F0B8D0B8F51
:100A200009910785078505840B8404830D8303845E
:100A30000D8402830F8302830F8302830F8302835B
:100A40000F8302830F8302840D8402840D84038448
:100A50000B840486078605930791098F0D897F7F94
:100A600031379603960396039616831583158315DF
:100A700083158414841484158315841484158414B4
:100A800084158315841583158415841583158415A1
:100A90008316831584158316831683168315841590
:100AA00083168316837F7F532486118B0C8E0A90C6
:100AB000088605850685098405840B8305830C84D7
:100AC00003840D8303830E830383168315831683A8
:100AD00004860A83028B0783008E069405880586A8
:100AE0000486098404850B8403840D8303840D84A8
:100AF00002830F8302830F8302830F8302830F839A
:100B000002830F8303830D8403830D8304840B848A
:100B100005840985058605860791098F0C8C0F8849
:100B20007F7F313A910891089108910882168316C7
:100B3000831683168217821782168302870B83001F
:100B40008B09910892078605860684098505830B23
:100B500084168316841683168316831683168303DE
:100B6000830E8303830D8403830D8304840B840528
:100B7000840985058605860791098F0B8D0F877F70
:100B80007F3245831584148513861386128711835B
:100B9000008311830083108301830F8302830E84FB
:100BA00002830E8303830D8304830C8305830B84EC
:100BB00005830B8306830A830783098407830983DC
:100BC00008830883098307830A830797029702979C
:100BD0000297118316831683168316831683168352
:100BE000168316837F7F4A23870F8D0B900891070A
:100BF0008605860684098405840B8404840B84049A
:100C0000830D8304830D8304830D8315841584145D
:100C10008414850D8B0E89108B0E8C14861584160A
:100C200084158402830F8302830F8302830F830260
:100C3000840D8402840C8503840B84048509850556
:100C40008605860791098F0B8D0F877F7F4D24873F
:100C5000108C0B8F0991088505860684098406840B
:100C60000A8306830B8404840C8304830D8304832A
:100C70000D8304830D8316831584158414841485D1
:100C8000138512861187108810880F8810871186A7
:100C90001285138514841484158316831596039680
:100CA000039603967F7F4529821782168316831544
:100CB00084148512870D8C0D8C0D8700830D8403A1
:100CC000831683168316831683168316831683165C
:100CD000831683168316831683168316831683164C
:100CE000831683168316831683168316831683163C
:100CF000837F7F4C23870F8D0B8F09910786058695
:100D00000684098406830B8305840B8404830D8386
:100D100004830D8304830D8303830F8302830F8376
:100D200002830F8302830F8302830F8302830F8367
:100D300002830F8302830F8302830F8302830F8357
:100D400002830F8302830F8302830F8302830F8347
:100D500003830D8304830D8304830D8304840B8438
:100D600005830B8306840984068605860791098F0F
:100D70000B8D0F877F7F327F7F7F558409840984A5
:100D8000098409847F387F7F458A058A058A058A18
:100D90007F7F7F2B7F7F7F7F3F19118309810181B7
:100DA0000781038203800080068101810080078320
:100DB0007F7F2C01830A820A810A810A810A810AC3
:100DC000810A810A810A810A810B810B82088109CB
:100DD000810A810A810A810A810A810A810A810ABB
:100DE00081098207831304810A810A810A810A81A9
:100DF0000A810A810A810A810A810A810A810A819B
:100E00000A810A810A810A810A810A810A810A818A
:100E10000A810A810A810A81120683078209810AEE
:100E2000810A810A810A810A810A810A810A81096B
:100E30008108820B810B810A810A810A810A810A59
:100E4000810A810A810A810A820A830E48890189FE
:100E50000882078207820782088108820782078248
:100E6000078208890189544D82068200810681012A
:100E7000810681028104810381048103810481044C
:100E8000810281058102810581028106810081073D
:100E90008100810781008108820982098209810914
:100EA0008206840783144E810681018204820281B6
:100EB00004810481028105820082068408820884FC
:100EC00006820082058102810481048102820482FB
:100ED000018106815B6B81048204810081048204AC
:100EE00081008104800080048101810281008102EF
:100EF00081028102810081028102810281008102DE
:100F000081028102800280028103810081028100CE
:100F100081048100810281008104810081028100BD
:100F2000810582048206820482068204827F014750
:100F30008106810081068101810481028104810290
:100F4000810481038102810481028104810281057F
:100F500081008106810081068407820882585581BC
:100F60000681028106810281068102810681028159
:100F70000681028106810281068102810681028149
:100F80000681028105820282038303860081048434
:100F90000181620F81048104810481028500850240
:100FA0008104810481048104810481048104810419
:100FB0008104830382314A8405870282038102818E
:100FC000058101810A8407860784098101810581E1
:100FD00001820382028704855631810082018501E6
:100FE00082048105810581058105810581058105D1
:100FF00081058105813B5E83018104860081038335
:1010000001840381058202820681028107810281B7
:1010100007810281078102820681038105820383A1
:10102000018404860081068301810C810C810C817E
:101030000C810C811F5B8101830681008604840181
:101040008303820581038106820281078102810771
:101050008102810781028106820282058103840167
:1010600083038100860481018306810C810C810C3D
:10107000810C81285E8407880483028303810681B2
:101080000282068201810881018108810181088133
:101090000182068202810681038302830488078419
:1010A0006D5B8101840581008604830382038205D0
:1010B0008103810681038106810381068103810604
:1010C00081038106810381068103810681038106F4
:1010D00081038106816A7F05810183038305810085
:1010E00085008604830284028203820482048103D1
:1010F00081058105810381058105810381058105C4
:1011000081038105810581038105810581038105B5
:1011100081058103810581058103810581058103A5
:1011200081058105817F1B07810381038103810381
:10113000810381038103810381038103810381038F
:1011400081038103810381038103812B198109813B
:10115000098109810981048201810382028102825D
:101160000381018204810082058505860482018154
:10117000048102820381038103810382028104814D
:1011800002810482530781038103810F810381035C
:10119000810381038103810381038103810381032F
:1011A0008103810381038103810381038101830121
:1011B00082080781038103810F81038103810381F9
:1011C00003810381038103810381038103810381FF
:1011D00003812B10810C810C810C810C810C81010D
:1011E00084058100860483038203820581038106CE
:1011F00081038106810381068103810681038106C3
:1012000081038106810381068103810681038106B2
:10121000816A5E83018104860081038301840381E6
:101220000582028107810281078102810781028193
:10123000078102820681038105820383018404867B
:101240000081068301810C8102810781028106826F
:101250000382038204890685130A830284028105BE
:10126000810581038600860281058105810581054E
:10127000810581058105810581058105813B5883B3
:101280000787048301830381058102820681018B24
:10129000018B01810B820B8105820283018304870C
:1012A00007836619810C810C810C810C81068301F6
:1012B0008104860081038301840381058202820602
:1012C00081028107810281078102810781028206F2
:1012D00081038105820383018404860081068301E2
:1012E000816A52830687038301820381058101821B
:1012F00009810A810A810A820581028105810283AE
:101300000182048706835E10810C810C810C810CA4
:10131000810C810183068100860484018303820598
:101320008103810682028107810281078102810790
:101330008102810682028205810384018303810088
:1013400086048101836D57850588048104820381A9
:1013500005810B810587038902820581028106814F
:101360000281068102820383038600830284028253
:10137000610B830385018201820081038100810367
:101380008100820182018503837F1A7F7F1D8C2665
:10139000108207810081058102810381048101811E
:1013A00006817F6F09840384068106810681068198
:1013B00006810681068106810681068106810681F5
:1013C00006810681068106810681068106810384E5
:1013D00003841401800B800B810B800B800B810B2D
:1013E000800B800B810B800B800B810B800B800BA3
:1013F000810B800B800B810B800B800B810B800B92
:10140000800B810B800E0B8403840381068106818F
:101410000681068106810681068106810681068194
:101420000681068106810681068106810681068184
:101430000684038412118C028C0C820B820B820CAA
:10144000810C810C820B820B820C810C810C820B33
:10145000820B820B820C8D018D700F8209820082BB
:10146000078202810781038205820481058106814A
:10147000038107820182088101810A830B830C8129
:101480000D810D810D810D810D810D810D81760FF5
:10149000810881018206820281068104810481051E
:1014A000820282068102810881008109840A820BFE
:1014B000820A8100810882008207810281068104FC
:1014C00081048204820381068102820682008208EE
:1014D0008268168206820682008106820681018168
:1014E00006820681018204810081048202810481D6
:1014F00000810481038104810081048103810481CE
:1015000000810481038202810281028204810281BE
:1015100002810281058102810281028105810281AD
:10152000028102810582008104810082068100819E
:10153000048100810781008104810081078100818D
:10154000048100810783068308820682098206825D
:101550007F250E8208820081088101810881018136
:10156000088102810681038106810381068104814D
:10157000048105810481058104810681028107813E
:10158000028107810281088100810981008109842B
:101590000A820B826E13810981038109810381090B
:1015A0008103810981038109810381098103810903
:1015B00081038109810381098103810981038109F3
:1015C00081038109810381098103810981038207E4
:1015D0008204820582068908877F020D9B05810BA4
:1015E000810B810B810B810B810B810B810B810B9B
:1015F000810B810B810B810B810B810B8167148522
:1016000007890482058203810781038107810381A1
:10161000078202820D840B860B850C830D8201826A
:101620000881028108810281088102830582038A80
:10163000068673128B048C03810882028109810261
:101640008109810281098102810981028108810366
:101650008C038B0481078203810881038108820245
:101660008109810281098102810981028109810246
:10167000810981771886098A068304830482088297
:1016800003810A8102820A8201810C8101810C811D
:1016900001810C8101810C8101810C8101810C810E
:1016A0000182068002820281058201810382058512
:1016B00004830483068C07860182108073118A04D8
:1016C0008B038107820281088102810881028108DF
:1016D000810281088102810782028B038A04810DC5
:1016E000810D810D810D810D810D810D817B18860C
:1016F000098A068304830482088203810A810282A4
:101700000A8201810C8101810C8101810C8101819E
:101710000C8101810C8101810C8101820A8202818C
:101720000A810382088204830483068A09867F0A69
:101730001382088103820881038307810384068161
:10174000038100810681038100820581038101827A
:101750000481038102810481038102820381038168
:101760000382028103810481028103810482018159
:101770000381058200810381068100810381068443
:101780000381078303810882038108827F16820A0E
:101790008203830883038308830383088303810010
:1017A000810681008103810081068100810381001F
:1017B000810681008103810181048101810381010E
:1017C00081048101810381018104810181038102FE
:1017D00081028102810381028102810281038102EF
:1017E00081028102810381038100810381038103DE
:1017F00081008103810381038403810381048204C6
:10180000810381048204817F140E810A810A810A86
:10181000810A810A810A810A810A810A810A810A70
:10182000810A810A810A810A810A8A018A5A1281FF
:101830000882028107820381068204810582058174
:101840000482068103820781028208810182098164
:10185000008309870883018207820382068105814C
:101860000681058205810682048107820381088240
:10187000028109827615810A810A810A810A810A18
:10188000810A810A810A810A810A810A810181060D
:10189000810181068101810681018204820288041E
:1018A000865E0781038103810381038103810381B4
:1018B0000381038103810381038103810381038108
:1018C0000381038103812B13810981038109810332
:1018D00081098103810981038109810381098103D0
:1018E000810981038D038D038109810381098103AE
:1018F00081098103810981038109810381098103B0
:1019000081098103810981038109817F1886098A00
:1019100006820583048208810481098202820F8184
:101920001081108105870281058702810B81028168
:101930000B8102820A810381098203820783048367
:10194000048405890081078503807F06108B028B44
:1019500002810C810C810C810C810C810C8A038A20
:1019600003810C810C810C810C810C810C810C8118
:1019700073118C028C02810D810D810D810D810D01
:10198000810D8B038B03810D810D810D810D810DE7
:10199000810D8C028C701389078B0581068304816D
:1019A0000882038109810381098202810A810281FF
:1019B0000A8102810A8102810A8102810A810281EF
:1019C0000A810281098202810981038108820381DF
:1019D0000683048B05897F031786088A05830483A1
:1019E0000382088103810A8101820A8101810F81BA
:1019F0000F810F810F810F810B8101820A8102818A
:101A000009820282088104830483058A08867F0292
:101A1000128A058C03810782038108810381088172
:101A2000038108810381088103810782038A058C71
:101A30000381078203810981028109810281098171
:101A40000281098102810782038C038A7A15830B44
:101A5000830B830A81018109810181098101810848
:101A60008103810781038107810381068105810547
:101A70008105810589048B03810781038107810228
:101A800081098101810981008209826F21880D828B
:101A9000068209820A8107810D8105810F810480F8
:101AA0000683018003810281048102830381028114
:101AB0000381048104810181048104810481018105
:101AC00003810581048101810381058104810181F4
:101AD00003810481048102810381048104810281E4
:101AE00003810481038104810381028202810581D3
:101AF000048301840781178117810B810982058383
:101B00000D876C10850488038203820182058101A0
:101B10008106810181068109820882088208820982
:101B200081098209822382098209825F62820C8292
:101B30000C830C820D8108820783078208827F153F
:101B40005186018613860186636B820882078307AC
:101B50008208810D820D820C820C827F0C2B820305
:101B6000820382348203820382058004810480041C
:101B700081172B8203820382348203820382321F05
:101B80008505880482038202820581028107810122
:101B9000810781018107810182058202820383021C
:101BA0008A048401810B81018106810281068103FF
:101BB0008104820388058665208307870581038168
:101BC00004810581038105810381058104810381ED
:101BD00006850687048203820281078101810781CD
:101BE00001810781018107810282038203890585C2
:101BF000651C8B018B0A810A8209820A810A820A8A
:101C0000810A810B810A820A810B810B810A810B77
:101C1000810B816920840688038204810381068107
:101C20000281068101810B810184048A028303827F
:101C3000028205820181078101810781018107817B
:101C4000028105820282038204880585651D89035D
:101C50008903810B810B810B810084058902830339
:101C600082028106820B810B810B81018107810138
:101C700082058202820382038905856524810A82A6
:101C8000098309830881008107810181068102811E
:101C9000068102810581038104810481038105811C
:101CA000038B018B09810B810B810B81641F8506DE
:101CB000870482038203810581028205810B810AE8
:101CC00082078408850B820B8101810781018107CE
:101CD00081018205820282038203890585651F8551
:101CE00005890382038202820681018107810181C5
:101CF00007810B810A820883078406840783088290
:101D000009820A810B8B018B6222810B810A820777
:101D10008507850B810B810B810B810B810B810B5F
:101D2000810B810B810B810B810B816620830787DF
:101D30000483018303810581028205820181078179
:101D4000018107810181078101810781018107816B
:101D5000018107810181078101820582028105815C
:101D60000383018304870783660D81058105800550
:101D70008105810580058105810580058105810535
:101D80008005810581058005810581058005810526
:101D9000812D7182038203823258850185687182A8
:101DA0000382038205800481048004811753810724
:101DB000810781048701870481078107816710817A
:101DC00009810981068001810180028903850683DA
:101DD0000681018104820182048003807F360781AD
:101DE00006800681068006810581058106810581C0
:101DF00005810581058105810581058105810581B3
:101E000004810581058105800581058005810D0D11
:101E10008105800581058005810581058104810595
:101E20008105810581058105810581058105810582
:101E3000810681058105810680068106800681076D
:101E40000682028202820480038102817415840A60
:101E50008608820282078104810781048107810349
:101E600082088101820A840A830B8503810382012F
:101E7000820281028203820181028105840381063C
:101E8000830381078104820485038801820385041A
:101E900082762D8207810586058006810281048174
:101EA0000581048102810681048102800781048109
:101EB0000181088102810280098601800C820281F1
:101EC00002820C80018609800281028108810181E1
:101ED00004810780028104810681028104810581D9
:101EE00004810281068005860581078207807F0CB8
:101EF0001F85058903820382028107810181078191
:101F000001810B820B810A8707810B810B810B8179
:101F10000A810B860280018B01810483632E81017B
:101F2000810C8002800D8002800C8101810C800276
:101F3000800D800280088D088002800D8002800D57
:101F4000800280088D088002800D8002800C810153
:101F5000810C8002800D8002800C8101817F0D093F
:101F60008001800380018003800180038001800361
:101F700080018003800180038001807F110A810538
:101F80008105810581058105810581058105810521
:101F9000810581058105811581058105813A7F01D2
:101FA0000000304848300000000000000000000041
:101FB000000000324C0000000000000000000000A3
:101FC0000040202020202020102020202020204001
:101FD00000004040404040404040404040404000C1
:101FE0000010202020202020402020202020201011
:101FF000000000000000FC0408304080FC000000ED
:1020000000000000000084848484844C3404087040
:1020100000000000000088885020508888000000E0
:102020000000000000008282829292AA4400000018
:10203000000000000000828282824428100000001C
:1020400000000000000084848484844C340000007C
:10205000000000004040E0404040404030000000B0
:102060000000000000007088807008887000000088
:10207000000000000000B0C8808080808000000068
:10208000000000000000344C8484844C34040406B6
:10209000000000000000B0C8848484C8B080808044
:1020A00000000000000038448282824438000000B2
:1020B000000000000000B0C8848484848400000014
:1020C000000000000000ACD29292929292000000B8
:1020D000000000C040404040404040404000000000
:1020E0000000008080808890A0C0A0908800000040
:1020F0000000000010003010101010101010906040
:1021000000000000400040404040404040000000CF
:10211000000000808080B0C8848484848400000033
:10212000000000000000304C8484844C34040870AB
:102130000000003048404040E04040404000000087
:10214000000000000000384484F88044380000009B
:10215000000000000404344C8484844C34000000EB
:1021600000000000000038448080804438000000F7
:10217000000000008080B0C8848484C8B0000000E3
:10218000000000000000700804748C8C74000000D3
:10219000000000404040200000000000000000005F
:1021A0000000000000000000000000000000FF0030
:1021B000000000000000000000000000000000001F
:1021C0000010284400000000000000000000000093
:1021D00000000000000000000000000000000000FF
:1021E0000000E020202020202020202020E00000EF
:1021F00000000404080810102020404080800000E7
:102200000000E080808080808080808080E000000E
:10221000000000FE0204081010204080FE000000B4
:10222000000000828282442810101010100000006C
:10223000000000828244281010284482820000009E
:10224000000000000000808080808080888088807E
:102250004900550055002200220000000000000047
:10226000000000828282824444282810100000006E
:1022700000000082828282828282824438000000D2
:10228000000000FE101010101010101010000000C0
:1022900000000038448280601C0282443800000044
:1022A000000000F884828284F89088848200000014
:1022B000000000384482828282828244380806000C
:1022C000000000F88482828284F880808000000010
:1022D00000000038448282828282824438000000FA
:1022E000000000C2C2A2A292928A8A8686000000E2
:1022F000000000000000C180C180A280A280948004
:1023000094808880888080808080000000000000A9
:10231000000000808080808080808080FC00000041
:10232000000000848890A0C0A090888482000000F3
:102330000000000202020202020282443800000091
:10234000000000E04040404040404040E0000000CD
:1023500000000084848484FC8484848484000000DD
:102360000000003C428080809C8282423C00000051
:10237000000000FE808080F8808080808000000067
:10238000000000FE808080FC80808080FE000000D5
:10239000000000F88482828282828284F800000039
:1023A0000000003C42808080808080423C00000031
:1023B000000000F8848284F884828284F80000009F
:1023C0000000001010282844447C82828200000013
:1023D0000000003C4299A5A5A5A59E403E00000036
:1023E00000000038448202040810100010000000B1
:1023F00000000000804020100810204080000000F5
:1024000000000000000000F800F8000000000000DC
:10241000000000000810204080402010080000004C
:10242000000000000000C0C000C0C04080000000EC
:10243000000000000000C0C000C0C000000000009C
:1024400000000038448282463A020204780000000C
:10245000000000384482443844828244380000003E
:102460000000007E020204040808101010000000A2
:102470000000003C408080B8C482824438000000E4
:10248000000000FC808080F80402028478000000D4
:10249000000000040C14244484FE04040400000022
:1024A00000000078840204380402028478000000EE
:1024B000000000384482020418204080FE00000022
:1024C0000000001030501010101010107C000000A0
:1024D0000000003844448282828244443800000074
:1024E00000000404080810102020404080800000F4
:1024F0000000000000000000000000C0C00000005C
:102500000000000000000000F800000000000000D3
:102510000000000000000000000000C0C04080007B
:102520000000000000002020F82020000000000033
:102530000000000010925438549210000000000077
:1025400000C020100808040404040408081020C077
:10255000000C102040408080808080404020100C83
:10256000000040404080000000000000000000002B
:10257000000000205088885020528C8C730000008E
:1025800000000061919264081026498986000000CD
:102590000000003C4240407040704040FE0000009F
:1025A000000000242424FF2424FF2424240000000D
:1025B0000000A0A0A000000000000000000000003B
:1025C00000000040404040404040400040000000CB
:1025D00000000000000000000000000000000000FB
:1025E0000C0C0C0C0C0C0C0C0C0C0C0C0C0C0C0C2B
:1025F000202020202020202020200C0C0C0C0C0C53
:102600000C0C0C0C0C0C0C0C0C0C0C0C0C0C0C0C0A
:102610000C0C0C0C0C0C0C0C0C0C0C0C0C0C0C0CFA
:102620000C0C0C0C0C0C0C0C0C0C0C0C0C0C0C0CEA
:102630000C0C0C0C0C0C0C0C0C0C0C0C0C0C0C0CDA
:10264000C207C207C207C207C207C207C207C20742
:10265000C207C207C207C207C207C207B407C20740
:102660000B07BE065306EA056F0508057B04250423
:102670007203E502CD02C207C207C207C207C20742
:10268000C207C207C207C207C207C207C207C20702
:10269000C207C207C207C207C207C207C207C207F2
:1026A000C207C207C207C207C207C207C207C207E2
:1026B000C207C207C207C207C207C207C207C207D2
:1026C000C207C207C207C207C207C207C207C207C2
:1026D000C207C207C207C207C207C207C207C207B2
:1026E000C207C207C207C207C207C207C207C207A2
:1026F000C207C207C207C207C207C207C207C20792
:102700000C0C0C0C0C0C0C0C0C0C0C0C0C110F0C01
:102710001B1B1B1B1B1B1B1B1B1B0F0C0C0C0C0C60
:102720000C0C0C0C0C0C0C0C0C0C0C0C0C0C0C0CE9
:102730000C0C0C0C0C0C0C0C0C0C0C0C0C0C0C0CD9
:102740000C1B0C0C0C0C0C0C0C0C0C0C0C2A0C0C9C
:102750001D0C0C0C0C0C0C0C0C0C0C0C070C0C0CAD
:10276000940D940D940D940D940D940D940D940D61
:10277000940D940D940D940D940D860D770D940D7C
:10278000F40CA70C4E0CE70B820B230BA80A610A72
:10279000E6096B095309940D940D940D940D940D55
:1027A000940D940D940D940D940D940D940D940D21
:1027B000940D940D940D940D940D940D940D940D11
:1027C000940D940D940D940D940D940D940D940D01
:1027D000940D940D940D940D940D940D940D940DF1
:1027E000940DF308940D940D940D940D940D940D87
:1027F000940D940D940D940D940D4C08940D940D1E
:10280000C707940D940D940D940D940D940D940D93
:10281000940D940D940D940D940D940D940D940DB0
:10282000050808130E15110608080C0A0708070802
:102830000E0E0E0E0E0E0E0E0E0E07070E090E0DCC
:102840001910111212100F1312060D110D1512137B
:10285000101311100E120F170F1010090D090C0D87
:10286000090E0F0D0F0E080F0F06060C06160F0FA0
:102870000F0F080C070E0C120D0D0C0D0D0D0F0196
:102880009E1F7D1F5F1F1D1FF01E921E4D1E401EAE
:102890000F1EDE1DBE1DAD1D9E1D991D921D691DC5
:1028A0002C1D091DDE1CAD1C7C1C4D1C141CF11BB9
:1028B000B81B7F1B721B5D1B491B401B2C1B031B82
:1028C0008C1A4D1A101AD819961971194C190C191D
:1028D000C718A21875182E1809188D173017EE167C
:1028E000BD1674163316FE15DB1595155215D21448
:1028F0008F145A1435140614D313A41390138B1386
:10290000711346130713E212A3127E125912121208
:10291000D311B21185114C112711D610A1107410CA
:102920003510F60FD90FB60F930F5E0F2F0FD50E80
:10293000A60E670E4C0E190EE60DB30D9A0D990DED
:102940000603040908090903070708060306050723
:102950000808080808080808080803030606060807
:10296000090808080808080808040808070A0808E9
:10297000080808080808080A0808080407040709DE
:1029800004070707070706070704050604080708E2
:1029900007080606050708080607070503050806D1
:1029A000D025C025B025A02590258025702560253F
:1029B000502540253025202510250025F024E02431
:1029C000D024C024B024A024902480247024602427
:1029D000502440243024202410240024F023E02319
:1029E000D023C023B023A02390238023702360230F
:1029F00050234023302320231023F022E022D02232
:102A0000C022B022A0229022802270226022402286
:102A10003022202210220022F021E021C021A0211A
:102A200090218021702160215021402130212021DE
:102A300010210021F020E020D020C020B020A020D4
:102A400090208020702060205020402030202020C6
:102A500010200020F01FE01FD01FC01FB01FA01FBC
:102A6000000020002300260029002C002F00320047
:102A70000001000003010601090100000000000040
:102A800000000008A0294029100000000000802854
:102A900020281A000000000060270027304026E0B0
:102AA0002530000000000000002200250028002B37
:102AB000002E003100340002010000050108010B66
:102AC0000105050505070508080808020202020AB3
:102AD0000A080804040404010101010101010103C1
:102AE00003030303030303040707070C0C0C0C0C7C
:102AF0000C0C0C0202020206060606060606060B6F
:102B00000B0B0B0B0B0B0B010210202008081020E5
:102B10004010204080020102010804020101020469
:102B20000810204080804020100804020180040228
:102B3000018040201008040201080402010102047F
:102B4000081020408001020408102040800000008E
:102B500000003E5B4F5B3E3E6B4F6B3E1C3E7C3E3F
:102B60001C183C7E3C181C577D571C1C5E7F5E1C4D
:102B700000183C1800FFE7C3E7FF0018241800FF07
:102B8000E7DBE7FF30483A060E2629792926407F01
:102B9000050507407F05253F5A3CE73C5A7F3E1C10
:102BA0001C08081C1C3E7F14227F22145F5F005FFC
:102BB0005F06097F017F006689956A6060606060DA
:102BC00094A2FFA29408047E040810207E2010081E
:102BD000082A1C08081C2A08081E101010100C1EB9
:102BE0000C1E0C30383E3830060E3E0E060000003B
:102BF000000000005F00000007000700147F147F42
:102C000014242A7F2A12231308646236495620505E
:102C10000008070300001C2241000041221C002A7A
:102C20001C7F1C2A08083E08080080703000080835
:102C3000080808000060600020100804023E5149A6
:102C4000453E00427F400072494949462141494D75
:102C5000331814127F1027454545393C4A494931FC
:102C600041211109073649494936464949291E007B
:102C70000014000000403400000008142241141425
:102C8000141414004122140802015909063E415D42
:102C9000594E7C1211127C7F494949363E414141CF
:102CA000227F4141413E7F494949417F090909014C
:102CB0003E414151737F0808087F00417F41002059
:102CC00040413F017F081422417F404040407F0245
:102CD0001C027F7F0408107F3E4141413E7F09096D
:102CE00009063E4151215E7F091929462649494975
:102CF0003203017F01033F4040403F1F2040201F1F
:102D00003F4038403F6314081463030478040361B0
:102D100059494D43007F41414102040810200041C0
:102D200041417F040201020440404040400003074B
:102D3000080020545478407F2844443838444444A0
:102D400028384444287F385454541800087E090217
:102D500018A4A49C787F0804047800447D400020D7
:102D600040403D007F1028440000417F40007C042B
:102D70007804787C080404783844444438FC1824E7
:102D8000241818242418FC7C0804040848545454BB
:102D90002404043F44243C4040207C1C2040201C50
:102DA0003C4030403C44281028444C9090907C4457
:102DB00064544C4400083641000000770000004194
:102DC00036080002010204023C2623263C1EA1A173
:102DD00061123A4040207A3854545559215555795A
:102DE000412154547841215554784020545579401C
:102DF0000C1E52721239555555593954545459397B
:102E0000555454580000457C410002457D42000164
:102E1000457C40F0292429F0F0282528F07C5455E1
:102E200045002054547C547C0A097F493249494961
:102E3000323248484832324A4848303A4141217A91
:102E40003A42402078009DA0A07D39444444393D59
:102E50004040403D3C24FF2424487E4943662B2FBC
:102E6000FC2F2BFF0929F620C0887E09032054542B
:102E700079410000447D413048484A323840402280
:102E80007A007A0A0A727D0D19317D2629292F28A8
:102E9000262929292630484D4020380808080808E6
:102EA000080808382F10C8ACBA2F102834FA0000D0
:102EB0007B000008142A142222142A1408AA0055A0
:102EC00000AAAA55AA55AA000000FF00101010FF82
:102ED00000141414FF001010FF00FF1010F010F089
:102EE000141414FC001414F700FF0000FF00FF147A
:102EF00014F404FC141417101F10101F101F1414C6
:102F0000141F00101010F0000000001F101010100F
:102F10001F10101010F010000000FF101010101003
:102F200010101010FF10000000FF140000FF00FF41
:102F300000001F10170000FC04F4141417101714DD
:102F400014F404F40000FF00F714141414141414FF
:102F5000F700F7141414171410101F101F14141472
:102F6000F4141010F010F000001F101F0000001FDC
:102F700014000000FC140000F010F01010FF10FF0F
:102F8000141414FF141010101F00000000F010FFA4
:102F9000FFFFFFFFF0F0F0F0F0FFFFFF0000000088
:102FA00000FFFF0F0F0F0F0F38444438447C2A2ACC
:102FB0003E147E02020606027E027E0263554941ED
:102FC000633844443C04407E201E2006027E0202F8
:102FD00099A5E7A5991C2A492A1C4C7201724C300C
:102FE0004A4D4D303048784830BC625A463D3E49E3
:102FF0004949007E0101017E2A2A2A2A2A44445F87
:10300000444440514A444040444A51400000FF017A
:1030100003E080FF000008086B6B08361236243688
:10302000060F090F060000181800000010100030ED
:1030300040FF0101001F01011E00191D1712003C75
:103040003C3C3C000000000000000A0B02090C0D93
:103050000E0807030401000000000000000000004B
:103060000000000000000000000000000000000060
:10307000000000001211100000000000000000001D
:103080000000000000000000000000000000185CCC
:10309000B15D11241FBECFEFD1E2DEBFCDBF00E096
:1030A0000CBF19E0A0E0B2E0EEE1FBEC00E00BBFEA
:1030B00002C007900D92AC3DB107D9F72EE0ACED00
:1030C000B9E001C01D92A135B207E1F718E1C8E4EB
:1030D000D8E100E006C021970109802FFE010E947F
:1030E0003763C734D10780E00807A9F70E94D75299
:1030F0000C947E650C940000089580E090E00895A3
:10310000CF92DF92EF92FF920F931F93CF93DF93B3
:10311000CDB7DEB72C970FB6F894DEBF0FBECDBF8C
:103120006B017C018A0166EA75E0CE0101960E947E
:10313000B924B701A601CE0101960E94AF236BEC22
:1031400075E0CE0101960E940E2420E030E040E1BF
:1031500051E4C701B6010E94086120E030E040EA76
:1031600050E40E94786220E030E040E052E40E94A7
:103170001462AB01BC01CE0101960E947F2360ED79
:1031800075E0CE0101960E940E24BE016F5F7F4F55
:10319000CE0107960E94A024CE0107960E942847E0
:1031A000CE0107960E949B246BED79E0CE0101963B
:1031B0000E94862463ED75E0CE0101960E940E24E4
:1031C000B801CE0101960E94DF2365EF75E0CE01C4
:1031D00001960E940E24BE016F5F7F4FCE010796BD
:1031E0000E94A024CE0107960E942847CE01079690
:1031F0000E949B24CE0101960E949B242C960FB620
:10320000F894DEBF0FBECDBFDF91CF911F910F911C
:10321000FF90EF90DF90CF900895CF92DF92EF92E2
:10322000FF920F931F93CF93DF93CDB7DEB72C9709
:103230000FB6F894DEBF0FBECDBF6B017C018A01D3
:1032400067EF75E0CE0101960E94B924B701A6018F
:10325000CE0101960E94AF236BEC75E0CE01019682
:103260000E940E2420E030E040E151E4C701B601A5
:103270000E94086120E030E040EA50E40E94786259
:1032800020E030E040E052E40E941462AB01BC0157
:10329000CE0101960E947F2360ED75E0CE0101967C
:1032A0000E940E24BE016F5F7F4FCE0107960E94E1
:1032B000A024CE0107960E942847CE0107960E94BF
:1032C0009B246BED79E0CE0101960E9486246CE18F
:1032D00076E0CE0101960E940E24B801CE0101963F
:1032E0000E94DF2365EF75E0CE0101960E940E2457
:1032F000BE016F5F7F4FCE0107960E94A024CE01D2
:1033000007960E942847CE0107960E949B24CE0173
:1033100001960E949B242C960FB6F894DEBF0FBE38
:10332000CDBFDF91CF911F910F91FF90EF90DF9074
:10333000CF9008958F929F92AF92BF92CF92DF92DB
:10334000EF92FF920F931F93CF93DF93CDB7DEB72A
:103350002C970FB6F894DEBF0FBECDBFEE24EA94D3
:10336000FE2C0EE316E02CED30E040E451E064E189
:1033700070E080E090E00E94D84611E010930A02CD
:1033800061E087E00E94C72561E087E00E94982500
:1033900068EE73E080E090E00E9422260E94FC2B01
:1033A0004B015C0180E00E94682B81E00E94682B49
:1033B0006B017C0165E576E0CE0107960E94B92499
:1033C000B501A401CE0107960E94AF2369E676E01D
:1033D000CE0107960E940E24B701A601CE010796E2
:1033E0000E94AF2360ED75E0CE0107960E940E2487
:1033F000BE01695F7F4FCE0101960E94A024CE01DD
:1034000001960E942847CE0101960E949B2480913C
:10341000DF098823D9F180E89BE00E941F3B6B0104
:103420007C0180E89BE00E94DD2A9C01A4E6B0E0DC
:103430000E9404622FEF33E040E050E00E94BC6144
:1034400049015A0121E7821627E19206A104B1043D
:10345000DCF020E030E040E85FE3C701B6010E9405
:10346000A36087FF11C01092DF0964EB73E0CE0107
:1034700001960E94B924CE0101960E942847CE01F0
:1034800001960E949B2434C0A4012FC066E380E80B
:103490009BE00E94082B882359F10E94F849109361
:1034A000DF096AE776E0CE0101960E94B924CE01D9
:1034B00001960E942847CE0101960E949B2480E835
:1034C0009BE00E941F3B6B017C0180E89BE00E9417
:1034D000DD2A9C01A4E6B0E00E9404622FEF33E0F5
:1034E00040E050E00E94BC61A901C701B60195DE31
:1034F0008091DE098823C9F187E79BE00E941F3B8A
:103500006B017C0187E79BE00E94DD2A9C01A4E619
:10351000B0E00E9404622FEF33E040E050E00E94F0
:10352000BC6149015A012137374141055105DCF0A1
:1035300020E030E040E85FE3C701B6010E94A360ED
:1035400087FF11C01092DE0962E074E0CE0101969F
:103550000E94B924CE0101960E942847CE0101960F
:103560000E949B2435C0A40130C067E387E79BE03D
:103570000E94082B882361F10E94F84981E0809322
:10358000DE096CE976E0CE0101960E94B924CE01F5
:1035900001960E942847CE0101960E949B2487E74E
:1035A0009BE00E941F3B6B017C0187E79BE00E9430
:1035B000DD2A9C01A4E6B0E00E9404622FEF33E014
:1035C00040E050E00E94BC61A901C701B60198DD4E
:1035D0008091DD098823D9F18EE69BE00E941F3B94
:1035E0006B017C018EE69BE00E94DD2A9C01A4E633
:1035F000B0E00E9404622FEF33E040E050E00E9410
:10360000BC6149015A0121E7821627E19206A10413
:10361000B104DCF020E030E040E85FE3C701B60130
:103620000E94A36087FF11C01092DD0960E574E07D
:10363000CE0101960E94B924CE0101960E9428472E
:10364000CE0101960E949B2436C0A40130C068E3DD
:103650008EE69BE00E94082B882369F10E94F849BE
:1036600081E08093DD096EEB76E0CE0101960E9449
:10367000B924CE0101960E942847CE0101960E94EE
:103680009B248EE69BE00E941F3B6B017C018EE633
:103690009BE00E94DD2A9C01A4E6B0E00E94046247
:1036A0002FEF33E040E050E00E94BC61A901C70168
:1036B000B6010E94974A8091DC098823C9F185E60A
:1036C0009BE00E941F3B6B017C0185E69BE00E9412
:1036D000DD2A9C01A4E6B0E00E9404622FEF33E0F3
:1036E00040E050E00E94BC6149015A012137374156
:1036F00041055105DCF020E030E040E85FE3C70120
:10370000B6010E94A36087FF11C01092DC096EE928
:1037100074E0CE0101960E94B924CE0101960E9468
:103720002847CE0101960E949B2436C0A40130C0D8
:1037300069E385E69BE00E94082B882369F10E94DB
:10374000F84981E08093DC0960EE76E0CE010196D5
:103750000E94B924CE0101960E942847CE0101960D
:103760000E949B2485E69BE00E941F3B6B017C012D
:1037700085E69BE00E94DD2A9C01A4E6B0E00E9461
:1037800004622FEF33E040E050E00E94BC61A901E9
:10379000C701B6010E940C4ACE0107960E949B24E5
:1037A0008091DF09882309F497C080E89BE00E949C
:1037B000DD2A9C01A4E6B0E00E9404626D3C7B4CD3
:1037C000810591050CF088C080910602882309F4D8
:1037D00083C080E89BE00E94DD2A9C01A4E6B0E063
:1037E0000E9404622FEF33E040E050E00E94BC6191
:1037F00062E370E0621B730B20910702072E000C3E
:10380000880B990B222309F442C20E94A9606B0124
:103810007C0120918E0230918F0245E0429FC001D1
:10382000439F900D1124BC01990F880B990B0E94A6
:10383000A96020E030E048EC52E40E9478629B01ED
:10384000AC01C701B6010E9408610E94E0628B01D1
:1038500062E077E0CE0101960E94B924B801012E02
:10386000000C880B990B0E94A96020E030E040E238
:1038700051E40E947862AB01BC01CE0101963FD7B2
:1038800067E277E0CE010196C9D7BE016F5F7F4F37
:10389000CE0107960E94A024CE0107960E942847D9
:1038A000CE0107960E949B2460E082E00E9498254A
:1038B00084E6809FB001819F700D1124072E000CBB
:1038C000880B990B0E94222661E082E00E949825D5
:1038D000CE0101960E949B248091DE09882309F481
:1038E00093C087E79BE00E94DD2A9C01A4E6B0E03C
:1038F0000E9404626D3C7B4C810591050CF084C0F4
:1039000080910402882309F47FC087E79BE00E942E
:10391000DD2A9C01A4E6B0E00E9404622FEF33E0B0
:1039200040E050E00E94BC6162E370E0621B730BF8
:1039300020910502072E000C880B990B222309F415
:10394000AFC10E94A9606B017C012091840230917B
:10395000850245E0429FC001439F900D1124BC01A8
:10396000990F880B990B0E94A96020E030E048EC89
:1039700052E40E9478629B01AC01C701B6010E942B
:1039800008610E94E0628B016DE277E0CE01019652
:10399000F0D7B801012E000C880B990B0E94A9608A
:1039A00020E030E040E251E40E947862AB01BC01CB
:1039B000CE010196A4D667E277E0CE0101962ED71C
:1039C000BE016F5F7F4FCE010796BAD7CE01079633
:1039D0000E942847CE010796AED760E083E00E94A0
:1039E000982584E6809FB001819F700D1124072ED9
:1039F000000C880B990B0E94222661E083E00E9454
:103A00009825CE01019697D78091DD09882309F486
:103A100093C08EE69BE00E94DD2A9C01A4E6B0E004
:103A20000E9404626D3C7B4C810591050CF084C0C2
:103A300080910202882309F47FC08EE69BE00E94F9
:103A4000DD2A9C01A4E6B0E00E9404622FEF33E07F
:103A500040E050E00E94BC6162E370E0621B730BC7
:103A600020910302072E000C880B990B222309F4E6
:103A700020C10E94A9606B017C0120917A023091E3
:103A80007B0245E0429FC001439F900D1124BC0181
:103A9000990F880B990B0E94A96020E030E048EC58
:103AA00052E40E9478629B01AC01C701B6010E94FA
:103AB00008610E94E0628B0162E577E0CE01019629
:103AC00058D7B801012E000C880B990B0E94A960F1
:103AD00020E030E040E251E40E947862AB01BC019A
:103AE000CE0101960CD667E277E0CE01019696D61C
:103AF000BE016F5F7F4FCE01079622D7CE0107969A
:103B00000E942847CE01079616D760E084E00E9405
:103B1000982584E6809FB001819F700D1124072EA7
:103B2000000C880B990B0E94222661E084E00E9421
:103B30009825CE010196FFD68091DC09882309F4EF
:103B400090C085E69BE00E94DD2A9C01A4E6B0E0DF
:103B50000E9404626D3C7B4C810591050CF081C094
:103B600080910002882309F47CC085E69BE00E94D6
:103B7000DD2A9C01A4E6B0E00E9404622FEF33E04E
:103B800040E050E00E94BC6162E370E0621B730B96
:103B900020910102072E000C880B990B222309F4B7
:103BA00091C00E94A9606B017C012091700230914C
:103BB000710245E0429FC001439F900D1124BC015A
:103BC000990F880B990B0E94A96020E030E048EC27
:103BD00052E40E9478629B01AC01C701B6010E94C9
:103BE00008610E94E0628B0167E777E0CE010196F1
:103BF000C0D6B801012E000C880B990B0E94A96059
:103C000020E030E040E251E40E947862AB01BC0168
:103C1000CE01019674D567E277E0CE010196FED51C
:103C2000BE016F5F7F4FCE0107968AD6CE01079601
:103C30000E942847CE0107967ED660E085E078D7BF
:103C400084E6809FB001819F700D1124072E000C27
:103C5000880B990BF7D761E085E06AD7CE01019612
:103C60006AD660E087E064D72C960FB6F894DEBF82
:103C70000FBECDBFDF91CF911F910F91FF90EF90BD
:103C8000DF90CF90BF90AF909F908F9008950E944B
:103C9000A9606B017C012091980230919902BDCD01
:103CA0000E94A9606B017C012091980230919902D9
:103CB00050CE0E94A9606B017C0120919802309146
:103CC0009902DFCE0E94A9606B017C0120919802CD
:103CD000309199026ECF8F929F92AF92BF92CF9206
:103CE000DF92EF92FF920F931F93CF93DF93CDB7A5
:103CF000DEB764970FB6F894DEBF0FBECDBF6CE998
:103D000077E0CE010F9635D654E1E52EF12C00E098
:103D100010E080E078D7080F191F6AE070E080E0BB
:103D200090E090D721E0E21AF10899F781E06BD793
:103D30008F3893401CF066EA77E030C0C80164E138
:103D400070E00E942463CB01770FAA0BBB0B9C0190
:103D5000AD012C53324041095109A4E6B0E00E9464
:103D6000D8612FE131E040E050E00E94BC61CA011F
:103D7000B9012AE08E010F5F1F4FA8010E94E65D86
:103D8000F80101900020E9F73197AF01401B510B7A
:103D9000B801CE010F9686D465EF75E0CE010F967F
:103DA0003DD5EE24EA94FE2C0BED19E024E130E041
:103DB00040EA50E060E070E080EA90E00E94D8467F
:103DC00022E030E042E050E062EA70E08F859889BE
:103DD0000E947D29E12C48EFF42E20E130E040E103
:103DE00050E062E070E08CE890E00E94D84683E208
:103DF00077D6892B71F420E2E22E2DEFF22E20E10E
:103E000030E040E150E062E070E08CE890E00E9439
:103E1000D84684E265D6892B81F490EEE92EFF2402
:103E2000FA940BED19E020E130E040E150E062E06F
:103E300070E08CE890E00E94D84685E251D6892B4C
:103E400081F480EEE82E87E0F82E0BED19E020E1FA
:103E500030E040E150E062E070E08CE890E00E94E9
:103E6000D84681E0D0D68F389340ECF0809137026D
:103E70009091380290936102809360028091410298
:103E800090914202909363028093620280914B0270
:103E900090914C0290935D0280935C028091550258
:103EA000909156021CC080910F0290911002909345
:103EB0006102809360028091190290911A0290939E
:103EC0006302809362028091230290912402909376
:103ED0005D0280935C0280912D0290912E0290935E
:103EE0005F0280935E020E94FC2B6B017C0181E0EB
:103EF0000E94682B4B015C018091620290916302E9
:103F0000BC01990F880B990B0E94A9609B01AC0121
:103F1000C501B4010E94116318164CF481E080932E
:103F2000F6098093F50961E08FE102D631C08091F6
:103F30005E0290915F02BC01990F880B990B0E9461
:103F4000A9609B01AC01C701B6010E94116318165C
:103F50002CF481E08093F50961E003C01092F5092B
:103F600060E08FE1E5D580915C0290915D02BC013B
:103F7000990F880B990B0E94A9609B01AC01C701A6
:103F8000B6010E94A36087FF05C081E08093F60917
:103F900061E003C01092F60960E08EE1C9D5CE0160
:103FA0000F96C9D464960FB6F894DEBF0FBECDBF8E
:103FB000DF91CF911F910F91FF90EF90DF90CF9005
:103FC000BF90AF909F908F9008958F929F92AF92E5
:103FD000BF92CF92DF92EF92FF920F931F93CF93F6
:103FE000DF93CDB7DEB7AD970FB6F894DEBF0FBE47
:103FF000CDBF63EB77E0CE010196BBD4CE01019635
:104000000E942847CE01019696D41092B60B1092CA
:10401000B50B8FEF9FEF9093B80B8093B70B0E9477
:10402000FC2B4B015C0180E00E94682B81E00E9428
:10403000682B6B017C016EE576E0CE01829699D407
:10404000B501A401CE0182968AD365EF75E0CE0159
:104050008296E4D3BE016E5D7F4FCE01019670D48F
:10406000AE014F5F5F4F6EE170E082E090E00E9432
:10407000BA2ACE0101965FD46CE676E0CE01829634
:1040800045D4B701A601CE01829669D361ED77E0F0
:10409000CE018296C3D3BE016E5D7F4FCE010196E5
:1040A0004FD4AE014F5F5F4F65E370E082E090E078
:1040B0000E94BA2ACE0101963ED4C090890BD090BE
:1040C0008A0BE0908B0BF0908C0BF4D580908D0BCD
:1040D00090908E0BA0908F0BB090900BC80CD91CB9
:1040E000EA1CFB1CA7019601261B370B480B590B3A
:1040F000CA01B90120E63AEE40E050E00E94E261D8
:10410000CA01B9016F5F7F4F8F4F9F4F19A618A645
:104110001BA61AA61DA61CA62AE0AE014F5F5F4F84
:104120000E94F45DBE016F5F7F4FCE018896EED393
:10413000BE01685D7F4FCE0182967ED3CE01889608
:10414000FAD36AED77E0CE01829668D3BE016E5D48
:104150007F4FCE010196F4D3AE014F5F5F4F6CE409
:1041600070E082E090E00E94BA2ACE010196E3D38B
:104170001092B80B1092B70B1092B60B1092B50BB1
:104180008091F609882329F060EEE62E67E0F62E8E
:1041900003C0E12C58EFF52E0FEE17E023E230E0DC
:1041A00046E950E064E670E085E090E00E94D84681
:1041B0008091F509882329F040EEE42E47E0F42EA3
:1041C00003C0E12C38EFF32E0AEF17E023E230E0D2
:1041D00046E950E064E670E085EA90E00E94D84647
:1041E000EE24EA94FE2C0BED19E025E030E046E9E0
:1041F00050E06DE770E085EA90E00E94D8469FE1CC
:10420000E92EF12C25E030E046E950E062E870E06C
:1042100085EA90E00E94D846EE24EA94FE2C2AE03B
:1042200030E046E950E06DE770E085E090E00E9404
:10423000D846CE0182967FD3AD960FB6F894DEBFF6
:104240000FBECDBFDF91CF911F910F91FF90EF90E7
:10425000DF90CF90BF90AF909F908F9008951F9266
:104260000F920FB60F9211248F930FB6F894A89562
:1042700080916000886180936000109260000FBEA2
:104280008F910F900FBE0F901F9018950895CF92A9
:10429000DF92EF92FF920F931F93CF93DF936C0106
:1042A0007A018B01C0E0D0E0CE15DF0589F0D8019E
:1042B0006D918D01D601ED91FC910190F081E02D81
:1042C000C6011995892B11F47E0102C02196ECCF0D
:1042D000C701DF91CF911F910F91FF90EF90DF9079
:1042E000CF900895FC01538D448D252F30E0842F0D
:1042F00090E0821B930B541710F0CF96089501970E
:104300000895FC01918D828D981761F0828DDF01F7
:10431000A80FB11D5D968C91928D9F5F9F73928FB8
:1043200090E008958FEF9FEF0895FC01918D828DAD
:10433000981731F0828DE80FF11D858D90E008957A
:104340008FEF9FEF0895FC01918D228D892F90E0D2
:10435000805C9F4F821B91098F739927089584E990
:104360009AE0F1DF21E0892B09F420E0822F089503
:10437000FC01848DDF01A80FB11DA35ABF4F2C9102
:10438000848D90E001968F739927848FA689B789D1
:104390002C93A089B1898C9180648C93938D848DAA
:1043A000981306C00288F389E02D80818F7D808379
:1043B0000895EF92FF920F931F93CF93DF93EC0139
:1043C00081E0888F9B8D8C8D981305C0E889F989D1
:1043D000808185FD23C0F62E0B8D10E00F5F1F4FEF
:1043E0000F731127E02E8C8DE8120BC00FB607FC5F
:1043F000FACFE889F989808185FFF5CFCE01B8DF52
:10440000F2CF8B8DFE01E80FF11DE35AFF4FF082D2
:104410000B8FEA89FB898081806207C0EE89FF8962
:104420006083E889F98980818064808381E090E0FD
:10443000DF91CF911F910F91FF90EF900895CF934F
:10444000DF93EC01888D8823C1F0EA89FB898081A4
:1044500085FD05C0A889B9898C9186FD0EC00FB66F
:1044600007FCF5CF808185FFF2CFA889B9898C91AF
:1044700085FFEDCFCE017CDFE8CFDF91CF910895AE
:1044800080E090E0892B19F06ADF811125C080E07F
:1044900090E0892B41F080E090E0892B21F00E9490
:1044A000000081111CC080E090E0892B41F080E089
:1044B00090E0892B21F00E940000811113C080E060
:1044C00090E0892BA1F080E090E0892B81F00E94A0
:1044D000000081110AC008950E940000D8CF0E94F8
:1044E0000000E1CF0E940000EACF0C940000089584
:1044F00090E0FC013197E231F10508F04EC08827C9
:10450000E658FF4F8F4F0C943763809180008F7770
:1045100003C0809180008F7D8093800008958091FA
:104520008000877FF9CF84B58F7702C084B58F7DF7
:1045300084BD08958091B0008F7703C08091B00052
:104540008F7D8093B0000895809190008F7707C091
:10455000809190008F7D03C080919000877F809331
:10456000900008958091A0008F7707C08091A000EF
:104570008F7D03C08091A000877F8093A000089565
:10458000809120018F7707C0809120018F7D03C02B
:1045900080912001877F8093200108953FB7F89490
:1045A0008091880A9091890AA0918A0AB0918B0A19
:1045B00026B5A89B05C02F3F19F00196A11DB11D7E
:1045C0003FBFBA2FA92F982F8827820F911DA11DB9
:1045D000B11DBC01CD0142E0660F771F881F991FF6
:1045E0004A95D1F7089585ED8093BC008091BC0079
:1045F00084FDFCCF10928E0A08950895E091920AEE
:104600008091910AE81730F4F0E0E850F64F80818D
:1046100090E008958FEF9FEF08959091920A809116
:10462000910A981750F4E92FF0E0E850F64F2081F6
:1046300030E09F5F9093920A02C02FEF3FEFC901D5
:1046400008958091910A90E02091920A821B91092D
:1046500008950E946A650F931F93CF93DF93EC0137
:1046600088819981009729F02A813B812617370795
:1046700088F48B016F5F7F4F0E948664009761F022
:10468000998388831B830A832C813D81232B11F41A
:10469000FC01108281E001C080E0DF91CF911F9189
:1046A0000F910895EF92FF920F931F93CF93DF9393
:1046B000FC01248135816115710511F480E018C079
:1046C00041155105A1F07B01EC018A01020F131F76
:1046D000B801C1DF882391F3288139818C819D81C4
:1046E000B701820F931F0E9477651D830C8381E0C1
:1046F000DF91CF911F910F91FF90EF900895EF926E
:10470000FF920F931F93CF93DF93CDB7DEB76497DC
:104710000FB6F894DEBF0FBECDBF7C01CB01BA014E
:104720008E010F5F1F4F22E044E00E94BD5DBC017F
:10473000FC0101900020E9F73197AF01481B590BAC
:10474000C701B0DF64960FB6F894DEBF0FBECDBFD1
:10475000DF91CF911F910F91FF90EF900895EF920D
:10476000FF920F931F93CF93DF93CDB7DEB764977C
:104770000FB6F894DEBF0FBECDBF7C01CB01BA01EE
:104780008E010F5F1F4F22E044E00E94BD5DBC011F
:10479000FC0101900020E9F73197AF01481B590B4C
:1047A000C70180DF64960FB6F894DEBF0FBECDBFA1
:1047B000DF91CF911F910F91FF90EF900895EF92AD
:1047C000FF920F931F93CF93DF93CDB7DEB7289758
:1047D0000FB6F894DEBF0FBECDBF7C01CB014AE01F
:1047E0008E010F5F1F4FB8010E94DC5DF801019040
:1047F0000020E9F73197AF01401B510BB801C70109
:1048000051DF28960FB6F894DEBF0FBECDBFDF9103
:10481000CF911F910F91FF90EF9008956115710551
:1048200049F0FB0101900020E9F73197AF01461BE9
:10483000570B38CF80E008950F931F93CF93DF93EA
:104840008C01EB01FC01808191810097B1F06881BE
:1048500079816115710579F0428153812C813D8107
:104860004217530740F00E9477658C819D81F801C3
:104870009583848313C00E94EE6388819981F80137
:10488000918380838A819B81938382838C819D81A4
:1048900095838483198218821B821A821D821C824E
:1048A000DF91CF911F910F910895CF93DF93EC018A
:1048B00088819981009711F00E94EE631982188215
:1048C0001D821C821B821A82DF91CF910895EF9284
:1048D000FF920F931F93CF93DF93EC017B018A012B
:1048E000BA01B9DE811103C0CE01DFDF07C01D832D
:1048F0000C83B701888199810E947765CE01DF9191
:10490000CF911F910F91FF90EF900895CF93DF9378
:10491000EC016115710551F0FB0101900020E9F7F0
:104920003197AF01461B570BD2DF01C0BEDFCE016E
:10493000DF91CF910895FC01808191810C94EE6309
:10494000FB01DC0111961C921E9213961C921E9282
:10495000129715961C921E9214978617970741F08E
:10496000608171816115710519F044815581AFCF66
:104970000895FC0111821082138212821582148222
:104980006115710549F0FB0101900020E9F73197AD
:10499000AF01461B570B9BCF0895BF92CF92DF927A
:1049A000EF92FF920F931F93CF93DF937C016B01E4
:1049B0008A01E9012417350720F4812F8901C42FCA
:1049C000D82F6BED79E0C701D4DFD60114968D9115
:1049D0009C91159708171907C8F48C179D0708F4C0
:1049E000EC01D601ED91FC911197EC0FFD1FB08009
:1049F00010824D915C91BA01600F711FC70186DF73
:104A0000D601ED91FC91EC0FFD1FB082C701DF9143
:104A1000CF911F910F91FF90EF90DF90CF90BF90BB
:104A200008951F920F920FB60F9211240BB60F929A
:104A30002F933F934F935F936F937F938F939F93A6
:104A4000AF93BF93EF93FF9384E99AE091DCFF91DA
:104A5000EF91BF91AF919F918F917F916F915F91F6
:104A60004F913F912F910F900BBE0F900FBE0F9063
:104A70001F9018951F920F920FB60F9211240BB62C
:104A80000F922F938F939F93EF93FF93E091A40A3C
:104A9000F091A50A8081E091AA0AF091AB0A82FD0B
:104AA00012C090818091AD0A8F5F8F732091AE0A02
:104AB000821751F0E091AD0AF0E0EC56F54F958F7A
:104AC0008093AD0A01C08081FF91EF919F918F91FA
:104AD0002F910F900BBE0F900FBE0F901F90189547
:104AE000CF93DF93282F30E0F901E85BFF4C8491EE
:104AF000F901E95FF44DD491F901EF53F54DC491FB
:104B0000CC2389F08111F4DCEC2FF0E0EE0FFF1FD5
:104B1000E05AF54DA591B491EC91ED2381E090E040
:104B200021F480E002C080E090E0DF91CF91089511
:104B30001F93CF93DF93282F30E0F901E85BFF4C00
:104B40008491F901E95FF44DD491F901EF53F54DEA
:104B5000C491CC23C1F0162F8111CADCEC2FF0E0F8
:104B6000EE0FFF1FE955F54DA591B4918FB7F8945D
:104B7000111105C09C91ED2FE095E92302C0EC9145
:104B8000ED2BEC938FBFDF91CF911F910895CF93C1
:104B9000DF9390E0FC01E95FF44D2491FC01EF53B9
:104BA000F54D8491882361F190E0880F991FFC01F5
:104BB000EA5BFD4FC591D491FC01E955F54DA591F6
:104BC000B491611109C09FB7F89488812095822320
:104BD0008883EC912E230BC0623061F49FB7F89468
:104BE0003881822F809583238883EC912E2B2C9300
:104BF0009FBF06C08FB7F894E8812E2B28838FBF04
:104C0000DF91CF910895863308F0865390917B0011
:104C1000282F2870977F922B90937B008770806459
:104C200080937C0080917A00806480937A008091E8
:104C30007A0086FDFCCF809178002091790090E089
:104C4000922B08958F929F92AF92BF92CF92DF9254
:104C5000EF92FF926B017C01A1DC4B015C01C1145E
:104C6000D104E104F104E9F099DCDC01CB018819FD
:104C70009909AA09BB09883E9340A105B10578F3BB
:104C800021E0C21AD108E108F10888EE880E83E01D
:104C9000981EA11CB11CC114D104E104F10421F738
:104CA000DECFFF90EF90DF90CF90BF90AF909F90BE
:104CB0008F9008952FB7F8946091840A7091850AB7
:104CC0008091860A9091870A2FBF08951F920F92B4
:104CD0000FB60F9211242F933F938F939F93AF930F
:104CE000BF938091840A9091850AA091860AB09121
:104CF000870A3091830A23E0230F2D3720F4019691
:104D0000A11DB11D05C026E8230F0296A11DB11DEE
:104D10002093830A8093840A9093850AA093860A3D
:104D2000B093870A8091880A9091890AA0918A0A93
:104D3000B0918B0A0196A11DB11D8093880A9093B2
:104D4000890AA0938A0AB0938B0ABF91AF919F9171
:104D50008F913F912F910F900FBE0F901F9018953C
:104D60001F920F920FB60F9211240BB60F922F9332
:104D70003F934F935F936F937F938F939F93AF93E3
:104D8000BF93EF93FF938091B900887F803609F439
:104D90009CC068F5883209F45BC090F4803109F456
:104DA00054C038F4882309F4F6C0883009F44DC0A3
:104DB000F5C0883109F44CC0803209F45DC0EEC002
:104DC000803409F468C048F4803309F455C088334E
:104DD00009F0E4C08093180AD8C0803509F44FC0A8
:104DE000883509F45DC0883409F0D8C0D6C0883948
:104DF00009F4C7C0A8F4883709F467C038F48836C6
:104E000009F463C0803709F460C0C8C0883809F469
:104E1000B8C0803909F45FC0803809F0BFC05BC0FA
:104E2000803B09F486C038F4803A09F466C0883AB9
:104E300009F47FC0B3C0803C09F4A7C0883C09F4E2
:104E4000A4C0883B09F48AC0A9C080913B0A10C065
:104E500090913A0A8091390A981770F5E0913A0AD0
:104E600081E08E0F80933A0AF0E0E75EF54F808193
:104E70008093BB0085EC86C08093180A8EC0E091B9
:104E80003A0A81E08E0F80933A0A8091BB00F0E0ED
:104E9000E75EF54F808390913A0A8091390A6EC09F
:104EA000E0913A0A81E08E0F80933A0A8091BB002C
:104EB000F0E0E75EF54F808380918D0A81116DC02F
:104EC00081E080938C0A84EA61C083E080938E0A3B
:104ED0001092820ACFCF8091820A803208F051C0AE
:104EE000E091820A81E08E0F8093820A8091BB005C
:104EF000F0E0EE59F54F8083BDCF85EC8093BC0088
:104F000010928E0A8091820A803230F4E091820AF7
:104F1000F0E0EE59F54F10826091820A70E0E09166
:104F2000600AF091610A82E69AE019951092820A6D
:104F300035C084E080938E0A10925F0A10925E0A58
:104F4000E0915C0AF0915D0A199580915E0A8111E9
:104F500005C081E080935E0A10923C0AE0915F0AEE
:104F600081E08E0F80935F0AF0E0E45CF54F808172
:104F70008093BB0090915F0A80915E0A981708F4B5
:104F800079CF85E88093BC0009C085EC8093BC0094
:104F900010928E0A03C01092180A25DBFF91EF9140
:104FA000BF91AF919F918F917F916F915F914F9141
:104FB0003F912F910F900BBE0F900FBE0F901F903F
:104FC000189540915E0A262F30E0240F311D2132C2
:104FD0003105DCF420918E0A2430C9F4FC0180E014
:104FE00090E0861758F430915E0A2191DC01A45CB0
:104FF000B54FA30FB11D2C930196F3CF80915E0A9C
:10500000680F60935E0A80E0089581E0089582E071
:105010000895CF92DF92EF92FF920F931F93CF9359
:10502000DF937C01262F972F8A018091F70988232F
:1050300091F0C62FD72F6E01C40ED51ECC15DD05FD
:1050400069F06991D701ED91FC910190F081E02D1B
:10505000C7011995F3CF642F822FB3DFC801DF9109
:10506000CF911F910F91FF90EF90DF90CF90089517
:10507000CF92DF92EF92FF92CF93DF93B091CB0B61
:10508000882311F0AB2F01C0A0E08091CC0B90E001
:10509000880F991F805A954DC090D10BD090D20B9C
:1050A000E090D30BF090D40B20E030E0FC01C591F0
:1050B000D491E881EB23A90160E070E0EA130CC011
:1050C0002F5F3F4F4C155D056E057F0578F33FEF71
:1050D0002FEF8FEF9FEF03C0322F252FCB01632FD0
:1050E000722FDF91CF91FF90EF90DF90CF900895D6
:1050F0009CB52091A50B2CBD8EBD00000DB407FE04
:10510000FDCF9CBD0895CF92DF92EF92FF920F9357
:105110001F93CF93DF93CDB7DEB7C054D1400FB606
:10512000F894DEBF0FBECDBFC5DD0091CD0B109151
:10513000CE0B2091CF0B3091D00B6B017C01C01AAC
:10514000D10AE20AF30A40EDC41647E0D406E104AE
:10515000F10418F48091D50BC0C06093CD0B70930F
:10516000CE0B8093CF0B9093D00B1092C80B109264
:10517000C70B1092C60B1092C50B1092C40B62E0C5
:105180008091C90B04DD61E070E080E090E05ADDC1
:1051900061E08091C90BFBDC60E08091C90BC8DC49
:1051A0008091CA0B8551823028F48BE291E10197FE
:1051B000F1F705C064E170E080E090E043DD62E07B
:1051C0008091C90BE4DC8091D60B90E08230910590
:1051D00038F0880F991F880F991F05970197F1F7ED
:1051E000F89480E045DF6F3F7F4F8F4F9F4F21F452
:1051F0001092D50B78943EC081E03ADF6F3F7F4F2D
:105200008F4F9F4FA9F38E010F5F1F4F6E012FEB42
:10521000C21A2EEFD20A780180E02ADFF7016083FC
:1052200071838283938381E023DFF7016483758335
:1052300086839783F8E0EF0EF11CEC14FD0461F710
:10524000789420E030E0F8014081518162817381DF
:10525000C480D580E680F7804F3FFFEF5F076F0780
:105260007F0731F08FEFC816D806E806F80621F45C
:105270001092D50B80E031C0F90183E0F595E795F8
:105280008A95E1F7EC53F44F8081880F4C155D054A
:105290006E057F0508F4816080832F5F3F4F085FB4
:1052A0001F4F2832310579F62091C80B30E040912C
:1052B000C40B8091C50B90E0840F911D4091C60BEB
:1052C000840F911D4091C70B840F911D99272817BA
:1052D000390771F681E08093D50BC05CDE4F0FB6C5
:1052E000F894DEBF0FBECDBFDF91CF911F910F911C
:1052F000FF90EF90DF90CF9008954F925F926F9262
:105300007F928F929F92AF92BF92CF92DF92EF9255
:10531000FF920F931F93CF93DF931F92CDB7DEB70A
:10532000A82F2B016A0179014091C10B411107C0DF
:105330002091AF0B3091B00B232B09F4A4C097013F
:10534000225031092730310538F585E08E9DF00176
:105350008F9DF00D1124E458F54DA590B49080E296
:10536000A81AB1082A2F392F60E070E0F901819165
:105370009F01882349F0F501E80FF11D87FDFA959B
:10538000E4916E0F711DF2CF8091C00B869F90014A
:10539000879F300D112402C020E030E085E08E9D13
:1053A000F0018F9DF00D1124E258F54DE491A0908D
:1053B000C00BEA9D5001112450E0FA013197E8300A
:1053C000F105E0F58827E457FF4F8F4F0C943763C2
:1053D000A90156954795441A550A26C0421A530A00
:1053E0002AC0A50156954795C41AD50A27C0A90118
:1053F00056954795441A550AA50156954795C41ADE
:10540000D50A12C0421A530AA50156954795C41AE7
:10541000D50A11C0CA18DB0811C0A90156954795D5
:10542000441A550ACA18DB08F2E0F98309C0421A87
:10543000530ACA18DB0883E0898302C0E1E0E983EC
:1054400057FE02C0412C512C4091B10B5091B20B30
:10545000B201620F731F4617570718F42A01421A48
:10546000530AD7FE02C0C12CD12C2091B30B30912E
:10547000B40BA6014A0D5B1D2417350740F46901E2
:10548000CA18DB0804C0A12CB12CF1E0F9836A2E04
:10549000792E812C912CF30161913F01662371F0EB
:1054A000A201480D591D062E000C770B87019601AD
:1054B0008FE99BE025D3880E991EEDCF2091AF0B8D
:1054C0003091B00B821693060CF041C0E090B70B00
:1054D000F090B80B8091B50B9091B60B8E159F058F
:1054E000B1F1B201680D791DF981F23029F0F33084
:1054F000F9F02819390926C0281939093595279551
:105500008501A6018FE99BE0A2D22091AF0B3091DB
:10551000B00B2819390935952795E090B70BF09015
:10552000B80BC901421653060CF4C201B20108C0FF
:10553000CB01261737070CF4C9019C01281939093A
:10554000681B790B8501A6018FE99BE080D2C4011D
:105550000F90DF91CF911F910F91FF90EF90DF900F
:10556000CF90BF90AF909F908F907F906F905F9003
:105570004F900895FA012091930A211107C024E069
:1055800030E0AB01BC0180819181B7CE0895EF92EC
:10559000FF920F931F93EFE9FBE00489158922899D
:1055A00033897C0140E050E060E070E0CF014FD2F1
:1055B0001F910F91FF90EF900895EF92FF920F933C
:1055C0001F93CF93DF931F921F92CDB7DEB728EEC4
:1055D000E22E23E0F22E02E09E012F5F3F4F40E1DA
:1055E0006FE00E94CB39098110E0102F00278A81DB
:1055F000082B61E070E080E090E024DBC8010F90B0
:105600000F90DF91CF911F910F91FF90EF90089530
:10561000CF92DF92EF92FF920F931F93CF93DF937E
:105620001F921F92CDB7DEB76C01FC0164831FEFA0
:1056300017831092920A1092910A1092900A109277
:105640008F0A10928E0A81E080938D0A10928C0A44
:1056500061E084E16DDA61E085E16ADA8091B900A8
:105660008E7F8093B9008091B9008D7F8093B900BF
:1056700088E48093B80085E48093BC001A8301E03D
:105680009E012E5F3F4F4FE760E0C6010E94CA387F
:1056900064EF71E080E090E0D5DA8DE7E82EF12C40
:1056A0009E012F5F3F4F41E060E0C6010E94CB3971
:1056B000998181E0953509F080E00F900F90DF919E
:1056C000CF911F910F91FF90EF90DF90CF900895B1
:1056D000CF92DF92EF92FF92CF93DF93C82F13DD2B
:1056E000882309F47EC08091CA0B8C3009F449C02C
:1056F00018F48B30D1F075C08551823008F071C03C
:10570000D091C60B6D2F6F7770E0762F6627809152
:10571000C70B682B80E090E00E94A7602DEC3CEC6A
:105720004CEC5DE30E9408614BC06091C60B70E0D9
:1057300080E090E00E94A7606B017C01D091C70BD4
:10574000D7FF0AC09B01AC0160E070E080E89FEBEE
:105750000E9413626B017C018D2F8F70682F70E0A7
:1057600080E090E00E94A9602DEC3CEC4CEC5DE305
:105770000E9408619B01AC01C701B6010E9414623E
:1057800021C0D091C60B6D2F70E080E090E00E94A8
:10579000A7606B017C018091C70B8F70682F70E050
:1057A00080E090E00E94A9602DEC3CEC4CEC5DE3C5
:1057B0000E9408619B01AC01C701B6010E941462FE
:1057C000D7FD9058CC2389F026E636E646EE5FE317
:1057D0000E94086120E030E040E052E40E94146240
:1057E00004C060E070E080EC9FE7DF91CF91FF9014
:1057F000EF90DF90CF900895CF92DF92EF92FF92DB
:1058000082DC8823D1F18091CA0B8B30B0F18D30CE
:10581000B0F08551823088F56091C40B70E0762F2E
:1058200066278091C50B682B80E090E00E94A760FE
:105830002DEC3CEC4CEC5DE30E94086122C06091D1
:10584000C40B70E080E090E00E94A9606B017C01D5
:105850008091C50B682F70E080E090E00E94A96005
:105860002DEC3CEC4CEC5DE30E9408619B01AC012B
:10587000C701B6010E94146204C060E070E080ECD1
:105880009FE7FF90EF90DF90CF90089580E591E043
:10589000DBD680910B018D7F80930B0180910B01F2
:1058A0008E7F80930B018AE28EBD00960096009653
:1058B00001D001C0089580910B01826080930B019B
:1058C0001EBC00000096009601D001C00895109201
:1058D000BE0B1092BD0B1EBC0000009601D001C093
:1058E00008958091B10B9091B20B01979093AC0BFE
:1058F0008093AB0B9EBD00960096009601D001C030
:1059000008958EBD00000096009601D001C0089554
:1059100080910B018D7F80930B018BE28EBD0096F1
:105920000096009601D001C0089580910B0182601D
:1059300080930B011EBC00000096009601D001C0B0
:1059400008951092BC0B1092BB0B1EBC0000009679
:1059500001D001C008958091B30B9091B40B0197D1
:105960009093AE0B8093AD0B9EBD00960096009673
:1059700001D001C008958EBD00000096009601D0B0
:1059800001C0089580910B01816080930B010DB4DB
:1059900007FEFDCF58C6CF93DF93CBE0D1E09881CF
:1059A0009260988398819E7F9883A2DB8881816032
:1059B0008883DF91CF910895CF93DF939DB5909326
:1059C000A60BCBE0D1E098819D7F988398819E7F44
:1059D00098838EDB888181608883DF91CF910895E1
:1059E000AF92BF92CF92DF92EF92FF920F931F93ED
:1059F000CF93DF93E4E6F2E0C081D181C280D3800F
:105A0000A680B78044815581E12CF12C0BED19E083
:105A100024E130E0B601CE010E94D84680EEE82EA7
:105A200087E0F82E24E130E044E150E0B601CE01F9
:105A30008A0D9B1D0E94D846DF91CF911F910F9137
:105A4000FF90EF90DF90CF90BF90AF9008958F922E
:105A50009F92AF92BF92CF92DF92EF92FF920F93FD
:105A60001F93CF93DF9300D01F92CDB7DEB75C01B9
:105A70006901480180E591E04B835C8369837A8307
:105A8000E3D54B815C818A01080D191D0150110974
:105A900069817A819B012C0D3D1D21503109C50181
:105AA00047D581E0881A910890F0C601009771F0FF
:105AB000FEBC02D001D001C008950000EEBC0096EB
:105AC000009601D001C00895019791F7EACF809127
:105AD0000B01816080930B010DB407FEFDCF0F9089
:105AE0000F900F900F90DF91CF911F910F91FF902A
:105AF000EF90DF90CF90BF90AF909F908F90A3C515
:105B00002F923F924F925F926F927F928F929F92CD
:105B1000AF92BF92CF92DF92EF92FF920F931F93BB
:105B2000CF93DF93CDB7DEB766970FB6F894DEBF9D
:105B30000FBECDBF1C017B0158874F832901FC019B
:105B4000008CF18DE02DFC87EB87FC01C688D7889F
:105B50000130110509F003C1F1A1FD87FC01828923
:105B60009389481759070CF0F3C084899589281741
:105B700039070CF0EDC0FD85AF2EB12CCA0106E04F
:105B8000F09F800D911D1124181619060CF0E0C02D
:105B9000C50163E0880F991F6A95E1F7840D951D93
:105BA000181619060CF0D4C031E0398B4B855C8592
:105BB0004C155D0509F4198A80E591E045D5FF246F
:105BC0005D85513009F05DC06989662309F459C0CB
:105BD0008201085F1F4F2F8138852B5F3F4FA20145
:105BE0006F817885C101A4D485E08E9DA0018F9D31
:105BF000500D11249E012F5F3F4FD90180E090E0AE
:105C0000FC01E40FF51FE35BF44DE491ED93019685
:105C100085309105A9F71E826D2D5C8598E081E0A5
:105C200075E0720FF9014191482351F00DB407FE60
:105C3000FDCF6EBD00000DB407FEFDCFCEBC0AC087
:105C40000DB407FEFDCF5EBD00000DB407FEFDCF15
:105C50000B850EBD7E13E7CF880F0DB407FEFDCF79
:105C60005EBD0DB407FEFDCF4B854EBD9150D1F604
:105C70000DB407FEFDCF80910B01816080930B0175
:105C800063C085E08E9DB0018F9D700D11247E8BC9
:105C90006D8B8F819885988B8F87812C912C95E0C7
:105CA0008916910449F0ED89FE89E80DF91DE35B41
:105CB000F44D0491098701C019862D85213029F5FD
:105CC000720118E06F807884680C791C398530FF88
:105CD00005C09601A701B301C101B9D44985469514
:105CE000498711505FEFE51AF50A1111EFCF6FEFF9
:105CF000861A960A8F8598898A0D9B1D988B8F87A7
:105D000096E08916910459F61FC03201E8E0EB8B4A
:105D1000F985F0FF02C0760105C00989002349F02A
:105D2000EB84FC8485019501A3016F857889C1010D
:105D30008EDE2985269529873B8931503B8B6A0C5D
:105D40007B1C3111E5CFD3CF0DB407FEFDCF7BD443
:105D5000F10181A1F6E08F9FC001112448C3605278
:105D60007109CB01880F991F0230110599F4FC01CC
:105D7000E056F64D259134913E872D87FB01E05C7E
:105D8000F64DE4914E2F50E05A87498740E1642E4A
:105D9000712C25C045E0409F9001419F300D11249A
:105DA000F901E658F54D45915491FA01E80FF91FB4
:105DB000859194919E878D87F901E458F54D8591E1
:105DC0009491FC01E60FF71FE4914E2F50E05A87A3
:105DD0004987F901E258F54DE4916E2E712CC98A7C
:105DE000DB8A0230110509F0D1C1F10121A14985F9
:105DF0005A85249FC001259F900D11246F817885BD
:105E0000680F791F42895389641775070CF0EFC238
:105E100089859A850696BC0133E0759567953A9514
:105E2000E1F7788B6F878B859C85C816D90619F0AA
:105E3000213009F447C11C8A1B8A1A8A198A698988
:105E40007A896615770509F4C9C2F101E08CF18CF5
:105E5000868997898E159F0581F001A110E04985FB
:105E60005A85409F9001419F300D509F300D112465
:105E7000A2016F817885C101EADD6B897C898D85FE
:105E80009E85680F791F7E8B6D8BAF80B8841C86D2
:105E90001B864B855C856F8578894617570709F403
:105EA00000C1EB85FC852D893E89E20FF31F94909C
:105EB000992009F4ECC0F10121A1213009F056C06C
:105EC00097FE06C026893789A201B501C101BFD35B
:105ED00096FE09C0F10126893789A201B5016F5FDD
:105EE0007F4FC101B4D395FE09C0F10126893789DE
:105EF000A201B5016E5F7F4FC101A9D394FE09C015
:105F0000F10126893789A201B5016D5F7F4FC1017B
:105F10009ED393FE09C0F10126893789A201B501FC
:105F20006C5F7F4FC10193D392FE09C0F1012689B6
:105F30003789A201B5016B5F7F4FC10188D391FE04
:105F400009C0F10126893789A201B5016A5F7F4F37
:105F5000C1017DD390FE9BC0F10126893789A20142
:105F6000B501695F7F4FC10172D391C030E0C501B7
:105F70004F815885841B950B829F6001839FD00CB5
:105F8000929FD00C1124C40ED51E97FE08C0F101BB
:105F9000E688F7888901A201B601C10158DD96FEA5
:105FA0000CC0F10121A130E0E688F788B601620F4C
:105FB000731F8901A201C1014ADD95FE0EC0F101E6
:105FC00021A130E0E688F788B901660F771F6C0DD4
:105FD0007D1D8901A201C1013ADD94FE10C0F101CD
:105FE00081A1282F30E0E688F788B601F3E08F9F83
:105FF000600D711D11248901A201C10128DD93FEEC
:1060000010C0F10181A1E688F788282F30E0B601A1
:10601000F4E08F9F600D711D11248901A201C1015F
:1060200016DD92FE10C0F10181A1282F30E0E68834
:10603000F788B601F5E08F9F600D711D112489016D
:10604000A201C10104DD91FE10C0F10181A1282F40
:1060500030E0E688F788B601F6E08F9F600D711D8D
:1060600011248901A201C101F2DC90FE10C0F101EE
:1060700081A1282F30E0E688F788B601F7E08F9FEE
:10608000600D711D11248901A201C101E0DC2B8585
:106090003C852F5F3F4F3C872B8738E0A30EB11C18
:1060A000F8CEF10181A1480E511C29893A892F5F50
:1060B0003F4F3A8B298B4B895C89460F571F5C8B6E
:1060C0004B8BBDCE80E591E0BFD28201060D171D3E
:1060D000015011092F85388983E0220F331F8A95DB
:1060E000E1F78F819885280F391F21503109A201CE
:1060F000BC01C1011DD21C8520E030E040E050E031
:106100004615570509F435C0AD85BE85A20FB31FEE
:1061100080E090E06F8578898617970729F1FC0168
:10612000EA0FFB1FE49168E070E0F0E80F2F0E2308
:1061300059F00DB407FEFDCF0B890EBD00000DB464
:1061400007FEFDCF098909C00DB407FEFDCF1EBDB6
:1061500000000DB407FEFDCF0B850EBDF695615016
:10616000710921F70196D6CF4F5F5F4F260F371F7A
:10617000C7CF0DB407FEFDCF80910B0181608093E6
:106180000B010DB407FEFDCF5ED228C180E591E082
:106190005BD21EBC89859A85869D4001879D900CA7
:1061A000969D900C1124F10181A1E08CF18C26893F
:1061B0003789813021F42E153F0509F0BEC02E1518
:1061C0003F05B1F090E0869D8001879D100D969D62
:1061D000100D112449855A85489F9001499F300D23
:1061E000589F300D1124A2016F817885C1012FDCE9
:1061F000F101C1A0CC9CF02D1124FD8BCA94612C1F
:10620000712C2C2D30E0388B2F87681479040CF01A
:1062100088C0ED85FE8584913196FE87ED8787FFE6
:106220007CC08F77DD24D394D80ECC20F1F0F1011F
:1062300021A130E0C30169857A850E942463289FEB
:106240007001299FF00C389FF00C11244F81588564
:10625000E40EF51E269F5001279FB00C369FB00C10
:106260001124A40CB51CDB8639C0C30169857A856D
:106270000E942463EF80F884E80EF91E5201A60EF6
:10628000B71EF1CF0DB407FEFDCF0F8518890A0D9B
:106290001B1D2F8538892E0D3F1DA501B701C1019A
:1062A00047D1CC2061F18D898150F0F4F10181A1B9
:1062B00090E0E80EF91E49855A85489F9001499F54
:1062C000300D589F300D11246F817885260F371FB0
:1062D000E216F3061CF0A80EB91E7B017B857150F7
:1062E0007B877F3F79F616C00DB407FEFDCF5B8933
:1062F0005EBD0DB407FEFDCF69896EBDD5CF0DB46F
:1063000007FEFDCF7B897EBD0DB407FEFDCF8989D9
:106310008EBDCCCF6D0C711C78CF8F5F680E711C59
:1063200074CF0DB407FEFDCF80910B018160809387
:106330000B010DB407FEFDCF27CF80E591E084D19E
:106340008201060D171D015011092F81388589859D
:106350009A85280F391F21503109A2016F81788554
:10636000C101E6D0181419040CF02CC02D853E850F
:106370002F5F3F4FED85FE85849187FF09C08F77A2
:106380008F5F90E0881A990AF1014689578907C002
:106390008F5F90E0881A990AF101408D518D009726
:1063A00071F05EBD02D001D001C0089500004EBD65
:1063B0000096009601D001C00895019791F73E879D
:1063C0002D87D0CF0DB407FEFDCF80910B018160EA
:1063D00080930B010DB407FEFDCFD6CEF10121A1B4
:1063E00049855A85249FC001259F900D11246696EA
:1063F0000FB6F894DEBF0FBECDBFDF91CF911F91D6
:106400000F91FF90EF90DF90CF90BF90AF909F9053
:106410008F907F906F905F904F903F902F90089556
:106420000F931F93CF93DF93DC01462F6D3009F458
:1064300078C090960C91909770E0023051F4FB0177
:10644000E05EF64D849190E00696887FE0E1F0E012
:106450001BC085E0089F90011124F901E458F54D17
:1064600085919491FB01B097E80FF91F8491F90190
:10647000E258F54DE491013019F090E0F0E004C0ED
:10648000E8E0F0E086E090E09196CC919197D0E042
:10649000EC9F9001ED9F300DFC9F300D11241A965A
:1064A000ED91FC911B974A3059F42E0F3F1F1B961C
:1064B0003C932E931A9719961C921E92189731C0EE
:1064C00094964C9194974423F1F08C9FA0018D9F5A
:1064D000500D9C9F500D112418968D919C911997E9
:1064E000840F951F52964D915C9153978417950791
:1064F00050F02E0F3F1F1B963C932E931A97199620
:106500001C921E921897ED0110E02A853B85488564
:106510005985CD01F5DA28853985820F931F998732
:10652000888781E090E0DF91CF911F910F910895CE
:106530000F931F93FC0180910B018D7F80930B01C2
:1065400080910B018E7F80930B018AE28EBD0096B5
:106550000096009601D001C0089580910B018260E1
:1065600080930B017EBD0000009601D001C008950C
:106570008FEF9FEF978F868F6EBD0000009601D042
:1065800001C00895848595852817390781F03EBD9F
:106590000000009601D001C00895000035872487CF
:1065A0002EBD00000096009601D001C00895809194
:1065B0000B018D7F80930B018BE28EBD00960096C0
:1065C000009601D001C0089580910B0182608093F4
:1065D0000B015EBD0000009601D001C008958FEF51
:1065E0009FEF958F848F4EBD0000009601D001C0B3
:1065F0000895868597850817190781F01EBD00004C
:10660000009601D001C008950000178706870EBDCF
:1066100000000096009601D001C0089580910B0102
:106620008D7F80930B018CE28EBD0000009600965A
:1066300001D001C0089580910B01826080930B010D
:106640001F910F91089508958CBD9DBD0895CF921F
:10665000DF92EF92FF920F931F93CF93DF931F92DE
:106660001F92CDB7DEB76C017B018A01FC018289E4
:1066700093896817790708F0A3C08489958948171A
:10668000590708F09DC080E591E029833A83DCDF5B
:1066900080910B018E7F80930B01F601868D978D83
:1066A00029813A818E159F0509F42BC080910B0139
:1066B0008D7F80930B018AE28EBD0000009601D091
:1066C00001C00895F78EE68E80910B018260809361
:1066D0000B01FEBC02D001D001C008950000EEBC49
:1066E00002D001D001C008950000FEBC02D001D04C
:1066F00001C008950000EEBC0000009601D001C06A
:106700000895F601848D958D8017910709F42CC0AA
:1067100080910B018D7F80930B018BE28EBD000079
:10672000009601D001C00895158F048F80910B0150
:10673000826080930B011EBD02D001D001C008957C
:1067400000000EBD02D001D001C0089500001EBDA2
:1067500002D001D001C0089500000EBD00000096D7
:10676000009601D001C0089580910B018D7F809328
:106770000B018CE28EBD00960096009601D001C000
:10678000089580910B01826080930B013EBD0096BD
:106790000096009601D001C00895F601F586E486C2
:1067A0002EBD0000009601D001C00895178706870E
:1067B00080910B01816080930B010DB407FEFDCF2A
:1067C0000F900F90DF91CF911F910F91FF90EF905D
:1067D000DF90CF900895CF92DF92EF92FF920F93C8
:1067E0001F93CF93DF93FC0122852223A9F1EC01B3
:1067F0000E945A266B017C018C819D81AE81BF81F4
:106800000097A105B10509F1488159816A817B8111
:1068100097018601081B190B2A0B3B0B0417150760
:106820002607370790F4C816D906EA06FB06A0F437
:1068300080959095A095B0958C199D09AE09BF09DA
:1068400084179507A607B70738F0E885F9851995E5
:10685000CC82DD82EE82FF82DF91CF911F910F917A
:10686000FF90EF90DF90CF900895EF92FF920F93FB
:106870001F93CF93DF9300D000D0CDB7DEB7813028
:10688000910509F041C080910702811123C08091D8
:1068900098029091990290938F0280938E028AE8D9
:1068A00092E00E949C4320918E0230918F02809151
:1068B0009802909199022817390709F4FDC081E0E8
:1068C000809307028091200C9091210C019709F090
:1068D00006C1CBC08AE892E00E949C4320918E02C0
:1068E00030918F0280919802909199022817390770
:1068F00009F0F5C0109207028091200C9091210CB4
:10690000019709F0ECC0D8C08230910509F041C070
:1069100080910502811123C0809198029091990283
:10692000909385028093840280E892E00E949C43C9
:106930002091840230918502809198029091990271
:106940002817390709F4B8C081E0809305028091C7
:10695000200C9091210C029709F0C1C086C080E8FC
:1069600092E00E949C4320918402309185028091A4
:106970009802909199022817390709F0B0C0109237
:1069800005028091200C9091210C029709F0A7C07C
:1069900093C08330910509F041C0809103028111B9
:1069A00023C0809198029091990290937B028093EA
:1069B0007A0286E792E00E949C4320917A0230910D
:1069C0007B0280919802909199022817390709F467
:1069D00073C081E0809303028091200C9091210C80
:1069E000039709F07CC041C086E792E00E949C4377
:1069F00020917A0230917B028091980290919902C5
:106A00002817390709F06BC0109203028091200CFF
:106A10009091210C039709F062C04EC0049709F0D1
:106A20005EC080910102811130C0809198029091E6
:106A3000990290937102809370028CE692E00E941A
:106A40009C43209170023091710280919802909144
:106A500099022817390781F181E080930102809122
:106A6000200C9091210C0497D1F5EE24EA94FE2C91
:106A70000BED19E02EE130E044E650E06FE570E008
:106A80008FE090E00E94D8462AC08CE692E00E94F7
:106A90009C432091700230917102809198029091F4
:106AA000990228173907D9F4109201028091200C1D
:106AB0009091210C049799F466E078E0CE0101965C
:106AC0000E94B924AE014F5F5F4F6FE570E08FE029
:106AD00090E00E94BA2ACE0101960E949B2426963D
:106AE0000FB6F894DEBF0FBECDBFDF91CF911F91DF
:106AF0000F91FF90EF900895CF92DF92EF92FF9267
:106B00000F931F93CF93DF9300D000D0CDB7DEB7A4
:106B10009093210C8093200C009751F484E090E036
:106B20009093E1098093E00981E080930A02BAC161
:106B30006C0185E090E09093E1098093E009EE24F8
:106B4000EA94FE2C0BED19E02CED30E040E451E02E
:106B500064E170E080E090E00E94D84681E0C816D1
:106B6000D10409F05FC080910602811123C06EE05C
:106B700078E0CE0101960E94B924AE014F5F5F4FCD
:106B800063E270E08FE090E00E94BA2ACE010196A5
:106B90000E949B24B0EEEB2EB7E0FB2E03E218E040
:106BA0002EE630E040EA50E062E870E080E090E0FD
:106BB0000E94D84680910602882311F16AE278E0AB
:106BC000CE0101960E94B924AE014F5F5F4F63E290
:106BD00070E08FE090E00E94BA2ACE0101960E94F8
:106BE0009B24E12CA8EFFA2E0EE318E02EE630E00D
:106BF00040EA50E062E870E080E090E00E94D84611
:106C0000FFE1EF2EF12C07E615E02EE630E040EA3A
:106C100050E062E870E080EA90E00E94D8468AE89E
:106C200092E02BC182E0C816D10409F05FC08091C8
:106C30000402811123C064E578E0CE0101960E9430
:106C4000B924AE014F5F5F4F63E270E08FE090E0E8
:106C50000E94BA2ACE0101960E949B24E0EEEE2EFD
:106C6000E7E0FE2E03E218E02EE630E040EA50E0D6
:106C700062E870E080E090E00E94D84680910402D3
:106C8000882311F169E678E0CE0101960E94B924CB
:106C9000AE014F5F5F4F63E270E08FE090E00E94D3
:106CA000BA2ACE0101960E949B24E12C78EFF72EA0
:106CB0000EE318E02EE630E040EA50E062E870E0D3
:106CC00080E090E00E94D8466FE1E62EF12C07E6C6
:106CD00015E02EE630E040EA50E062E870E080EA3D
:106CE00090E00E94D84680E892E0C7C083E0C816D2
:106CF000D10409F05FC080910202811123C06DE7C9
:106D000078E0CE0101960E94B924AE014F5F5F4F3B
:106D100063E270E08FE090E00E94BA2ACE01019613
:106D20000E949B2450EEE52E57E0F52E03E218E07A
:106D30002EE630E040EA50E062E870E080E090E06B
:106D40000E94D84680910202882311F162E978E01E
:106D5000CE0101960E94B924AE014F5F5F4F63E2FE
:106D600070E08FE090E00E94BA2ACE0101960E9466
:106D70009B24E12C48EFF42E0EE318E02EE630E0E1
:106D800040EA50E062E870E080E090E00E94D8467F
:106D90003FE1E32EF12C07E615E02EE630E040EA75
:106DA00050E062E870E080EA90E00E94D84686E712
:106DB00092E063C084E0C816D10409F073C08091EA
:106DC0000002811123C066EA78E0CE0101960E949C
:106DD000B924AE014F5F5F4F63E270E08FE090E057
:106DE0000E94BA2ACE0101960E949B2420EEE22E38
:106DF00027E0F22E03E218E02EE630E040EA50E011
:106E000062E870E080E090E00E94D8468091000245
:106E1000882311F16BEB78E0CE0101960E94B92432
:106E2000AE014F5F5F4F63E270E08FE090E00E9441
:106E3000BA2ACE0101960E949B24E12C98EFF92EEC
:106E40000EE318E02EE630E040EA50E062E870E041
:106E500080E090E00E94D8468FE1E82EF12C07E612
:106E600015E02EE630E040EA50E062E870E080EAAB
:106E700090E00E94D8468CE692E00E94624666E46A
:106E800078E0CE0101960E94B924AE014F5F5F4FBA
:106E900061E470E08FE090E00E94BA2ACE01019692
:106EA0000E949B2426960FB6F894DEBF0FBECDBF7E
:106EB000DF91CF911F910F91FF90EF90DF90CF90D6
:106EC000089520918F0A9091290E213208F04AC02E
:106ED00080918E0A8111FCCF32E030938E0A31E02E
:106EE00030938D0A3FEF3093180A10923A0A20939C
:106EF000390AAAE2BEE049E15AE0FA013E2F341B0A
:106F0000321718F43D913193F9CF10923B0A20913A
:106F10003B0A990F922B90933B0A90918C0A9130E7
:106F200061F410928C0A90913B0A9093BB0090916F
:106F3000BC0093FDF8CF95EC01C095EE9093BC009A
:106F400090918E0A9230E1F39091180A9F3F79F068
:106F50008091180A803241F08091180A803331F014
:106F600084E005C081E003C082E001C083E01092AC
:106F7000900A10928F0A1092F7090895CF93DF9329
:106F80001F92CDB7DEB769832091F7092223D1F094
:106F900020918F0A203240F021E030E0FC01338361
:106FA000228380E090E015C08091900AE82FF0E005
:106FB000E65DF14F998190838F5F8093900A809373
:106FC0008F0A05C061E0CE0101960E94E12781E0B1
:106FD00090E00F90DF91CF910895CF93DF93809150
:106FE000240C882399F1C091220CD091230C40915C
:106FF0009E0250919F026091A0027091A10229E22D
:107000003CE0CE010E947852811102C080E01FC096
:107010004091250C5091260C6091270C7091280C02
:10702000411551056105710579F029E23CE0CE0179
:107030000E947852882351F31092250C1092260C4E
:107040001092270C1092280C1092240C81E0DF91F2
:10705000CF910895BF92CF92DF92EF92FF920F935C
:107060001F93CF93DF936B017C01B42E80919E021E
:1070700090919F02A091A002B091A1028C159D0554
:10708000AE05BF0509F475C0A8DF882309F478C0F0
:10709000C091220CD091230C8E81882369F08881C5
:1070A0009981AA81BB81C816D906EA06FB0621F49C
:1070B0008F819885892BB1F1C882D982EA82FB82BF
:1070C0008B85A7019601833039F089E0220F331FA9
:1070D000441F551F8A95D1F761E1CE010E942152CC
:1070E000882319F083E08D8337C00E945A268B01D4
:1070F0000E94ED518A878F3F49F40E945A26601BF7
:10710000710B6D327140A0F38FE003C08E3F31F000
:107110008DE08D83CE010E94DF511EC018861F8234
:1071200081E08E8309E21CE00E94ED51F801819319
:107130008F01FEE009321F07B9F78F8198859E5FA6
:1071400098878F832985222319F08115924048F072
:10715000CE010E94095205C0CE010E94DF5180E09D
:107160000FC0C0929E02D0929F02E092A002F092C5
:10717000A1028091240C482F4B294093240C81E0DC
:10718000DF91CF911F910F91FF90EF90DF90CF9003
:10719000BF900895CF92DF92EF92FF920F93CF931B
:1071A000DF931F92CDB7DEB76C017901DC01149635
:1071B0008C91149791E09093F7098093290E109287
:1071C000900A10928F0A15968D919C911697DC016A
:1071D000ED91FC910190F081E02D49831995F60124
:1071E00085819681DC01ED91FC910190F081E02D8B
:1071F0004981642F1995F60185819681DC01ED9115
:10720000FC91402F50E00280F381E02DB7011995E9
:10721000F60187818F3F71F4D60115968D919C916F
:1072200016970F90DF91CF910F91FF90EF90DF9025
:10723000CF9047CEF60187810E947025892BD1F32C
:10724000EBCFCF92DF92EF92FF920F93CF93DF932A
:10725000CDB7DEB7A0970FB6F894DEBF0FBECDBF97
:107260006C01862FFB010E2F081B9191E02EF12C53
:10727000992341F0A1E0B0E0AC0FBD1FAE0DBF1DE2
:107280009C93F1CF9E012F5F3F4F45E062E0C60126
:1072900081DFC701A0960FB6F894DEBF0FBECDBF49
:1072A000DF91CF910F91FF90EF90DF90CF900895F5
:1072B0000F93CF93DF931F92CDB7DEB7698301E0C1
:1072C0009E012F5F3F4F45E062E064DF61E070E0C8
:1072D00080E090E00E94222681E090E00F90DF9114
:1072E000CF910F9108950F93CF93DF9300D0CDB737
:1072F000DEB76450643088F4E62FF0E0E85FFC4FBE
:10730000208127FD0AC029835A834B8303E09E0115
:107310002F5F3F4F42E068E03DDF0F900F900F90EE
:10732000DF91CF910F910895EF92FF920F931F93EA
:10733000CF93DF9300D0CDB7DEB76450643008F54B
:10734000E62FF0E0EC5FFC4F108117FD1AC0622FB2
:107350009A017C01603151F0AFEFBFEF0E940462EF
:107360002FEF30E040E050E00E94BC6119833A8387
:107370002B8303E09E012F5F3F4F41E068E0C70190
:1073800009DF0F900F900F90DF91CF911F910F9118
:10739000FF90EF9008952F923F924F925F926F92DD
:1073A0007F928F929F92AF92BF92CF92DF92EF9295
:1073B000FF920F931F93CF93DF9300D000D0CDB7F0
:1073C000DEB79E838D83562E442E3C832B8347014C
:1073D000C701880F991F880F991F3C0125E0621A89
:1073E000710810E0FF24F394202E312C35ECE32EAD
:1073F000101708F0CDC0AD81BE8114968C91149702
:10740000F092F7098093290E1092900A10928F0A39
:1074100015968D919C911697DC01ED91FC91019050
:10742000F081E02D652D1995ED81FE818581968194
:10743000DC01ED91FC910190F081E02D642D199516
:10744000ED81FE8187818F3F79F4AD81BE811596F4
:107450008D919C91169735DDB2E08B16910460F00A
:10746000C3010197F1F708C0ED81FE8187810E9479
:107470007025892BC9F3E9CFAD81BE8117968C9118
:107480008F3F21F4ED81FE81348109C0AD81BE8141
:1074900017968C910E947025892BC1F3F3CF8091B0
:1074A0008E0A8111FCCFC101811B910981329105A6
:1074B00014F080E290E0282F813208F020E2F09270
:1074C0008E0AF0928D0ABFEFB093180A10923A0A12
:1074D0004FEF420F4093390AF0923B0A40913B0A2A
:1074E000330F342B30933B0A30918C0A313069F4DE
:1074F00010928C0A30913B0A3093BB003091BC0053
:1075000033FDF8CFE092BC0003C0E5EEE093BC0091
:1075100030918E0A3130E1F330913A0A321710F48B
:1075200020913A0AA9E1BAE0E8EFF9E03E2F48EFEE
:1075300059E0341B321718F43D913193F7CF109274
:10754000920A2093910AA12CB12C6C01DD24812F89
:107550008A0DAC14BD04D4F42B813C81280F311D5D
:107560003A832983AD81BE8115968D919C911697A2
:10757000DC01ED91FC910284F385E02D1995E98100
:10758000FA818083FFEFAF1ABF0AE1CF182F30CF07
:1075900026960FB6F894DEBF0FBECDBFDF91CF9118
:1075A0001F910F91FF90EF90DF90CF90BF90AF9021
:1075B0009F908F907F906F905F904F903F902F9013
:1075C0000895EF92FF920F931F93CF93DF931F9233
:1075D0001F92CDB7DEB7633059F020F4623021F549
:1075E00040E009C0643031F06530F1F443E003C09D
:1075F00041E001C042E0495F24EFE22EFF24F39412
:1076000002E09E012F5F3F4F69E0C5DE098110E077
:10761000102F00278A81082B61E070E080E090E065
:107620000E942226C80102C080E090E00F900F90D7
:10763000DF91CF911F910F91FF90EF900895EF92FE
:10764000FF920F93CF93DF9300D01F92CDB7DEB799
:1076500028EEE22E23E0F22E04E09E012F5F3F4F42
:1076600044E060E098DE29816A81862F90E0A0E006
:10767000B0E0DC0199278827B22B2C81822B2B814B
:10768000BC01CD01722B0E94A96020E030E040E8EF
:1076900057E30E9408610F900F900F900F90DF91B9
:1076A000CF910F91FF90EF900895EF92FF920F937B
:1076B000CF93DF9300D01F92CDB7DEB72DE7E22E38
:1076C000F12C04E09E012F5F3F4F42E060E063DE5B
:1076D00029816A81862F90E0A0E0B0E0DC01992743
:1076E0008827B22B2C81822B2B81BC01CD01722BE0
:1076F0000F900F900F900F90DF91CF910F91FF900F
:10770000EF9008954F925F926F927F928F929F9227
:10771000AF92BF92CF92DF92EF92FF920F931F939F
:10772000CF93DF93EC016A017B01280139014230DC
:1077300051056105710510F480E072C089859A8554
:10774000AB85BC850196A11DB11D84179507A607C1
:10775000B70790F38B889C88AD88BE888F8980316D
:1077600029F4BB27AF2D9E2D8D2D09C0DB01CA0149
:1077700047E0B695A795979587954A95D1F7880ED6
:10778000991EAA1EBB1E80919E0290919F02A091FD
:10779000A002B091A10288169906AA06BB0679F448
:1077A0008F89803199F4DD24EE24FF24C601880FEF
:1077B000991FFC01E75DF34F5182408218C040E001
:1077C000C501B40147DC8111EBCFB6CFE894C7F80F
:1077D000DD24EE24FF24C601880F991F880F991F0E
:1077E000FC01E75DF34F4082518262827382809197
:1077F000240C81608093240C8A89823080F08D81F2
:107800009E81AF81B885880E991EAA1EBB1E8092EC
:10781000250C9092260CA092270CB092280C81E0A7
:10782000DF91CF911F910F91FF90EF90DF90CF905C
:10783000BF90AF909F908F907F906F905F904F9090
:1078400008958F929F92AF92BF92CF92DF92EF9264
:10785000FF920F931F93CF93DF93FC018185928555
:10786000A385B4850196A11DB11D84179507A607B0
:10787000B70710F480E05BC083899489A589B68935
:10788000C789C03129F4852E962EA72EBB2409C0A6
:107890004A015B01C7E0B694A79497948794CA9570
:1078A000D1F7E9016A017B018F01BC01CD01680DAF
:1078B000791D8A1D9B1D80909E0290909F02A09032
:1078C000A002B090A102681579058A059B0599F47C
:1078D000F80187898031A1F4B701A60155276627F1
:1078E0007727440F551FFA01E75DF34F808191819F
:1078F000A0E0B0E017C040E0ADDB8111E9CFBACF26
:10790000B701A6014F77552766277727440F551FE4
:10791000440F551FFA01E75DF34F80819181A281E9
:10792000B381BF7088839983AA83BB8381E0DF9191
:10793000CF911F910F91FF90EF90DF90CF90BF906C
:10794000AF909F908F9008954F925F926F927F9229
:107950008F929F92AF92BF92EF92FF920F931F93DD
:10796000CF93DF9300D01F921F92CDB7DEB78C016B
:107970006D83DC0115968C911597813009F056C006
:1079800014968C9181FF52C059C0038CF48DE02D68
:10799000258530E0275F3F4F2A013B01B1E04B1ABC
:1079A000510861087108022E04C0769467945794B8
:1079B00047940A94D2F7D501C4010197A109B109EE
:1079C00004C0B695A795979587952A95D2F7841503
:1079D0009505A605B70508F06FC0F8014789508DD9
:1079E000618D728D46835783608771872C013D01BD
:1079F0007801E6E0EE0EF11CD80141145104610457
:107A0000710409F463C016964D915D916D917C915E
:107A1000199797015B968D919C915C9712DFB1E06D
:107A20004B1A5108610871088111E6CF81E090E09E
:107A3000F8019383828380E090E04AC182FF0EC008
:107A4000F801428553856485758583889488A58867
:107A5000B688481559056A057B05F1F4D8011A96D0
:107A60004D915D916D917C911D975B968D919C914F
:107A70005C97FC0174807A944A015B0129E0B6941A
:107A8000A794979487942A95D1F778207A01F1E00A
:107A9000FF22772011F163C081149104A104B10485
:107AA00009F073CF1682178210861186F8011286AC
:107AB000138614861586D2CF452B462B472B09F407
:107AC0008CCF84199509A609B70990CF1A968D9283
:107AD0009D92AD92BC921D97C1CFE114F10409F0C3
:107AE0003EC0F80146815781608571854115510579
:107AF0006105710549F48789908DA18DB28D00973C
:107B0000A105B10539F520C09E012F5F3F4F99DED9
:107B1000882309F490CF89819A81AB81BC81F801D7
:107B2000238D348DF9012789203129F048EF5FEF4B
:107B30006FEF7FE004C048EF5FEF60E070E0841714
:107B40009507A607B70730F0C8010E94DC508111E5
:107B500006C06CCFF80186839783A087B187D801D0
:107B60005B96ED91FC915C9716968D909D90AD90F3
:107B7000BC901997B2E08B1A9108A108B10805844E
:107B800004C0880C991CAA1CBB1C0A94D2F78685D9
:107B90009785A089B189880E991EAA1EBB1E870CE5
:107BA000911CA11CB11CE114F10401F5F8014285FE
:107BB00053856485758583899489A589B689481715
:107BC00059076A077B0790F008DA882309F42ECF5B
:107BD00080929E0290929F02A092A002B092A10277
:107BE0008091240C81608093240C07C041E0C50182
:107BF000B40130DA882309F419CFF701E75DF34FB8
:107C00008D818083F80182859385A485B585019651
:107C1000A11DB11D82879387A487B58743895489A5
:107C200065897689481759076A077B0738F4838B7B
:107C3000948BA58BB68B848180688483D80114963D
:107C40008C9183FD03C081E090E042C0F8019581F2
:107C5000992309F4EBCE87FF37C066857785808945
:107C6000918941E0F7D9882309F4E0CED8015296F2
:107C7000EC91B0E2EB9F90011124D901A75DB34FC5
:107C8000109709F4D3CEF8018581823050F44389EE
:107C90005489658976895C964D935D936D937C9349
:107CA0005F97F8018789908DA18DB28DF901E75D0D
:107CB000F34F938F828FB58BA48BD80114968C9140
:107CC00014978F7714968C9388D98111BCCFAECE40
:107CD0000F900F900F900F900F90DF91CF911F9109
:107CE0000F91FF90EF90BF90AF909F908F907F90FB
:107CF0006F905F904F9008952F923F924F925F92B6
:107D00006F927F928F929F92AF92BF92CF92DF92AB
:107D1000EF92FF920F931F93CF93DF93CDB7DEB710
:107D200062970FB6F894DEBF0FBECDBF8C01DC01A9
:107D3000CD90DC9011971296AD90BC90139714964D
:107D40002D903C9015970E948E4E2F83388749873F
:107D50005A876B877C872F813885E984FA84EB8585
:107D6000FC85FE87ED878091510B9091520B8E1709
:107D70009F070CF0EEC04090B30B5090B40B052C55
:107D8000000C66087708C901330FAA0BBB0B9C01D6
:107D9000AD01245631094109510966277727CB01E6
:107DA00064197509860997090E94156320E233E07A
:107DB00040E050E00E94BC61DA01C901840D951DCC
:107DC000A61DB71D8F87988BA98BBA8B8F84988837
:107DD0002091B10B3091B20B2901330F660877085F
:107DE0008FEC98E00E94854EC701FF0CAA0BBB0BDD
:107DF0009C01AD01265931094109510966277727B0
:107E0000CB0164197509860997090E9415632EEE46
:107E100032E040E050E00E94BC61BA01A901440D8B
:107E2000551D661D771D80E491E07C01E41AF50A7A
:107E3000C7010E94864E84ED98E00E94854E8F8592
:107E400098890E94864E8AED98E00E94854E8D8525
:107E50009E850E94704EC6018897E816F9060CF4BC
:107E600078C04F96E816F9060CF073C035019FE014
:107E7000690E711C6814790404F1C5014E978816C7
:107E80009906DCF0D80118968D919C9119972816C7
:107E900039069CF414968D919C911597059615962C
:107EA0009C938E9314976BED79E0CE0101960E941E
:107EB000B924B1016B5F7F4F1FC0C5010E968815B5
:107EC00099050CF046C08E96881599050CF441C0B2
:107ED000F8018681978182159305DCF5848195816F
:107EE0000597958384836BED79E0CE0101960E941E
:107EF000B924B10165507109CE0101960E94DF23BA
:107F0000EE24EA94FE2C0BED19E029E130E046E482
:107F100050E0B301C6014CD724E030E0A301B60124
:107F200089819A810E947D29B5016E5E7F4FC601CD
:107F300088960E94CC4DB601655D7F4F24E030E00D
:107F4000A30181ED95E00E947D29CE0101960E945A
:107F50009B2462960FB6F894DEBF0FBECDBFDF91B3
:107F6000CF911F910F91FF90EF90DF90CF90BF9036
:107F7000AF909F908F907F906F905F904F903F90C9
:107F80002F9008952F923F924F925F926F927F921F
:107F90008F929F92AF92BF92CF92DF92EF92FF9219
:107FA0000F931F93CF93DF93CDB7DEB762970FB6D2
:107FB000F894DEBF0FBECDBF8C01DC01CD90DC900C
:107FC00011971296AD90BC90139714962D903C90FB
:107FD00015970E948E4E2F83388749875A876B8763
:107FE0007C872F813885E984FA84EB85FC85FE87C0
:107FF000ED878091510B9091520B8E179F070CF0DB
:10800000EFC04090B30B5090B40B052C000C6608E9
:108010007708C901330FAA0BBB0B9C01AD01245695
:1080200031094109510966277727CB016419750980
:10803000860997090E94156320E233E040E050E092
:108040000E94BC61DA01C901840D951DA61DB71DF2
:108050008F87988BA98BBA8B8F8498882091B10BCE
:108060003091B20B2901330F660877088FEC98E046
:108070000E94854EC701FF0CAA0BBB0B9C01AD01F2
:10808000265931094109510966277727CB0164191F
:108090007509860997090E9415632EEE32E040E0CB
:1080A00050E00E94BC61BA01A901440D551D661D36
:1080B000771D80E491E07C01E41AF50AC7010E9473
:1080C000864E84ED98E00E94854E8F8598890E94A7
:1080D000864E8AED98E00E94854E8D859E850E9491
:1080E000704EC6018B5B9F4F8E159F050CF078C0BC
:1080F00089968E159F050CF473C035019FE0690EBB
:10810000711C6814790404F1C5014E97881699060C
:10811000DCF0D80118968D919C9119972816390694
:108120009CF414968D919C911597059615969C93A9
:108130008E9314976BED79E0CE0101960E94B924DD
:10814000B1016B5F7F4F1FC0C5010E968815990561
:108150000CF046C08E96881599050CF441C0F801C4
:108160008681978182159305DCF584819581059739
:10817000958384836BED79E0CE0101960E94B9244A
:10818000B10165507109CE0101960E94DF23EE24F2
:10819000EA94FE2C0BED19E029E130E046E450E0D2
:1081A000B301C60105D624E030E0A301B601898100
:1081B0009A810E947D29B5016E5E7F4FC601889627
:1081C0000E94CC4DB601655D7F4F24E030E0A301F5
:1081D00081ED95E00E947D29CE0101960E949B24AD
:1081E00062960FB6F894DEBF0FBECDBFDF91CF9180
:1081F0001F910F91FF90EF90DF90CF90BF90AF90C5
:108200009F908F907F906F905F904F903F902F90B6
:1082100008952F923F924F925F926F927F928F922A
:108220009F92AF92BF92CF92DF92EF92FF920F9305
:108230001F93CF93DF93CDB7DEB764970FB6F89453
:10824000DEBF0FBECDBF8C01DC01CD90DC9011975D
:1082500012962D903C9013971496ED91FC911597E2
:10826000FE87ED870E948E4E2F83388749875A8775
:108270006B877C872F813885E984FA844B855C8500
:10828000588B4F878091510B9091520B8417950713
:108290000CF0EFC08090B30B9090B40B092C000C45
:1082A000AA08BB08C901330FAA0BBB0B9C01AD0187
:1082B000245631094109510966277727CB016819EE
:1082C00079098A099B090E94156320E233E040E0A6
:1082D00050E00E94BC61DA01C901880D991DAA1DF8
:1082E000BB1D898B9A8BAB8BBC8B89889A884090FD
:1082F000B10B5090B20B052C000C660877088FEC80
:1083000098E00E94854EC701FF0CAA0BBB0B9C0195
:10831000AD01265931094109510966277727CB015B
:1083200064197509860997090E9415632EEE32E0DB
:1083300040E050E00E94BC61420E531E641E751E58
:1083400080E491E07C01E418F508C7010E94864EA4
:1083500084ED98E00E94854E89899A890E94864E14
:108360008AED98E00E94854E8F8598890E94704E14
:10837000C6018897E816F9060CF47BC04F96E816FC
:10838000F9060CF076C051019FE0A90EB11CA814AB
:10839000B9041CF1C1014E9788169906F4F0D80172
:1083A00018968D919C911997ED85FE85E817F90730
:1083B000A4F414968D919C911597059615969C930F
:1083C0008E9314976BED79E0CE0101960E94B9244B
:1083D0006D857E856B5F7F4F2AC0C1010E96881523
:1083E00099050CF046C0FCE32F0E311C281439040B
:1083F0000CF43FC0D80116968D919C911797ED858E
:10840000FE858E179F07ACF514968D919C9115975C
:10841000059715969C938E9314976BED79E0CE019A
:1084200001960E94B9246D857E8565507109CE0143
:1084300001960E94DF2365EF75E0CE0101960E9450
:108440000E24EE24EA94FE2C0BED19E029E130E035
:1084500046E450E0B501C601ABD424E030E0A5010C
:10846000B60189819A810E947D29CE0101960E94E0
:108470009B2464960FB6F894DEBF0FBECDBFDF918C
:10848000CF911F910F91FF90EF90DF90CF90BF9011
:10849000AF909F908F907F906F905F904F903F90A4
:1084A0002F9008952F923F924F925F926F927F92FA
:1084B0008F929F92AF92BF92CF92DF92EF92FF92F4
:1084C0000F931F93CF93DF93CDB7DEB764970FB6AB
:1084D000F894DEBF0FBECDBF8C01DC01CD90DC90E7
:1084E000119712962D903C9013971496ED91FC9154
:1084F0001597FE87ED870E948E4E2F833887498718
:108500005A876B877C872F813885E984FA844B856D
:108510005C85588B4F878091510B9091520B84173B
:1085200095070CF0F0C08090B30B9090B40B092C21
:10853000000CAA08BB08C901330FAA0BBB0B9C0196
:10854000AD01245631094109510966277727CB012E
:10855000681979098A099B090E94156320E233E0B2
:1085600040E050E00E94BC61DA01C901880D991D0C
:10857000AA1DBB1D898B9A8BAB8BBC8B89889A8873
:108580004090B10B5090B20B052C000C6608770898
:108590008FEC98E00E94854EC701FF0CAA0BBB0B25
:1085A0009C01AD01265931094109510966277727F8
:1085B000CB0164197509860997090E9415632EEE8F
:1085C00032E040E050E00E94BC61420E531E641E47
:1085D000751E80E491E07C01E418F508C7010E9453
:1085E000864E84ED98E00E94854E89899A890E9482
:1085F000864E8AED98E00E94854E8F8598890E946C
:10860000704EC6018B5B9F4F8E159F050CF07BC093
:1086100089968E159F050CF476C051019FE0A90E36
:10862000B11CA814B9041CF1C1014E978816990613
:10863000F4F0D80118968D919C911997ED85FE85DF
:10864000E817F907A4F414968D919C911597059657
:1086500015969C938E9314976BED79E0CE0101965D
:108660000E94B9246D857E856B5F7F4F2AC0C10152
:108670000E96881599050CF046C0FCE32F0E311CB0
:10868000281439040CF43FC0D80116968D919C91A2
:108690001797ED85FE858E179F07ACF514968D9183
:1086A0009C911597059715969C938E9314976BED57
:1086B00079E0CE0101960E94B9246D857E856550D2
:1086C0007109CE0101960E94DF2365EF75E0CE01AE
:1086D00001960E940E24EE24EA94FE2C0BED19E084
:1086E00029E130E046E450E0B501C60161D324E061
:1086F00030E0A501B60189819A810E947D29CE01D1
:1087000001960E949B2464960FB6F894DEBF0FBEBC
:10871000CDBFDF91CF911F910F91FF90EF90DF9030
:10872000CF90BF90AF909F908F907F906F905F9011
:108730004F903F902F9008952F923F924F925F92CB
:108740006F927F928F929F92AF92BF92CF92DF9261
:10875000EF92FF920F931F93CF93DF93CDB7DEB7C6
:1087600064970FB6F894DEBF0FBECDBF8C01DC015D
:10877000CD90DC90119712962D903C901397149603
:10878000ED91FC911597FE87ED870E948E4E2F8309
:10879000388749875A876B877C872F813885E9849A
:1087A000FA844B855C85588B4F878091510B909153
:1087B000520B841795070CF0F0C08090B30B90908B
:1087C000B40B092C000CAA08BB08C901330FAA0B73
:1087D000BB0B9C01AD0124563109410951096627A3
:1087E0007727CB01681979098A099B090E941563CB
:1087F00020E233E040E050E00E94BC61DA01C901B0
:10880000880D991DAA1DBB1D898B9A8BAB8BBC8BC8
:1088100089889A884090B10B5090B20B052C000CBF
:10882000660877088FEC98E00E94854EC701FF0C20
:10883000AA0BBB0B9C01AD01265931094109510915
:1088400066277727CB0164197509860997090E9465
:1088500015632EEE32E040E050E00E94BC61420E13
:10886000531E641E751E80E491E07C01E418F50837
:10887000C7010E94864E84ED98E00E94854E89894A
:108880009A890E94864E8AED98E00E94854E8F85D7
:1088900098890E94704EC6018B5B9F4F8E159F0575
:1088A0000CF07BC089968E159F050CF476C05101A3
:1088B0009FE0A90EB11CA814B9041CF1C1014E9788
:1088C00088169906F4F0D80118968D919C91199705
:1088D000ED85FE85E817F907A4F414968D919C9117
:1088E0001597449615969C938E9314976BED79E0AB
:1088F000CE0101960E94B9246D857E856C5E7F4F06
:108900002AC0C1010E96881599050CF046C0FCE3FB
:108910002F0E311C281439040CF43FC0D8011696D0
:108920008D919C911797ED85FE858E179F07ACF56D
:1089300014968D919C911597449715969C938E93C0
:1089400014976BED79E0CE0101960E94B9246D85F4
:108950007E8564517109CE0101960E94DF2365EF87
:1089600075E0CE0101960E940E24EE24EA94FE2CBE
:108970000BED19E029E130E046E450E0B501C60115
:1089800017D224E030E0A501B60189819A810E94C6
:108990007D29CE0101960E949B2464960FB6F8941F
:1089A000DEBF0FBECDBFDF91CF911F910F91FF9022
:1089B000EF90DF90CF90BF90AF909F908F907F907F
:1089C0006F905F904F903F902F9008952F923F921D
:1089D0004F925F926F927F928F929F92AF92BF92CF
:1089E000CF92DF92EF92FF920F931F93CF93DF937B
:1089F00000D000D0CDB7DEB7FC01C080D180A2800E
:108A0000B3802480358036018AE0681A71084601F7
:108A100089E1881A9108B5016C5E7F4F260188E2D2
:108A2000481A51089501255031097B018301A401A1
:108A3000C20163D7B501625E7F4F9501295C3F4F4C
:108A40007B01A401C20159D76BED79E0CE010196FB
:108A50000E94B924B101CE0101960E94DF23450195
:108A60008FE0880E911C24E030E0A401B6018981DA
:108A70009A810E947D29B5016E5E7F4FC60188965E
:108A80000E94CC4DB601655D7F4F24E030E0A4012B
:108A900081ED95E00E947D29CE0101960E949B24E4
:108AA00026960FB6F894DEBF0FBECDBFDF91CF91F3
:108AB0001F910F91FF90EF90DF90CF90BF90AF90FC
:108AC0009F908F907F906F905F904F903F902F90EE
:108AD00008952F923F924F925F926F927F928F9262
:108AE0009F92AF92BF92CF92DF92EF92FF920F933D
:108AF0001F93CF93DF9300D000D0CDB7DEB7FC013A
:108B0000C080D180A280B38024803580360189E680
:108B1000680E711C46018AE5880E911CB5016C5ED9
:108B20007F4F26018BE4480E511C950125503109D9
:108B30007B018301A401C201E0D6B501625E7F4FD3
:108B40009501295C3F4F7B01A401C201D6D66BED94
:108B500079E0CE0101960E94B924B101CE010196BF
:108B60000E94DF2345018FE0880E911C24E030E055
:108B7000A401B60189819A810E947D29B5016E5EAA
:108B80007F4FC60188960E94CC4DB601655D7F4F30
:108B900024E030E0A40181ED95E00E947D29CE0122
:108BA00001960E949B2426960FB6F894DEBF0FBE56
:108BB000CDBFDF91CF911F910F91FF90EF90DF908C
:108BC000CF90BF90AF909F908F907F906F905F906D
:108BD0004F903F902F9008952F923F924F925F9227
:108BE0006F927F928F929F92AF92BF92CF92DF92BD
:108BF000EF92FF920F931F93CF93DF9300D000D09B
:108C0000CDB7DEB7FC01A080B180C280D3802480C4
:108C1000358035018AE0681A7108450189E1881AB2
:108C20009108B6016C5E7F4F250188E2481A510811
:108C30009601255031097B018301A401C2015DD653
:108C4000B601625E7F4F9601295C3F4F7B01A40114
:108C5000C20153D66BED79E0CE0101960E94B92492
:108C6000B101CE0101960E94DF2365EF75E0CE01D0
:108C700001960E940E24A601415F5F4F24E030E080
:108C8000B50189819A810E947D29CE0101960E94B9
:108C90009B2426960FB6F894DEBF0FBECDBFDF91A2
:108CA000CF911F910F91FF90EF90DF90CF90BF90E9
:108CB000AF909F908F907F906F905F904F903F907C
:108CC0002F9008952F923F924F925F926F927F92D2
:108CD0008F929F92AF92BF92CF92DF92EF92FF92CC
:108CE0000F931F93CF93DF9300D000D0CDB7DEB7A3
:108CF000FC01A080B180C280D38024803580350102
:108D000089E6680E711C45018AE5880E911CB60142
:108D10006C5E7F4F25018BE4480E511C9601255057
:108D200031097B018301A401C201E7D5B601625E6E
:108D30007F4F9601295C3F4F7B01A401C201DDD525
:108D40006BED79E0CE0101960E94B924B101CE010C
:108D500001960E94DF2365EF75E0CE0101960E9427
:108D60000E24A601415F5F4F24E030E0B501898108
:108D70009A810E947D29CE0101960E949B2426960D
:108D80000FB6F894DEBF0FBECDBFDF91CF911F911C
:108D90000F91FF90EF90DF90CF90BF90AF909F909A
:108DA0008F907F906F905F904F903F902F9008959D
:108DB0006F927F928F929F92AF92BF92CF92DF92EB
:108DC000EF92FF920F931F93CF93DF93E091930A5B
:108DD000E1112FC0E80139015A014B016C0184E017
:108DE0008093BF0B89019A01AB01B6018FE99BE02B
:108DF0000E94272DF090C10B81E08093C10BF301FD
:108E000077FC3196AF0155954795480D591D4F5048
:108E10005109B501B7FE02C06F5F7F4F7595679529
:108E20006C0D7D1D24E030E0CE010E947D29F09282
:108E3000C10BDF91CF911F910F91FF90EF90DF90C9
:108E4000CF90BF90AF909F908F907F906F9008953C
:108E50000F931F93CF93DF9300D000D0CDB7DEB731
:108E60008C0120914A0E30914B0E2F5F3F4F309373
:108E70004B0E20934A0E2F313105BCF02091430B4D
:108E80003091440B45E350E06FE37BE0CE01019667
:108E90000E94CD24BE016F5F7F4F8FE39BE00E9455
:108EA0001C24CE0101960E949B24F8014481558127
:108EB000608171818FE39BE04533510588F40E9406
:108EC0005223F80104811581053311055CF466E82D
:108ED00073E08FE39BE00E940E240F5F1F4FF4CFDF
:108EE0000E9452238091930A882319F11092A80BB3
:108EF0001092A70B1092AA0B1092A90B8FEF9FEF65
:108F00009093B60B8093B50B1092B80B1092B70BE1
:108F100081E08093C00B8093BF0B4091430B509135
:108F2000440B60913F0B7091400B8FE99BE00E94D6
:108F3000472126960FB6F894DEBF0FBECDBFDF9156
:108F4000CF911F910F9108958F929F92AF92BF92F0
:108F5000CF92DF92EF92FF920F931F93CF93DF9305
:108F600000D000D0CDB7DEB78B012091E009309161
:108F7000E10921153105A9F4009749F4672B51F552
:108F800081E090E09093E1098093E0092EC0019781
:108F900009F09CC16115710509F0B1C182E090E052
:108FA0001FC02130310521F122303105E9F1233094
:108FB000310509F445C02430310509F4E7C02530F6
:108FC000310509F083C18130910509F006C1672B95
:108FD00009F474C10130110509F078C183E090E013
:108FE0009093E1098093E00981E080930A026EC1C9
:108FF0000097D1F46130710509F068C1E12CF12CC2
:109000000BED19E020EF30E040E451E060E070E06B
:1090100080E090E0CDDE61E089E00E94C72560E05D
:1090200089E00E94982552C1019709F04FC1013093
:10903000110509F04BC11092E1091092E009B3C08B
:10904000019791F56130710511F51092E1091092C7
:10905000E00981E080930A021092210C1092200C0A
:1090600081E090E00E94353482E090E00E94353447
:1090700083E090E00E94353484E090E00E94353433
:109080006DE770E080E090E00E9422260DC0672B23
:1090900059F484E090E09093E1098093E00981E045
:1090A00080935B0280930A0239D629833A834B83EB
:1090B0005C836D837E83C090B30BD090B40B0D2C7A
:1090C000000CEE08FF0829813A81C901330FAA0B71
:1090D000BB0B9C01AD01245631094109510966279A
:1090E0007727CB016C197D098E099F090E941563B2
:1090F00020E233E040E050E00E94BC61C20ED31E8B
:10910000E41EF51E8090B10B9090B20B092C000C60
:10911000AA08BB082B813C81C901330FAA0BBB0BEA
:109120009C01AD012659310941095109662777276C
:10913000CB01681979098A099B090E9415632EEEF3
:1091400032E040E050E00E94BC61820E931EA41EFB
:10915000B51E00E411E00819190917FDB7C0013563
:1091600011050CF041C1C60182589109C89708F059
:10917000F7C081E090E00E94353481E090E00E94E9
:109180007C3581E090E00E943534EAC08130910561
:1091900071F46130710509F099C083E090E090931B
:1091A000E1098093E00981E080930A020FC0892BD6
:1091B00009F08CC06130710509F088C080915B02B4
:1091C00091E0892780935B0290930A026DE770E03B
:1091D00080E090E00E94222679C0892B09F076C0B9
:1091E0006130710509F072C08091200C9091210CC2
:1091F000019799F49091060281E0892780930602F5
:1092000067EE78E0CE0101960E94B924CE01019666
:109210001FDECE0101960E949B248091200C90912C
:10922000210C029799F49091040281E089278093A0
:10923000040260E079E0CE0101960E94B924CE01DB
:10924000019606DECE0101960E949B248091200C9F
:109250009091210C039799F49091020281E0892763
:109260008093020269E179E0CE0101960E94B9245F
:10927000CE010196EDDDCE0101960E949B248091E6
:10928000200C9091210C049799F49091000281E0B8
:1092900089278093000262E379E0CE0101960E9463
:1092A000B924CE010196D4DDCE0101960E949B2403
:1092B0008091200C9091210C0E947C358091200C93
:1092C0009091210C009711F00E94353462E370E018
:1092D00080E090E00E94222626960FB6F894DEBF2A
:1092E0000FBECDBFDF91CF911F910F91FF90EF90F7
:1092F000DF90CF90BF90AF909F908F900895613096
:10930000710521F78091080290910902892B51F093
:109310001092930B81E080930A021092090210923E
:10932000080219C0FF24F394F092930BE091910B83
:10933000F091920B19950E945A2660938D0B7093B1
:109340008E0B80938F0B9093900BF0920A021093E8
:109350000902009308026AEF70E080E090E03ACFE3
:1093600000351105B1F4C60182589109C89760F41F
:1093700082E090E00E94353482E090E00E947C35EB
:1093800082E090E00E94353417FD0EC001351105D2
:109390002CF4C601895B9109C897C8F000551109E2
:1093A0000135110508F092CF89EBC81AD10888E37E
:1093B000C816D10408F08ACF84E090E00E943534CA
:1093C00084E090E00E947C3584E090E07DCF83E0F3
:1093D00090E00E94353483E090E00E947C3583E089
:1093E00090E00E943534DACF013A11057CF6BBCF0C
:1093F0006BED79E08BE49BE00E9486246BED79E0D5
:109400008FE39BE00E94862410924B0E10924A0E2E
:1094100080E090E00C94C72ACF92DF92EF92FF9207
:109420000F931F93CF93DF93CDB7DEB72C970FB673
:10943000F894DEBF0FBECDBF6B017C018A016BE4E7
:1094400079E0CE0101960E94B924B701A601CE01B0
:1094500001960E94AF236BEC75E0CE0101960E944D
:109460000E2420E030E040E151E4C701B6010E9443
:10947000086120E030E040EA50E40E94786220E099
:1094800030E040E052E40E941462AB01BC01CE0126
:1094900001960E947F2360ED75E0CE0101960E9447
:1094A0000E24BE016F5F7F4FCE0107960E94A0245D
:1094B000CE010796CDDCCE0107960E949B246BED72
:1094C00079E0CE0101960E94862460E779E0CE0122
:1094D00001960E940E24B801CE0101960E94DF235E
:1094E00065EF75E0CE0101960E940E24BE016F5F0C
:1094F0007F4FCE0107960E94A024CE010796A8DCDC
:10950000CE0107960E949B24CE0101960E949B24C7
:109510002C960FB6F894DEBF0FBECDBFDF91CF9172
:109520001F910F91FF90EF90DF90CF900895CF9211
:10953000DF92EF92FF920F931F93CF93DF93CDB7FC
:10954000DEB72C970FB6F894DEBF0FBECDBF6B0110
:109550007C018A0162E979E0CE0101960E94B9247A
:10956000B701A601CE0101960E94AF236BEC75E016
:10957000CE0101960E940E2420E030E040E151E44B
:10958000C701B6010E94086120E030E040EA50E4E3
:109590000E94786220E030E040E052E40E941462D1
:1095A000AB01BC01CE0101960E947F2360ED75E006
:1095B000CE0101960E940E24BE016F5F7F4FCE0147
:1095C00007960E94A024CE01079642DCCE010796A2
:1095D0000E949B246BED79E0CE0101960E948624C7
:1095E00067EB79E0CE0101960E940E24B801CE010E
:1095F00001960E94DF2365EF75E0CE0101960E947F
:109600000E24BE016F5F7F4FCE0107960E94A024FB
:10961000CE0107961DDCCE0107960E949B24CE0149
:1096200001960E949B242C960FB6F894DEBF0FBEC5
:10963000CDBFDF91CF911F910F91FF90EF90DF9001
:10964000CF900895CF92DF92EF92FF920F931F93E6
:10965000CF93DF937C016B01EA0180E591E00E94EA
:10966000243397012C0F3D1F215031098601A6019B
:10967000B7018FE99BE00E94983220E0CE0100976D
:1096800071F02EBD02D001D001C0089500002EBDA2
:109690000096009601D001C00895019791F780913E
:1096A0000B01816080930B010DB407FEFDCFDF91AC
:1096B000CF911F910F91FF90EF90DF90CF900C947E
:1096C00023330F931F93CF93DF938C01EB01809192
:1096D000B10B9091B20B0817190708F091C0809157
:1096E000B30B9091B40B6817790708F089C080E537
:1096F00091E00E94243380910B018E7F80930B01B7
:109700008091BD0B9091BE0B8017910711F1809154
:109710000B018D7F80930B018AE28EBD00000096C5
:10972000009601D001C008951093BE0B0093BD0BAD
:1097300080910B01826080930B011EBD02D001D08D
:1097400001C0089500000EBD0000009601D001C0C8
:1097500008958091BB0B9091BC0B8C179D0719F15C
:1097600080910B018D7F80930B018BE28EBD0000F9
:109770000096009601D001C00895D093BC0BC09311
:10978000BB0B80910B01826080930B01DEBD02D088
:1097900001D001C008950000CEBD000000960096E3
:1097A00001D001C0089580910B018D7F80930B0142
:1097B0008CE28EBD00960096009601D001C00895FF
:1097C00080910B01826080930B011EBC02D001D0FE
:1097D00001C0089500001EBC00000096009601D054
:1097E00001C0089580910B01816080930B010DB43D
:1097F00007FEFDCFDF91CF911F910F910C94233382
:10980000DF91CF911F910F910895009769F0FC01AE
:1098100001900020E9F73197AF01481B590BBC01BB
:1098200084E99AE00C94472180E090E008958F92BB
:109830009F92AF92BF920F931F93CF93DF93CDB7B9
:10984000DEB7A1970FB6F894DEBF0FBECDBF19A249
:10985000423008F44AE08E010F5D1F4F842E912C98
:10986000A12CB12CA50194010E94E261E62FB9015F
:10987000CA0101501109EA3014F4E05D01C0E95C4D
:10988000D801EC93232B242B252B61F7C801BDDFD6
:10989000A1960FB6F894DEBF0FBECDBFDF91CF917A
:1098A0001F910F91BF90AF909F908F900895CF928E
:1098B000DF92EF92FF92CF93DF936B017C01E091F7
:1098C000940AF091950A0190F081E02D6DE284E90F
:1098D0009AE01995EC0166277727CB016C197D0971
:1098E0008E099F094AE0A3DF8C0F9D1FDF91CF9166
:1098F000FF90EF90DF90CF9008952F923F924F927C
:109900005F926F927F928F929F92AF92BF92CF920F
:10991000DF92EF92FF920F931F93CF93DF93CDB718
:10992000DEB72E970FB6F894DEBF0FBECDBF9E8771
:109930008D874B016A015901C801261737078CF43E
:10994000322F2B2DE616F7060CF004C157017B01D0
:10995000832E922E2D2D68018D859E854D872E8715
:109960000DC0E216F306C4F43A2D2B2D5701E32E59
:10997000F22E3C2D2D2D6C01832F922FA814B904AB
:109980005CF4382D292D4501A32EB22E3D852E8560
:10999000DE86CD86C32ED22E8E149F04E9F52D854A
:1099A0003E85C216D3066CF03D852E854D855E85BD
:1099B0004C155D0514F43C2D2D2DCD84DE843D87A2
:1099C0002E878C159D0544F02D853E852817390777
:1099D00014F49E878D87C6014D855E85481B590B03
:1099E0004F5F5F4FB4012E960FB6F894DEBF0FBEE7
:1099F000CDBFDF91CF911F910F91FF90EF90DF903E
:109A0000CF90BF90AF909F908F907F906F905F901E
:109A10004F903F902F9016CE96014D855E85241B6A
:109A2000350B3E832D8395012819390938872F83FB
:109A30003C01641A750A9701281939093A83298368
:109A40009C012C193D093C832B8397012A193B0962
:109A50003A8729879501AE14BF0411F021503109CE
:109A60008401412C512C212C312C201731077CF101
:109A7000C1016F8178850E942463ED85FE85E60F24
:109A8000F71FC20169817A810E9424634D855E853A
:109A9000640F751F8D819E81280E391E460C571C40
:109AA0006E177F072CF49E2F8F2FFB01692F782FC5
:109AB0006E1B7F0BAB014F5F5F4FB801CF012B8750
:109AC0003C87C0DD0F5F1F4F3C852B85CECFC80183
:109AD0008A199B092B813C81289F5001299FB00C3A
:109AE000389FB00C1124C80188199909689E40015B
:109AF000699E900C789E900C1124E016F1069CF162
:109B0000C50169857A850E9424639601260F371F57
:109B1000C40169817A810E9424634D855E85640F4A
:109B2000751F8B819C81A80EB91E860C971C62172D
:109B300073072CF4922F832F9B01692F782F621BC0
:109B4000730BAB014F5F5F4FB801C9017BDD0F5F46
:109B50001F4FD3CF5B01832E922E2D2DCD84DE841B
:109B60004D872E8719CF2E960FB6F894DEBF0FBE05
:109B7000CDBFDF91CF911F910F91FF90EF90DF90BC
:109B8000CF90BF90AF909F908F907F906F905F909D
:109B90004F903F902F9008952F923F924F925F9257
:109BA0006F927F928F929F92AF92BF92CF92DF92ED
:109BB000EF92FF920F931F93CF93DF9300D01F92EA
:109BC000CDB7DEB78C017C836B830E94462C6B8102
:109BD0007C81C801039675DD6B817C81C801039788
:109BE00070DD6B817C8163507109C8016ADD6B8116
:109BF0007C816D5F7F4FC80164DD21E030E0C12CC6
:109C0000D12C8AEF282E33243A949EEFA92EBB2420
:109C1000BA9443E0E42EF12C8FEFC81AD80A2E5FD5
:109C20003F4FA20EB31E28014C0C5D1C8B809C8004
:109C30008E0C9F1CB401C20129833A8342DD380196
:109C40006C187D08B401C3013CDD8B809C808E18AC
:109C50009F08B401C30135DDB401C20132DD8B8040
:109C60009C808C0C9D1CB40128014E0C5F1CC20111
:109C700028DDB40148018E189F08C40122DD6B80E5
:109C80007C806C187D08B301C4011BDDB301C201E7
:109C900018DD29813A81CE14DF045CF4B7FCBCCF17
:109CA00081E0E81AF10882E0280E311CA20CB31CF6
:109CB000B3CF0F900F900F900F90DF91CF911F9126
:109CC0000F91FF90EF90DF90CF90BF90AF909F905B
:109CD0008F907F906F905F904F903F902F9008955E
:109CE000CF93DF93BC01990F880B990B97FF02C0AC
:109CF000DEDD02C04AE09BDDEC0189ED99E085DD07
:109D00008C0F9D1FDF91CF9108957FCDBC01990FDE
:109D1000880B990B97FDCBCD4AE089CD4F925F928E
:109D20006F927F928F929F92BF92CF92DF92EF922B
:109D3000FF920F931F93CF93DF9300D000D0CDB746
:109D4000DEB760E08091530B0E94C72560E08091F0
:109D5000540B0E94C72561E08091560B0E94C725D5
:109D600061E08091550B0E94C7258091610BE091C5
:109D7000590BF0915A0B9081892B80839091620B43
:109D8000E0915D0BF0915E0B8081282F30E0892FF0
:109D900090E0809590958223932380838091530B4C
:109DA0000E9403268C018091530B0E940326980188
:109DB000281B390B2C5F3F4F2930310548F4A8018F
:109DC000480F591FCA0195958795BB24B39401C0CC
:109DD000B12C0FEF13E0081B190B60E08091560BBC
:109DE0000E94C72560E08091550B0E94C72561E065
:109DF0008091530B0E94C72561E08091540B0E9413
:109E0000C7259091640BE0915F0BF091600B80810E
:109E1000282F30E0892F90E080959095822393231E
:109E200080838091630BE0915B0BF0915C0B9081E0
:109E3000892B80838091550B0E9403267C018091A1
:109E4000550B0E940326A701481B590B4C5F5F4F1F
:109E50004930510538F49701280F391FC9019595EC
:109E6000879501C0B12C4FEF53E07A01E81AF90A47
:109E700061E08091560B0E94C72560E08091530BF2
:109E80000E94C7259091610BE091590BF0915A0BFC
:109E90008081282F30E0892F90E080959095822353
:109EA000932380838091640BE0915F0BF091600BB2
:109EB0009081892B80838091550B0E9403266C0131
:109EC0008091530B0E9403268090570B9090580B63
:109ED0008114910409F43FC0BC01990F880B990BC0
:109EE0000E94A9602B013C01B601DD0C880B990B87
:109EF0000E94A9609B01AC01C301B2010E9478627B
:109F000020E030E040E85FE30E9413622B013C0157
:109F1000B801012E000C880B990B0E94A9609B01CF
:109F2000AC01C301B2010E9408612B013C01B401E4
:109F300080E090E00E94A7609B01AC01C301B201E8
:109F40000E94086120E030E040E85AE30E94086186
:109F50000E94E06205C0B601681B790B61507C4F1E
:109F6000B11002C060E070E01A830983FC82EB82CA
:109F70007E836D83202F3A814E2D5C817E8180E02F
:109F800090E026960FB6F894DEBF0FBECDBFDF91EE
:109F9000CF911F910F91FF90EF90DF90CF90BF90E6
:109FA0009F908F907F906F905F904F9008950F9348
:109FB0001F930E945A2660939C0A70939D0A809377
:109FC0009E0A90939F0AE091940AF091950A028468
:109FD000F385E02D84E99AE0199597FF1FC00E9450
:109FE0005A2600919C0A10919D0A20919E0A309158
:109FF0009F0ADC01CB01801B910BA20BB30B0091DC
:10A00000980A1091990A20919A0A30919B0A801718
:10A010009107A207B307B8F28FEF9FEF1F910F913F
:10A020000895CF93DF93EC0161E086E00E94C7259D
:10A03000209711F460E004C0CF3FD10531F461E016
:10A0400086E0DF91CF910C949825EEE4F0E3E49163
:10A050008E2F90E0FC013197E231F10508F09DC0B0
:10A060008827EC56FF4F8F4F0C94376384B5806878
:10A0700084BDC7BD97C084B5806284BDC8BD92C091
:10A0800080918000806880938000D0938900C09385
:10A09000880088C080918000806280938000D09387
:10A0A0008B00C0938A007EC080918000886080937E
:10A0B0008000D0938D00C0938C0074C08091B0005C
:10A0C00080688093B000C093B3006CC08091B000F2
:10A0D00080628093B000C093B40064C0809190000F
:10A0E000806880939000D0939900C09398005AC0E4
:10A0F00080919000806280939000D0939B00C093E9
:10A100009A0050C080919000886080939000D09316
:10A110009D00C0939C0046C08091A0008068809301
:10A12000A0008091A0008F7B8093A000D093A90015
:10A13000C093A80037C08091A00080628093A000E7
:10A14000D093AB00C093AA002DC08091A00088607E
:10A150008093A000D093AD00C093AC0023C0809149
:10A160002001806880932001D0932901C0932801A9
:10A1700019C080912001806280932001D0932B012F
:10A18000C0932A010FC08091200188608093200134
:10A19000D0932D01C0932C0105C0C038D1050CF01F
:10A1A0004ECF48CFDF91CF9108958EBD00000DB402
:10A1B00007FEFDCF8EB508953F924F925F926F924A
:10A1C0007F928F929F92AF92BF92CF92DF92EF9247
:10A1D000FF920F931F93CF93DF93CDB7DEB72C97EA
:10A1E0000FB6F894DEBF0FBECDBF5C01DC015B96FD
:10A1F0008D909C905C971696CD90DD90ED90FC90A4
:10A200001997C114D104E104F10439F0BFEFCB1A5E
:10A21000DB0AEB0AFB0A312C07C0F401C080D180B5
:10A22000E280F38033243394F40181859285A38501
:10A23000B4859C01AD012F5F3F4F4F4F5F4F298782
:10A240003A874B875C87260137011D821E821F8259
:10A250001886F40181859285A385B4852D813E8180
:10A260004F815885281739074A075B0708F063C0F4
:10A2700089859A85AB85BC858C159D05AE05BF0586
:10A2800050F482E0C82ED12CE12CF12C92E0492E22
:10A29000512C612C712C9E012F5F3F4FB701A601FD
:10A2A000C4010E94213C882309F445C089819A8118
:10A2B000AB81BC81892B8A2B8B2B41F02601370186
:10A2C0009FEF491A590A690A790A05C0C414D504CE
:10A2D000E604F70491F02D813E814F8158852F5F70
:10A2E0003F4F4F4F5F4F2D833E834F8358873FEF44
:10A2F000C31AD30AE30AF30AACCF0FEF1FEF2FEF15
:10A300003FE0B301A201C4010E94823B882399F07F
:10A31000D50116964D915D916D917C9119974115DE
:10A3200051056105710549F093018201C4010E9444
:10A33000823B811102C080E02AC0D50116964D9261
:10A340005D926D927C921997332051F0D301C20136
:10A350000196A11DB11DF40180839183A283B38373
:10A36000F5018789908DA18DB28D892B8A2B8B2B3E
:10A3700069F4D50157964D925D926D927C925A97F1
:10A3800014968C911497806814968C9381E02C9687
:10A390000FB6F894DEBF0FBECDBFDF91CF911F91F6
:10A3A0000F91FF90EF90DF90CF90BF90AF909F9074
:10A3B0008F907F906F905F904F903F90089561E0F5
:10A3C000FC0184810E94982580914C0E882321F005
:10A3D00010924C0E0C94233308958FEFE6CE0F931A
:10A3E0001F93CF93DF93EB010E945A268B01F5DF79
:10A3F0008F3F49F00E945A26601B710B6C177D0736
:10A40000B0F380E001C081E0DF91CF911F910F9107
:10A410000895CF93DF93EC018E81882379F08F81AB
:10A4200098859C012F5F3F4F38872F838230924061
:10A4300010F4D3DFF4CFCE01C2DF1E82DF91CF91C3
:10A4400008958F929F92AF92BF92FF920F931F93A6
:10A45000CF93DF93EC01F62E49015A01DADF8091A8
:10A460004C0E811109C081E080934C0E8091310B1C
:10A470009091320B0E94243360E08C810E949825D9
:10A480006CE271E0CE01ABDF8F2D80648EDE08E1DF
:10A4900010E0D501C401002E04C0B695A79597958C
:10A4A00087950A94D2F781DE08501109083F8FEF93
:10A4B000180779F7FF2029F088E0F81204C087E830
:10A4C00003C085E901C08FEF70DE10E086DF8A8768
:10A4D00087FF04C01F3F11F01F5FF8CFDF91CF91BE
:10A4E0001F910F91FF90BF90AF909F908F90089514
:10A4F000EF92FF920F931F93CF93DF93EC017901BB
:10A50000411551056105710511F482E134C08B8557
:10A51000833039F089E0440F551F661F771F8A95F5
:10A52000D1F79A01AB0168E1CE018BDF882311F0EE
:10A5300084E021C08EEF39DE87018EEFF81AF80132
:10A5400081918F0132DE0E151F05C9F78FEF2DDEC9
:10A550008FEF2BDE42DF8A878F71853029F081E112
:10A560008D83CE012CDF08C068E572E0CE0137DFB5
:10A57000811106C085E18D83CE0121DF80E010C00E
:10A5800020E030E0A9016DE0CE015BDF811103C066
:10A5900024DF882311F084E1EECFCE0110DF81E0CB
:10A5A000DF91CF911F910F91FF90EF900895CF937E
:10A5B000DF93CDB7DEB76C970FB6F894DEBF0FBE52
:10A5C000CDBF789484B5826084BD84B5816084BD3C
:10A5D00085B5826085BD85B5816085BD80916E0041
:10A5E000816080936E001092810080918100826072
:10A5F00080938100809181008160809381008091AF
:10A6000080008160809380008091B100846080939D
:10A61000B1008091B00081608093B0008091910082
:10A62000826080939100809191008160809391007D
:10A63000809190008160809390008091A100826061
:10A640008093A1008091A10081608093A1008091FE
:10A65000A00081608093A00080912101826080939E
:10A66000210180912101816080932101809120014D
:10A6700081608093200180917A00846080937A00C9
:10A6800080917A00826080937A0080917A00816064
:10A6900080937A0080917A00806880937A0010928B
:10A6A000C10080E197E2A0E0B0E08093940B90932A
:10A6B000950BA093960BB093970B8BE69EE190932E
:10A6C0009D0B80939C0B81E080939E0B40E457E7A9
:10A6D0006BE170E04093890B50938A0B60938B0B76
:10A6E00070938C0B2AE939E13093920B2093910BF4
:10A6F0008093930B8093930A61E082E00E94C725C8
:10A7000061E082E00E94982561E083E00E94C72515
:10A7100061E083E00E94982561E084E00E94C72503
:10A7200061E084E00E94982561E085E00E94C725F1
:10A7300061E085E00E94982562E089E00E94C725DB
:10A7400062E082E20E94C72562E083E20E94C725A0
:10A7500062E084E20E94C72562E085E20E94C7258C
:10A7600061E08EE10E94C72561E08FE10E94C7256C
:10A770001092EC091092ED091092EE091092EF0977
:10A780008CE291E0A0E0B0E08093E8099093E909C1
:10A79000A093EA09B093EB0982E090E09093E70977
:10A7A0008093E6090E945A266093E2097093E309B8
:10A7B0008093E4099093E509E091A40AF091A50A39
:10A7C00082E08083E091A00AF091A10A1082E091DA
:10A7D000A20AF091A30A8FEC80831092AC0AE09158
:10A7E000A80AF091A90A86E08083E091A60AF09178
:10A7F000A70A808180618083E091A60AF091A70A70
:10A80000808188608083E091A60AF091A70A808108
:10A8100080688083E091A60AF091A70A80818F7DED
:10A82000808362E08091C90B0E94C7250E945A264E
:10A83000DC01CB01805D9740A109B1098093CD0B6C
:10A840009093CE0BA093CF0BB093D00B87E3809364
:10A85000D60B1FB7F8948091F009811127C0E6EF5D
:10A86000FAE28491ECE3FBE29491E82FF0E0EE0F42
:10A87000FF1FEA5BFD4FA591B491EC91E92321F410
:10A8800061E085E30E94982561E085E30E94C72589
:10A890008CB580618CBD8CB580648CBD61E084E337
:10A8A0000E94C72561E083E30E94C7258091F009DB
:10A8B0008F5F8093F0091FBF8CB58093A60B8CB57A
:10A8C0008C7F8CBD8DB581608DBD8CB58F7D8CBD31
:10A8D0008CB5837F8CBD8CB58093A50B61E088E03F
:10A8E0000E94982565E070E080E090E00E942226BA
:10A8F00060E088E00E94982564E170E080E090E0EC
:10A900000E94222661E088E00E94982566E970E0B6
:10A9100080E090E00E94222680E591E00E942433AE
:10A92000E0E6F2E0F49001E612E0FF2009F435C021
:10A93000F80184910E94DC2C5801F2E0AF0EB11CAA
:10A94000F80131960491202F2078E22E0F776501CF
:10A95000102F115040F0F60184910E94CB2CFFEF94
:10A96000CF1ADF0AF6CF6501C00ED11C8601EE209A
:10A9700091F02FEFC21AD20AF80164916F3F21F0D3
:10A9800070E080E090E004C064EF71E080E090E06F
:10A990000E9422268601FA94C8CF0DB407FEFDCF8F
:10A9A0000E94233381E08093C20B80E591E00E94F6
:10A9B000243386E30E94DC2C8091C20B90E0883027
:10A9C000910570F5FC018827EE58FF4F8F4F0C94CE
:10A9D000376388E40BC088E215C088E807C088EEBA
:10A9E00011C088EC03C088E60DC088E00E94CB2C23
:10A9F00080EF90E09093B20B8093B10B80E491E0F4
:10AA00000BC088EA0E94CB2C80E491E09093B20BBB
:10AA10008093B10B80EF90E09093B40B8093B30BD5
:10AA20000DB407FEFDCF0E9423330E94462C8FEF0A
:10AA30009FEF9093BC0B8093BB0B9093BE0B8093C6
:10AA4000BD0B9093AC0B8093AB0B9093AE0B8093AC
:10AA5000AD0B0E94C72A0E94F8496CE073E0CE015A
:10AA600001960E94B924CE0101960E942847CE018A
:10AA700001960E949B2464E273E0CE0101960E943D
:10AA8000B924CE0101960E942847CE0101960E946A
:10AA90009B246BED79E0CE0101960E94B924CE0192
:10AAA00001960E942847CE0101960E949B246AEFDE
:10AAB00070E080E090E00E94222663E373E0CE0124
:10AAC00001960E94B924CE0101960E942847CE012A
:10AAD00001960E949B2462E573E0CE0101960E94DC
:10AAE000B924CE0101960E942847CE0101960E940A
:10AAF0009B2468E873E0CE0101960E94B924CE0140
:10AB000001960E942847CE0101960E949B2460E096
:10AB100086E30E94C72511E010930A0266E380E8ED
:10AB20009BE00E94082B811111C064EB73E0CE0101
:10AB300001960E94B924CE0101960E942847CE01B9
:10AB400001960E949B241092DF0925C066ED73E0F8
:10AB5000CE0107960E94B92480E89BE00E94553BF5
:10AB600060E170E0CE0107960E94DF23BE01695FBD
:10AB70007F4FCE0101960E94A024CE0101960E9433
:10AB80002847CE0101960E949B241093DF09CE0135
:10AB900007960E949B2467E387E79BE00E94082BAF
:10ABA000811111C062E074E0CE0101960E94B924C7
:10ABB000CE0101960E942847CE0101960E949B2457
:10ABC0001092DE0926C064E274E0CE0107960E946E
:10ABD000B92487E79BE00E94553B60E170E0CE011D
:10ABE00007960E94DF23BE01695F7F4FCE01019669
:10ABF0000E94A024CE0101960E942847CE01019612
:10AC00000E949B2481E08093DE09CE0107960E947A
:10AC10009B2468E38EE69BE00E94082B811111C003
:10AC200060E574E0CE0101960E94B924CE01019640
:10AC30000E942847CE0101960E949B241092DD09B4
:10AC400026C062E774E0CE0107960E94B9248EE622
:10AC50009BE00E94553B60E170E0CE0107960E94A8
:10AC6000DF23BE01695F7F4FCE0101960E94A024C1
:10AC7000CE0101960E942847CE0101960E949B2496
:10AC800081E08093DD09CE0107960E949B2469E351
:10AC900085E69BE00E94082B811111C06EE974E0EB
:10ACA000CE0101960E94B924CE0101960E94284748
:10ACB000CE0101960E949B241092DC0926C060EC14
:10ACC00074E0CE0107960E94B92485E69BE00E94BD
:10ACD000553B60E170E0CE0107960E94DF23BE0184
:10ACE000695F7F4FCE0101960E94A024CE0101969C
:10ACF0000E942847CE0101960E949B2481E0809308
:10AD0000DC09CE0107960E949B241092930A80E0F2
:10AD100090E00E94C72AEE24EA94FE2C04E110E0A1
:10AD200020EA30E040E050E060E070E08FE99BE036
:10AD30000E94272D84E08093BF0B1092B80B1092D5
:10AD4000B70B1092B60B1092B50B6CEE74E0CE01FF
:10AD500001960E94B92422E030E042E050E062E037
:10AD600070E089819A810E947D2910920A02CE01A9
:10AD700001960E949B24F0E42F2E33243394A6E303
:10AD80008A2E99249394B8E14B2E55245394612C28
:10AD9000712C0E948E4E2B8B3C8B4D8B5E8B6F8B60
:10ADA000788F0B891C89AD88BE882F89388D80915A
:10ADB000510B9091520BC090F109D090F209E090A4
:10ADC000F309F090F40982179307D4F50E945A26EC
:10ADD000C616D706E806F90608F0CBC3CD28CE285C
:10ADE000CF2809F4C6C3A0916A02B0916B0226EE87
:10ADF00030E00E943F63A30192010E94BC61DA012E
:10AE0000C9014996A11DB11D0CD91092F1091092EA
:10AE1000F2091092F3091092F4096AEF70E080E0F1
:10AE200090E00E942226C1018A199B098C52914010
:10AE3000899718F5065F1F4F0F311105F0F48AC48A
:10AE40000E945A26C616D706E806F90608F0E2C49C
:10AE5000CD28CE28CF2809F0E3C40E945A26DC0171
:10AE6000CB01805A9541AF4FBF4F8093F10990932A
:10AE7000F209A093F309B093F409C090940BD09019
:10AE8000950BE090960BF090970B0E945A2600913C
:10AE9000980B1091990B20919A0B30919B0B0C0DF4
:10AEA0001D1D2E1D3F1D68017901C61AD70AE80A2B
:10AEB000F90AD701C6018A3F9105A105B10558F4E9
:10AEC0008091E0099091E109029729F48091930A19
:10AED000882309F4AAC480910A02882309F4BBC21A
:10AEE0008091E0099091E1090097F1F530EEE32EB1
:10AEF000FF24FA9406E315E02EE630E040EA50E045
:10AF000064E170E080E090E00E94D84640EEE42EDC
:10AF100047E0F42E0DE315E02EE630E040EA50E085
:10AF200064E170E080EA90E00E94D8465FE1E52E9F
:10AF3000F12C03E415E02EE630E040EA50E062E850
:10AF400070E080E090E00E94D846809108029091E5
:10AF50000902E12C68EFF62E892B19F00BE415E0BD
:10AF60002CC000E515E029C08130910579F580EE0F
:10AF7000E82E87E0F82E06E515E02EE630E040EA00
:10AF800050E062E870E080E090E00E94D846E12C5A
:10AF900098EFF92E0CE515E02EE630E040E451E0A4
:10AFA00064E170E080E090E00E94D8460E94F02CBE
:10AFB0002FE1E22EF12C07E615E02EE630E040EA24
:10AFC00050E062E870E080EA90E0C5C0029709F0C6
:10AFD000C4C0EE24EA94FE2C0BED19E02CED30E019
:10AFE00040E451E064E170E080E090E00E94D846E7
:10AFF0000FE1E02EF12C07E615E02EE630E040EA06
:10B0000050E062E870E080EA90E00E94D8460E943A
:10B01000E51F9091070280910602992369F0882329
:10B0200029F0B0EEEB2EB7E0FB2E03C0E12CA8EF29
:10B03000FA2E0CE615E00CC0882329F0F0EEEF2E76
:10B04000F7E0FF2E03C0E12CE8EFFE2E01E313E052
:10B050002DE230E046E450E067E870E085E090E003
:10B060000E94D8469091050280910402992369F0CC
:10B07000882329F070EEE72E77E0F72E03C0E12C4D
:10B0800068EFF62E0FE615E00CC0882329F050EE8D
:10B09000E52E57E0F52E03C0E12C48EFF42E07E82B
:10B0A00015E02DE230E046E450E067E870E085E529
:10B0B00090E00E94D8469091030280910202992369
:10B0C00069F0882329F030EEE32E37E0F32E03C039
:10B0D000E12C28EFF22E02E715E00CC0882329F0BE
:10B0E00090EEE92E97E0F92E03C0E12C88EFF82EC0
:10B0F00005E715E02DE230E046E450E06EEB70E04D
:10B1000085E090E00E94D846909101028091000273
:10B11000992369F0882329F000EEE02E07E0F02E55
:10B1200003C0E12C18EFF12E07E715E00CC08823CF
:10B1300029F0B0EEEB2EB7E0FB2E03C0E12CA8EF18
:10B14000FA2E0AE715E02DE230E046E450E06EEB1F
:10B1500070E085E590E00E94D8468091E0099091EA
:10B16000E109039709F0FCC0EE24EA94FE2C0BEDF4
:10B1700019E02CED30E040E451E064E170E080E063
:10B1800090E00E94D846FFE1EF2EF12C07E615E093
:10B190002EE630E040EA50E062E870E080EA90E0BD
:10B1A0000E94D84684E992E00E946246909107028C
:10B1B00080910602992369F0882329F070EEE72E2A
:10B1C00077E0F72E03C0E12C68EFF62E0CE615E0D1
:10B1D0000CC0882329F050EEE52E57E0F52E03C071
:10B1E000E12C48EFF42E01E313E02DE230E046E4D9
:10B1F00050E067E870E085E090E00E94D8469091CA
:10B20000050280910402992369F0882329F030EE29
:10B21000E32E37E0F32E03C0E12C28EFF22E0FE6E9
:10B2200015E00CC0882329F090EEE92E97E0F92E66
:10B2300003C0E12C88EFF82E07E815E02DE230E09E
:10B2400046E450E067E870E085E590E00E94D8466B
:10B250009091030280910202992369F0882329F0DA
:10B2600000EEE02E07E0F02E03C0E12C18EFF12EE7
:10B2700002E715E00CC0882329F0B0EEEB2EB7E012
:10B28000FB2E03C0E12CA8EFFA2E05E715E02DE216
:10B2900030E046E450E06EEB70E085E090E00E9424
:10B2A000D8469091010280910002992369F0882389
:10B2B00029F0F0EEEF2EF7E0FF2E03C0E12CE8EFCF
:10B2C000FE2E07E715E00CC0882329F070EEE72E6C
:10B2D00077E0F72E03C0E12C68EFF62E0AE715E0C1
:10B2E0002DE230E046E450E06EEB70E085E590E062
:10B2F0000E94D8466CE775E0CE0101960E94B92401
:10B30000AE014F5F5F4F69E170E08FE090E00E9417
:10B31000BA2ACE0101960E949B246CE478E0CE010B
:10B3200001960E94B924AE014F5F5F4F67E370E062
:10B330008FE090E00E94BA2ACE0101960E949B24E1
:10B3400050E2E52E5DEFF52E02E815E02EE630E046
:10B3500040EA50E064E170E080EA90E00E94D84664
:10B360008091E0099091E109049709F072C04FE1E2
:10B37000E42EF12C07E615E02EE630E040EA50E03E
:10B3800062E870E080EA90E00E94D84680915B021B
:10B39000882379F1EE24EA9427E0F22E0BED19E0F0
:10B3A0002EE630E040E451E064E170E080E090E0BF
:10B3B0000E94D84630E2E32E3DEFF32E09E815E077
:10B3C0002EE630E040EA50E062E870E080E090E095
:10B3D0000E94D84681E592E00E94EC4587E492E025
:10B3E0000E9462468DE392E00E94E64483E392E08D
:10B3F0002EC08FEEE82E83E0F82E0BED19E02EE63E
:10B4000030E040E451E064E170E080E090E00E94D0
:10B41000D84690E2E92E9DEFF92E04E915E02EE6DC
:10B4200030E040EA50E062E870E080E090E00E94A6
:10B43000D84689E292E00E94EC458FE192E00E94BA
:10B44000624685E192E00E94E6448BE092E00E9431
:10B45000694510920A0284E99AE00E94A321181615
:10B4600019060CF07BC06BED79E0CE0101960E94CD
:10B47000B9240E94D74F97FD0CC08F83188641E0F6
:10B4800050E0BE01695F7F4FCE0101960E945223BA
:10B49000F0CF6DE975E0CE0107960E94B9244D8189
:10B4A0005E8169817A81CE0107960E9452238111C3
:10B4B00004C0CE0107960E945524BE01695F7F4FEC
:10B4C000CE010D960E94A024CE0107960E949B24D7
:10B4D000CE0101960E949B2429893A8926333105A1
:10B4E00030F125E330E040E050E0BE01635F7F4F84
:10B4F000CE0101960E94CD24CE0101960E942847DC
:10B50000CE0101960E949B2429893A8945E350E0A7
:10B51000BE01635F7F4FCE0101960E94CD24BE0124
:10B520006F5F7F4FCE010D960E941C24D1CF21501A
:10B53000310940E050E0BE01635F7F4FCE010196CC
:10B540000E94CD24CE0101960E942847CE0101968B
:10B550000E949B24CE010D960E949B2484E99BE0CF
:10B560000E94EB3389E89BE00E94EB330E9440226B
:10B5700010CC1092F1091092F2091092F309109276
:10B58000F409C090B30BD090B40B0D2C000CEE0856
:10B59000FF08C801110FAA0BBB0B9C01AD0124567B
:10B5A00031094109510966277727CB016C197D09BB
:10B5B0008E099F090E94156320E233E040E050E0CD
:10B5C000DBD6DA01C9018C0D9D1DAE1DBF1D898F13
:10B5D0009A8FAB8FBC8FC090B10BD090B20B0D2C5B
:10B5E000000CEE08FF08C501BB0CAA0BBB0B9C01AD
:10B5F000AD01265931094109510966277727CB0149
:10B600006C197D098E099F090E9415632EEE32E0A8
:10B6100040E050E0B1D6C20ED31EE41EF51E560126
:10B62000898D9A8DC3978F349105A8F58091E00993
:10B630009091E109019779F5C4018C199D0997FD55
:10B6400005C090936B0280936A0204C010926B0253
:10B6500010926A0280916A0290916B028931914046
:10B6600034F088E191E090936B0280936A02A0919C
:10B670006A02B0916B0226EE30E00E943F63A301A4
:10B6800092017AD6DA01C9014996A11DB11D0E9425
:10B6900011500E94F02C8091E0099091E1090397EC
:10B6A00021F484E992E00E949C438091E00990910A
:10B6B000E109049719F580915B02882379F081E50F
:10B6C00092E00E94094187E492E00E9452428DE399
:10B6D00092E00E947C3E83E392E00EC089E292E019
:10B6E0000E9409418FE192E00E94524285E192E07E
:10B6F0000E947C3E8BE092E00E94C23F098D1A8D31
:10B70000C1018C199D09803A910534F40238110564
:10B710006CF460E070E010C0803A910509F483CBCE
:10B720000238110564F460E070E00FC003381105C1
:10B730000CF479CB61E070E080E090E008C0033861
:10B7400011050CF470CB61E070E081E090E00E94A4
:10B75000A44769CB8091930A91E089278093930A4B
:10B76000811143C091E090930A0280E090E00E9432
:10B77000C72AEE24EA94FE2C04E110E020EA30E02F
:10B7800040E050E060E070E08FE99BE00E94272DF0
:10B790001092B80B1092B70B1092B60B1092B50B1B
:10B7A0006CEE74E0CE0107960E94B92422E030E0EE
:10B7B00042E050E062E070E08F8198850E947D2930
:10B7C0000E946B1E69EF74E0CE0101960E94B924BD
:10B7D000CE0101960E942847CE0101960E949B242B
:10B7E000CE0107960E949B2448CB65E175E0CE010F
:10B7F00001960E94B924CE0101960E942847CE01ED
:10B8000001960E949B2464EF71E080E090E00E942A
:10B81000222633CBCD28CE28CF2809F02ECB1DCB26
:10B8200080E090E00E94115028CB0E94E51F53CB8E
:10B83000EF92FF920F931F93CF93DF93E4E9FAE027
:10B840001382128288EE93E0A0E0B0E084839583B7
:10B85000A683B7832CEA32E03183208325EC30E0E5
:10B860003587248724EC30E03787268720EC30E0CA
:10B87000318B208B21EC30E0338B228B22EC30E0BB
:10B88000358B248B26EC30E0378B268B118E128E75
:10B89000138E148E03E31BE0F8011382128284835B
:10B8A0009583A683B7838EEB92E091838083E1E357
:10B8B000FBE080E580831182E7EDFBE015821682D4
:10B8C0001186138682E090E0A0E0B0E0848795873F
:10B8D000A687B78713A215A614A680ED92E093A7BA
:10B8E00082A717A6A4ECBBE080E215968C9315976F
:10B8F00086E116968C931697E7E2FBE2E4911796A1
:10B90000EC931797E1EEFAE2E4911896EC9318970E
:10B9100040E85EE360E070E01D964D935D936D93AB
:10B920007C935097CFE9DBE01B821A828CED92E08A
:10B930009983888360E088E00E94982561E088E030
:10B940000E94C7258BE0E82EFF24F394F701808145
:10B950008260808361E080E30E94C725F7018081D7
:10B960008160808361E081E30E94C72580EF90E0E1
:10B970009B8B8A8B80E491E09D8B8C8B1BA219861C
:10B9800018861B861A8621E028A329A38FEF9FEF34
:10B990009F8B8E8B198E188E198A188A2CA31AA247
:10B9A0009D8F8C8F9F8F8E8F9D878C879F878E8793
:10B9B00086ED90E09B8F8A8FE4E9FBE0128611868A
:10B9C00010861082118212821382148215821682CE
:10B9D0001782E9E8FBE01286118610861082118238
:10B9E000128213821482158216821782E0E8FBE02D
:10B9F0001382128284EF92E0918380831683058301
:10BA0000E7E7FBE01382128291838083168305832C
:10BA1000EEE6FBE013821282918380831683058316
:10BA2000E5E6FBE01382128291838083168305830F
:10BA3000A1E5BBE08AE312968C9312978BE31496F0
:10BA40008C9314978EE113968C9313978FE1159630
:10BA50008C9315978DE491E017969C938E9316978F
:10BA6000E0EEFAE2E491F0E0EE0FFF1FE955F54D4C
:10BA70008591949119969C938E931897EBEFFAE227
:10BA8000E491F0E0EE0FFF1FE955F54D859194919B
:10BA90001B969C938E931A97ECEFFAE2E491F0E0F8
:10BAA000EE0FFF1FE955F54D859194911D969C93DE
:10BAB0008E931C97EFEDFAE2E491F0E0EE0FFF1F9A
:10BAC000E955F54D859194911F969C938E931E9701
:10BAD000E6E2FBE2E4915096EC935097E1E4FBE25E
:10BAE000E4915296EC935297E2E4FBE2E491519692
:10BAF000EC935197E5E2FBE2E4915396EC93539774
:10BB00008AE090E08D939C936BED79E08BE49BE071
:10BB10000E94B9246BED79E085E49BE00E94B92492
:10BB20006BED79E08FE39BE00E94B924809198024D
:10BB30009091990290938F0280938E029093850248
:10BB40008093840290937B0280937A029093710297
:10BB500080937002DF91CF911F910F91FF90EF9032
:10BB600008958FE39BE00E949B2485E49BE00E9464
:10BB70009B248BE49BE00C949B24EF920F931F93E8
:10BB8000CF93DF93E80147FD02C034E001C034E108
:10BB9000E42F440FFF0BF7FF03C0F195E195F10986
:10BBA000E32E022F2E2FAE0159D0CE01DF91CF917F
:10BBB0001F910F91EF900895BB274A3031F49923DC
:10BBC00022F4BDE2909581959F4F30C0BB272A306B
:10BBD00051F4992342F4BDE290958095709561955A
:10BBE0007F4F8F4F9F4F01C0BB27FA01A62F6217CF
:10BBF000710581059105330B30FB66F0AA27660FAE
:10BC0000771F881F991FAA1FA21710F0A21B639508
:10BC10003850A9F7A05DAA3308F0A95DA19336F7C3
:10BC2000B111B1931082CA017EC2BB27FB01552717
:10BC3000AA27880F991FAA1FA41710F0A41B839589
:10BC40005051B9F7A05DAA3308F0A95DA193009700
:10BC500079F7B111B1931192CB0165C24F925F9206
:10BC60006F927F929F92AF92BF92CF92DF92EF92AC
:10BC7000FF920F931F93CF93DF93CDB7DEB7299732
:10BC80000FB6F894DEBF0FBECDBF6A01122FB02EE3
:10BC90002BE3201720F0FF24F394F00E02C0BCE346
:10BCA000FB2E0F2D27E0AE014F5F5F4F64D1AC013B
:10BCB0008981982F9970913031F0E1FC06C0E0FE47
:10BCC00006C090E205C09DE203C09BE201C090E087
:10BCD000EE2DE07183FF3CC0911102C083E001C0F2
:10BCE00084E0811718F4212F281B01C020E0E11106
:10BCF0000BC0F601822F30E2882319F03193815076
:10BD0000FBCFC20ED11C20E0992329F0D6019C93D1
:10BD1000F60131966F01C6010396E2FE0AC03EE4C9
:10BD2000D6013C9341E411964C93119712963C93A3
:10BD300006C03EE6F601308341E641833283FC01D2
:10BD4000322F40E2332309F442C041933150FACFFD
:10BD500082FF44C0911102C083E001C084E08117DA
:10BD600018F4212F281B01C020E0E1110BC0F601BF
:10BD7000822F30E2882319F031938150FBCFC20E1D
:10BD8000D11C20E0992329F0D6019C93F60131962D
:10BD90006F01C6010396E2FE0BC039E4D6013C9365
:10BDA0003EE411963C93119736E412963C9307C0FB
:10BDB00039E6F60130833EE6318336E63283FC0114
:10BDC000322F40E2332319F041933150FBCFFC0175
:10BDD000E20FF11D10828EEF9FEFB7C0F1E09111DD
:10BDE00001C0F0E06F2F70E01416150624F49A01DC
:10BDF0002F5F3F4F02C021E030E0260F371FBB20EE
:10BE000029F06B2D70E06F5F7F4F02C060E070E043
:10BE1000260F371F612F70E0261737071CF4121BFF
:10BE2000212F01C020E03E2D387159F4D601322F68
:10BE300060E2332319F06D933150FBCFC20ED11C59
:10BE400020E0FF2331F0D6019C93B6016F5F7F4F56
:10BE50006B01E1110BC0F601922F30E3992319F029
:10BE600031939150FBCFC20ED11C20E09F2D940F37
:10BE70003A81782F7071A72E84FF03C0313309F403
:10BE80009150191624F4993018F098E001C091E00F
:10BE9000E42F852F57FF02C0E0E080E06E2F782F5F
:10BEA000E0E0F0E0AEE29A2E3A01691A71082A0148
:10BEB000461A570A0B2D10E01195019511096F3F95
:10BEC0008FEF780729F4D6019C92C60101966C0188
:10BED0004617570784F0661677066CF47F01E40C6A
:10BEE000F51CA1E0B0E0AC0FBD1FEA0EFB1ED701B0
:10BEF0001196BC9002C090E3B92E61507109319641
:10BF0000C60101967C016017710724F0D601BC922E
:10BF10006C01D5CF6417750741F4363320F43533FF
:10BF200021F4A11002C081E3B82EF601B082F7011E
:10BF3000822F90E2882319F091938150FBCFF70173
:10BF4000E20FF11D108280E090E029960FB6F89480
:10BF5000DEBF0FBECDBFDF91CF911F910F91FF903C
:10BF6000EF90DF90CF90BF90AF909F907F906F90B9
:10BF70005F904F900895283008F027E03327DA01CA
:10BF8000990F311D87FD916000966105710539F4A7
:10BF900032602E5F3D9330E32A95E1F708959F3F8D
:10BFA00030F080387105610509F03C5F3C5F3D93DE
:10BFB000913008F08068911DDF93CF931F930F930A
:10BFC000FF92EF92192F987F9695E92F9695969567
:10BFD000E90FFF27EA55FE4F99273327EE24FF2468
:10BFE000A701E70105900894079428F4360FE71E8F
:10BFF000F81E491F511D660F771F881F991F069451
:10C00000A1F70590079428F4E70EF81E491F561F64
:10C01000C11D770F881F991F661F0694A1F7059011
:10C02000079428F4F80E491F561FC71FD11D880F0B
:10C03000991F661F771F0694A1F70590079420F4B7
:10C04000490F561FC71FD81F990F661F771F881FDC
:10C050000694A9F784911095177041F0D695C7956D
:10C0600057954795F794E7941A95C1F7ECE4F1E0FA
:10C0700068941590159135916591959105907FE2A1
:10C080007395E118F10A430B560BC90BD009C0F7A1
:10C09000E10CF11E431F561FC91FD01D7EF47033E3
:10C0A00011F48A95E6CFE894015030F0080F0AF4B5
:10C0B0000027021708F4202F2395022F7A3328F047
:10C0C00079E37D932A95E9F710C07D932A9589F647
:10C0D000069497956795379517951794E118F10A87
:10C0E000430B560BC90BD00998F023957E9173959D
:10C0F0007A3308F070E37C932013B8F77E91706177
:10C100007D9330F0839571E37D9370E32A95E1F799
:10C110001124EF90FF900F911F91CF91DF919927FC
:10C1200087FD90950895DC01FC01672F71917723BD
:10C13000E1F7329704C07C916D9370836291AE17E2
:10C14000BF07C8F3089540D008F481E00895E8944B
:10C1500009C097FB3EF490958095709561957F4F4F
:10C160008F4F9F4F9923A9F0F92F96E9BB279395FD
:10C17000F695879577956795B795F111F8CFFAF40D
:10C18000BB0F11F460FF1BC06F5F7F4F8F4F9F4F3E
:10C1900016C0882311F096E911C0772321F09EE89C
:10C1A000872F762F05C0662371F096E8862F70E002
:10C1B00060E02AF09A95660F771F881FDAF7880FDC
:10C1C0009695879597F90895990F0008550FAA0B32
:10C1D000E0E8FEEF16161706E807F907C0F012169A
:10C1E0001306E407F50798F0621B730B840B950B9D
:10C1F00039F40A2661F0232B242B252B21F40895F2
:10C200000A2609F4A140A6958FEF811D811D08958E
:10C210000BD078C069D028F06ED018F0952309F0C3
:10C220005AC05FC01124A2C07ED0A0F3959FD1F365
:10C23000950F50E0551F629FF001729FBB27F00DD4
:10C24000B11D639FAA27F00DB11DAA1F649F662729
:10C25000B00DA11D661F829F2227B00DA11D621F78
:10C26000739FB00DA11D621F839FA00D611D221F32
:10C27000749F3327A00D611D231F849F600D211D16
:10C28000822F762F6A2F11249F5750408AF0E1F0B9
:10C2900088234AF0EE0FFF1FBB1F661F771F881F02
:10C2A00091505040A9F79E3F510570F014C05EC0F8
:10C2B0005F3FECF3983EDCF3869577956795B795ED
:10C2C000F795E7959F5FC1F7FE2B880F911D969517
:10C2D000879597F9089597F99F6780E870E060E087
:10C2E00008959FEF80EC089500240A94161617060F
:10C2F00018060906089500240A9412161306140657
:10C3000005060895092E0394000C11F4882352F0B9
:10C31000BB0F40F4BF2B11F460FF04C06F5F7F4F71
:10C320008F4F9F4F089557FD9058440F551F59F058
:10C330005F3F71F04795880F97FB991F61F09F3F12
:10C3400079F087950895121613061406551FF2CF3B
:10C350004695F1DF08C0161617061806991FF1CF8B
:10C3600086957105610508940895E894BB276627B2
:10C370007727CB0197F90895052E97FB16F40094C3
:10C380000FD057FD05D01ED007FC02D046F408C0E0
:10C3900050954095309521953F4F4F4F5F4F0895F1
:10C3A00090958095709561957F4F8F4F9F4F089521
:10C3B0002BD0A59F900DB49F900DA49F800D911D33
:10C3C00011240895A1E21A2EAA1BBB1BFD010DC06A
:10C3D000AA1FBB1FEE1FFF1FA217B307E407F50735
:10C3E00020F0A21BB30BE40BF50B661F771F881F11
:10C3F000991F1A9469F760957095809590959B01A7
:10C40000AC01BD01CF010895A29FB001B39FC0014F
:10C41000A39F700D811D1124911DB29F700D811D70
:10C420001124911D08955058BB27AA270ED06ACF1A
:10C430005BDF30F060DF20F031F49F3F11F41EF439
:10C4400050CF0EF4E095E7FB46CFE92F6CDF80F389
:10C45000BA17620773078407950718F071F49EF501
:10C4600084CF0EF4E0950B2EBA2FA02D0B01B9014D
:10C4700090010C01CA01A0011124FF27591B99F05A
:10C48000593F50F4503E68F11A16F040A22F232F66
:10C49000342F4427585FF3CF469537952795A795B6
:10C4A000F0405395C9F77EF41F16BA0B620B730B5D
:10C4B000840BBAF09150A1F0FF0FBB1F661F771FCE
:10C4C000881FC2F70EC0BA0F621F731F841F48F483
:10C4D000879577956795B795F7959E3F08F0B3CF09
:10C4E0009395880F08F09927EE0F979587950895F3
:10C4F0000CD008CF00DF40F0F7DE30F021F45F3FD2
:10C5000019F0E9CE511132CFECCE0DDF98F399231B
:10C51000C9F35523B1F3951B550BBB27AA27621707
:10C520007307840738F09F5F5F4F220F331F441F4C
:10C53000AA1FA9F333D00E2E3AF0E0E830D0915084
:10C540005040E695001CCAF729D0FE2F27D0660F71
:10C55000771F881FBB1F261737074807AB07B0E8B0
:10C5600009F0BB0B802DBF01FF2793585F4F2AF0C6
:10C570009E3F510568F0AFCEF9CE5F3FECF3983E99
:10C58000DCF3869577956795B795F7959F5FC9F723
:10C59000880F911D9695879597F90895E1E0660FAC
:10C5A000771F881FBB1F621773078407BA0720F025
:10C5B000621B730B840BBA0BEE1F88F7E09508958E
:10C5C00004D06894B111D2CE0895B5DE88F09F579B
:10C5D00090F0B92F9927B751A0F0D1F0660F771FCF
:10C5E000881F991F1AF0BA95C9F712C0B13081F0AF
:10C5F000BCDEB1E00895B9CE672F782F8827B85FE9
:10C6000039F0B93FCCF3869577956795B395D9F70F
:10C610003EF490958095709561957F4F8F4F9F4F19
:10C620000895D2DD08F48FEF0895DB018F939F9377
:10C63000BFDEBF91AF91A29F800D911DA39F900D72
:10C64000B29F900D1124089597FB072E16F40094C5
:10C6500006D077FD08D019D007FC05D03EF49095A0
:10C6600081959F4F0895709561957F4F0895EE0FC6
:10C67000FF1F881F8BBF0790F691E02D1994C4DE31
:10C68000B7FF0895821B930B0895AA1BBB1B51E1B2
:10C6900007C0AA1FBB1FA617B70710F0A61BB70B32
:10C6A000881F991F5A95A9F780959095BC01CD01D7
:10C6B0000895CF93DF938230910510F482E090E0EB
:10C6C000E0914F0EF091500E20E030E0C0E0D0E05D
:10C6D000309711F14081518148175907C0F0481730
:10C6E000590761F482819381209719F09B838A8393
:10C6F0002BC09093500E80934F0E26C0211531050C
:10C7000019F04217530718F49A01BE01DF01EF0137
:10C710000280F381E02DDCCF2115310509F1281BC2
:10C72000390B2430310590F412968D919C9113971A
:10C730006115710521F0FB019383828304C09093FE
:10C74000500E80934F0EFD01329644C0FD01E20F62
:10C75000F31F81939193225031092D933C933AC05A
:10C7600020914D0E30914E0E232B41F42091A402C6
:10C770003091A50230934E0E20934D0E2091A202CF
:10C780003091A3022115310541F42DB73EB74091F8
:10C79000A6025091A702241B350BE0914D0EF0919B
:10C7A0004E0EE217F307A0F42E1B3F0B2817390794
:10C7B00078F0AC014E5F5F4F2417350748F04E0FFD
:10C7C0005F1F50934E0E40934D0E8193919302C084
:10C7D000E0E0F0E0CF01DF91CF9108950F931F9338
:10C7E000CF93DF93009709F48CC0FC01329713823A
:10C7F000128200914F0E1091500E0115110581F417
:10C8000020813181820F931F20914D0E30914E0E69
:10C810002817390779F5F0934E0EE0934D0E71C04D
:10C82000D80140E050E0AE17BF0750F412962D91AA
:10C830003C911397AD012115310509F1D901F3CFD1
:10C840009D01DA013383228360817181860F971FF6
:10C850008217930769F4EC0128813981260F371F6D
:10C860002E5F3F4F318320838A819B819383828314
:10C87000452B29F4F093500EE0934F0E42C01396CF
:10C88000FC93EE931297ED01499159919E01240F6B
:10C89000351FE217F30771F480819181840F951F92
:10C8A000029611969C938E938281938113969C930A
:10C8B0008E931297E0E0F0E0D80112968D919C9152
:10C8C0001397009719F0F8018C01F6CF8D919C9188
:10C8D00098012E5F3F4F820F931F20914D0E309194
:10C8E0004E0E2817390769F4309729F41092500E2C
:10C8F00010924F0E02C01382128210934E0E0093BC
:10C900004D0EDF91CF911F910F9108956F927F92FD
:10C910008F929F92AF92BF92CF92DF92EF92FF924F
:10C920000F931F93CF93DF93EC01009781F4CB011A
:10C93000DF91CF911F910F91FF90EF90DF90CF90FB
:10C94000BF90AF909F908F907F906F90B2CEFC0180
:10C95000E60FF71F9C0122503109E217F30708F494
:10C96000A8C0D9010D911C91119706171707A8F0BF
:10C970000530110508F49BC0C80104978617970776
:10C9800008F495C002501109061B170B019311936F
:10C990006D937C93CF0122DF8AC05B01A01AB10A9C
:10C9A0004C01800E911EA0914F0EB091500E40E0B0
:10C9B00050E0E12CF12C109709F44AC0A815B905F4
:10C9C000D1F56D907C901197630182E0C80ED11C67
:10C9D000CA14DB0480F1A3014A195B096A0182E0F1
:10C9E000C80ED11C1296BC9012971396AC91B5E06C
:10C9F000CB16D10440F0B282A38351834083D90186
:10CA00006D937C930AC00E5F1F4FC301800F911F6F
:10CA1000F90191838083EB2DFA2FE114F10431F0B9
:10CA2000D7011396FC93EE93129741C0F093500EEA
:10CA3000E0934F0E3CC08D919C9111974817590778
:10CA400008F4AC017D0112960D90BC91A02DB3CFDE
:10CA500080914D0E90914E0E88159905E1F4461780
:10CA60005707C8F48091A2029091A302009741F465
:10CA70008DB79EB74091A6025091A702841B950BDB
:10CA8000E817F907B0F4F0934E0EE0934D0EF9015C
:10CA9000718360830CC0CB010CDE7C01009749F0F0
:10CAA000A801BE011BD0CE0199DEC70104C0CE0192
:10CAB00002C080E090E0DF91CF911F910F91FF9035
:10CAC000EF90DF90CF90BF90AF909F908F907F902E
:10CAD0006F90089581E090E0F89410C0FB01DC01B4
:10CAE00002C001900D9241505040D8F70895FB01CB
:10CAF000DC0101900D920020E1F7089518E1C8E4EF
:10CB0000D8E100E005C0802FFE01B1DD2196011DB6
:0ECB1000C934D10780E00807B1F7F894FFCFD1
:10CB1E000100010001000100010001CD00410041B2
:10CB2E000028009600CD001E005000280096002D13
:10CB3E000041004100000064002D001E004B00006B
:10CB4E00006400CD004100410028009600CD001E7B
:10CB5E00005500280096002D004100500000006492
:10CB6E00002D001E005A0000006400013700550021
:10CB7E003C0064000A005A002C011801C800320063
:10CB8E00000014002C01C8003200000014002C011B
:10CB9E00C8003200000014002C01C8003200000052
:10CBAE0014002C012D004600140014002C01FFFF70
:10CBBE00FFFF0000510E800000000000D921472128
:10CBCE0072211F22A3218121952100000000BE3772
:10CBDE0009287D18FD2221230D23FE2200000000CE
:10CBEE00A43C47217D187C1800000000103247211C
:10CBFE007D187C1800000000292347217D187C1821
:10CC0E0000000000583947217D187C189439E13A0C
:10CC1E00733921390001020300010203426F6F7460
:10CC2E00696E6720477265656E686F7573654F53E1
:10CC3E002E2E2E0056657273696F6E3A20302E348A
:10CC4E002E31005B4641494C45445D205344204300
:10CC5E00617264206E6F74206465746563746564BC
:10CC6E0021005B20204F4B20205D20456E61626CC1
:10CC7E00696E6720706F776572736176696E672073
:10CC8E0066656174757265732E2E2E20202020200D
:10CC9E0020202020202020005B4641494C45445D49
:10CCAE0020506F776572736176696E673A204172B4
:10CCBE0067756D656E74206D757374206265203EA8
:10CCCE0020302E005B20494E464F205D20536F6969
:10CCDE006C2073656E736F72203120756E706C757B
:10CCEE00676765642E005B20204F4B20205D20532C
:10CCFE006F696C2073656E736F72203120636F6E77
:10CD0E006E65637465642E2056657273696F6E3A34
:10CD1E0020005B20494E464F205D20536F696C20EA
:10CD2E0073656E736F72203220756E706C756767E7
:10CD3E0065642E005B20204F4B20205D20536F69D1
:10CD4E006C2073656E736F72203220636F6E6E652A
:10CD5E00637465642E2056657273696F6E3A200097
:10CD6E005B20494E464F205D20536F696C207365E2
:10CD7E006E736F72203320756E706C7567676564A5
:10CD8E002E005B20204F4B20205D20536F696C20BE
:10CD9E0073656E736F72203320636F6E6E6563748E
:10CDAE0065642E2056657273696F6E3A20005B20A3
:10CDBE00494E464F205D20536F696C2073656E732C
:10CDCE006F72203420756E706C75676765642E0007
:10CDDE005B20204F4B20205D20536F696C207365C4
:10CDEE006E736F72203420636F6E6E65637465644C
:10CDFE002E2056657273696F6E3A20005761746506
:10CE0E0072204C6576656C3A005B20494E464F2089
:10CE1E005D20457869746564206465627567206D70
:10CE2E006F64652E005B20494E464F205D20537780
:10CE3E0069746368656420746F2064656275672029
:10CE4E006D6F64652E0053797374656D0053746154
:10CE5E007473004F7074696F6E730053746F70004B
:10CE6E00537461727400526573657400427269671F
:10CE7E0068746E657373004261636B00312A003211
:10CE8E002A00332A003300342A00340057617465B7
:10CE9E007200506167652032004E69676874204DDC
:10CEAE006F646500446179204D6F6465005365724F
:10CEBE0069616C3A20005B20204F4B20205D20538F
:10CECE006F696C2073656E736F7220322074656D9E
:10CEDE0070657261747572653A200020432C2000D3
:10CEEE002046005B20204F4B20205D20536F696C45
:10CEFE002073656E736F722032206D6F6973747557
:10CF0E0072653A200025005B20204F4B20205D20CB
:10CF1E00536F696C2073656E736F72203120746568
:10CF2E006D70657261747572653A20005B20204FDA
:10CF3E004B20205D20536F696C2073656E736F728A
:10CF4E002031206D6F6973747572653A20005761D8
:10CF5E00746572696E672120506C65617365207708
:10CF6E006169742E005B20204F4B20205D20487598
:10CF7E006D69646974793A2000252C2054656D70B2
:10CF8E00657261747572653A20005B20494E464F9A
:10CF9E00205D20536F696C2073656E736F72203144
:10CFAE0020636F6E6E65637465642E005B20494E60
:10CFBE00464F205D20536F696C2073656E736F72E0
:10CFCE00203220636F6E6E65637465642E005B2085
:10CFDE00494E464F205D20536F696C2073656E730A
:10CFEE006F72203320636F6E6E65637465642E00FE
:10CFFE005B20494E464F205D20536F696C20736550
:10D00E006E736F72203420636F6E6E656374656429
:10D01E002E005B20494E464F205D2052756E6E6984
:10D02E006E67207761746572206F6E20626F782054
:10D03E003120666F722000207365632E005B2049DD
:10D04E004E464F205D2052756E6E696E6720776179
:10D05E00746572206F6E20626F78203220666F7258
:10D06E0020005B20494E464F205D2052756E6E6942
:10D07E006E67207761746572206F6E20626F782004
:10D08E003320666F7220005B20494E464F205D2094
:10D09E0052756E6E696E67207761746572206F6E61
:10D0AE0020626F78203420666F72200042617474A3
:10D0BE006572793A20005573696E6720736F6C61E3
:10D0CE00722E005B20494E464F205D2055706461E4
:10D0DE0074696E6720737461746973746963732EF7
:10D0EE0000206465677265657300206D696E7574E6
:10D0FE00657320756E74696C207761746572004972
:10D10E006E74616B652046616E004578686175735B
:10D11E00742046616E00496E2073796E6300506C08
:10D12E00616E7420426F7820312044697361626CA5
:10D13E00656400456E61626C6500506C616E7420B2
:10D14E00426F78203120456E61626C6564004469DF
:10D15E007361626C6500576174657220616D6F75E5
:10D16E006E743A00506C616E7420426F78203220DB
:10D17E0044697361626C656400506C616E74204228
:10D18E006F78203220456E61626C656400506C6170
:10D19E006E7420426F7820332044697361626C652F
:10D1AE006400506C616E7420426F78203320456E9F
:10D1BE0061626C656400506C616E7420426F782001
:10D1CE00342044697361626C656400506C616E74E6
:10D1DE0020426F78203420456E61626C6564005881
:10D1EE00203D20000959203D2000095072657373BF
:10D1FE00757265203D20005B20494E464F205D2014
:10D20E00546F67676C696E6720626F7820312E00ED
:10D21E005B20494E464F205D20546F67676C696EE8
:10D22E006720626F7820322E005B20494E464F20D9
:10D23E005D20546F67676C696E6720626F7820336C
:10D24E002E005B20494E464F205D20546F67676C61
:10D25E00696E6720626F7820342E005B20204F4B62
:10D26E0020205D20536F696C2073656E736F722082
:10D27E00342074656D70657261747572653A200044
:10D28E005B20204F4B20205D20536F696C2073650F
:10D29E006E736F722034206D6F6973747572653A98
:10D2AE0020005B20204F4B20205D20536F696C20A7
:10D2BE0073656E736F7220332074656D7065726165
:10D2CE00747572653A20005B20204F4B20205D2044
:10D2DE00536F696C2073656E736F722033206D6FA0
:0CD2EE006973747572653A20000D0A0027
:020000023000CC
:10E000000D9489F10D94B2F10D94B2F10D94B2F129
:10E010000D94B2F10D94B2F10D94B2F10D94B2F1F0
:10E020000D94B2F10D94B2F10D94B2F10D94B2F1E0
:10E030000D94B2F10D94B2F10D94B2F10D94B2F1D0
:10E040000D94B2F10D94B2F10D94B2F10D94B2F1C0
:10E050000D94B2F10D94B2F10D94B2F10D94B2F1B0
:10E060000D94B2F10D94B2F10D94B2F10D94B2F1A0
:10E070000D94B2F10D94B2F10D94B2F10D94B2F190
:10E080000D94B2F10D94B2F10D94B2F10D94B2F180
:10E090000D94B2F10D94B2F10D94B2F10D94B2F170
:10E0A0000D94B2F10D94B2F10D94B2F10D94B2F160
:10E0B0000D94B2F10D94B2F10D94B2F10D94B2F150
:10E0C0000D94B2F10D94B2F10D94B2F10D94B2F140
:10E0D0000D94B2F10D94B2F10D94B2F10D94B2F130
:10E0E0000D94B2F141546D656761323536300041AF
:10E0F000726475696E6F206578706C6F72657220DE
:10E1000073746B3530305632206279204D4C530099
:10E11000426F6F746C6F616465723E004875683F52
:10E1200000436F6D70696C6564206F6E203D200048
:10E130004350552054797065202020203D20005FF9
:10E140005F4156525F415243485F5F3D2000415658
:10E1500052204C696243205665723D20004743437C
:10E160002056657273696F6E203D20004350552024
:10E1700049442020202020203D20004C6F7720663D
:10E18000757365202020203D20004869676820665F
:10E190007573652020203D200045787420667573D6
:10E1A00065202020203D20004C6F636B2066757336
:10E1B000652020203D20004D617220203720323024
:10E1C000313300312E362E3800342E332E350056A2
:10E1D00023202020414444522020206F7020636F70
:10E1E00064652020202020696E73747275637469E1
:10E1F0006F6E2061646472202020496E74657272B3
:10E20000757074006E6F20766563746F7200726A49
:10E210006D702020006A6D70200057686174207056
:10E220006F72743A00506F7274206E6F7420737541
:10E2300070706F72746564004D7573742062652030
:10E2400061206C6574746572002000577269747483
:10E25000696E672045450052656164696E672045B7
:10E26000450045452065727220636E743D00504F35
:10E27000525400303D5A65726F2061646472003FF1
:10E280003D43505520737461747300403D454550C3
:10E29000524F4D207465737400423D426C696E6B41
:10E2A000204C454400453D44756D70204545505215
:10E2B0004F4D00463D44756D7020464C415348001B
:10E2C000483D48656C70004C3D4C69737420492F83
:10E2D0004F20506F72747300513D51756974005234
:10E2E0003D44756D702052414D00563D73686F7707
:10E2F00020696E7465727275707420566563746FF0
:10E30000727300593D506F727420626C696E6B00BD
:10E310002A0011241FBECFEFD1E2DEBFCDBF01E046
:10E320000CBF12E0A0E0B2E0EEE1FDEF03E00BBFB6
:10E3300002C007900D92A030B107D9F712E0A0E01B
:10E34000B2E001C01D92AE30B107E1F70F9460F367
:10E350000D948DFE01E20EBF0FEF0DBF11241FBE05
:10E360000D9460F30D9400F020E030E040ED57E0B4
:10E3700005C0FA013197F1F72F5F3F4F2817390792
:10E38000C0F308959C01260F311DC901A0E0B0E043
:10E390002F5F3F4FABBFFC018791882361F08093D3
:10E3A000C6008091C00086FFFCCF8091C0008064D1
:10E3B0008093C000EACF08958DE08093C6008091DD
:10E3C000C00086FFFCCF8091C00080648093C000B5
:10E3D0008AE08093C6008091C00086FFFCCF8091C8
:10E3E000C00080648093C00008950F94C2F10F9420
:10E3F000DCF10895FC019081992359F09093C600B7
:10E400008091C00086FFFCCF8091C0008064809323
:10E41000C0003196992379F70895282F982F929567
:10E420009F70892F805D8A3308F0895F8093C600D2
:10E430008091C00086FFFCCF8091C00080648093F3
:10E44000C000822F8F70982F905D9A3308F0995FEB
:10E450009093C6008091C00086FFFCCF8091C000E1
:10E4600080648093C00008959C01FB01853691056E
:10E470001CF46330710594F0C90164E670E00F94F8
:10E480002EFE605D7F4F6093C6008091C00086FFC6
:10E49000FCCF8091C00080648093C0002B30310598
:10E4A00014F43297B4F0C90164E670E00F942EFEC4
:10E4B0006AE070E00F942EFE605D7F4F6093C600AF
:10E4C0008091C00086FFFCCF8091C0008064809363
:10E4D000C000C9016AE070E00F942EFEC0968093E0
:10E4E000C6008091C00086FFFCCF8091C000806490
:10E4F0008093C00008951F93182F8EE692EE60E07F
:10E500000F94C2F11093C6008091C00086FFFCCF2B
:10E510008091C00080648093C0000F94DCF11F9153
:10E5200008952F923F924F925F926F927F928F92B7
:10E530009F92AF92BF92CF92DF92EF92FF920F9392
:10E540001F93DF93CF93CDB7DEB762970FB6F894E2
:10E55000DEBF0FBECDBF382E622ECA01DB015C01CB
:10E560006D01772420E2222E2E010894411C511CBB
:10E570008BC081E0A81680E0B80681E0C80680E084
:10E58000D80628F0C601AA27BB270F940DF2BB2797
:10E59000AD2D9C2D8B2D0F940DF28A2D0F940DF225
:10E5A0002092C6008091C00086FFFCCF8091C00001
:10E5B00080648093C0009DE29093C6008091C0006B
:10E5C00086FFFCCF8091C00080648093C0002092C1
:10E5D000C6008091C00086FFFCCF8091C00080649F
:10E5E0008093C00019828601750188249924A1E0D6
:10E5F0003A1651F03A1620F0B2E03B1661F409C029
:10E600000BBFF701779007C0C7010F9477FE782EF4
:10E6100002C0F7017080872D0F940DF22092C60082
:10E620008091C00086FFFCCF8091C0008064809301
:10E63000C000872D8052F401EF70F0708F3520F408
:10E64000E40DF51D708204C0E40DF51D8EE280839B
:10E650000894E11CF11C011D111D0894811C911CE2
:10E6600090E18916910409F0C2CF80E190E0A0E02A
:10E67000B0E0A80EB91ECA1EDB1E198AC2010F9493
:10E68000FAF10F94DCF16A94662009F072CF629679
:10E690000FB6F894DEBF0FBECDBFCF91DF911F91B3
:10E6A0000F91FF90EF90DF90CF90BF90AF909F9031
:10E6B0008F907F906F905F904F903F902F90089534
:10E6C0002F923F924F925F926F927F928F929F9282
:10E6D000AF92BF92CF92DF92EF92FF920F931F9370
:10E6E000DF93CF93CDB7DEB7CD53D1400FB6F894BB
:10E6F000DEBF0FBECDBF01E20EBF0FEF0DBF94B75F
:10E70000F894A89514BE80916000886180936000A1
:10E7100010926000789493FF05C0E0910002F091A0
:10E7200001021995279A2F9A8091C00082608093E8
:10E73000C00080E18093C40088E18093C1000000A4
:10E74000EE24FF24870144E0A42EB12CCC24DD2448
:10E7500024C0C5010197F1F70894E11CF11C011DCB
:10E76000111D21E2E2162EE4F20620E0020720E06D
:10E77000120718F031E0C32ED12CC801B70127ECE5
:10E780003BE140E050E00F9441FE611571058105C9
:10E79000910519F485B1805885B98091C00087FD35
:10E7A00003C0C114D104A9F2A6014F5F5F4FC25E3E
:10E7B000DE4F59834883CE51D140C25EDE4F8881FF
:10E7C0009981CE51D140019711F00D9410FEC05D9A
:10E7D000DE4F19821882C053D14060E0C15DDE4F28
:10E7E0001882CF52D14088249924C35DDE4F19820C
:10E7F0001882CD52D140C05EDE4F188219821A8233
:10E800001B82C052D140CE5CDE4F188219821A8220
:10E810001B82C253D140EE24FF2487010BBFF701B6
:10E8200007911691C45CDE4F19830883CC53D14005
:10E830000D940BFEC25EDE4F28813981CE51D1404E
:10E840002130310509F52091C600C25EDE4F1982E4
:10E850001882CE51D14022C02F5F3F4F4F4F5F4FA4
:10E86000213082E138078AE7480780E0580780F0C6
:10E87000C45CDE4FE881F981CC53D140EF5FFF4F9C
:10E8800019F0EE27FF27099420E030E040E050E047
:10E890008091C00087FFE0CF2091C600C35DDE4FAE
:10E8A00048815981CD52D1404F5F5F4FC35DDE4FEC
:10E8B00059834883CD52D140213209F063C64A3092
:10E8C000510508F05FC60894811C911C53E0851621
:10E8D000910409F059C600E010E018C081E280936D
:10E8E000C6008091C00086FFFCCF8091C00080648C
:10E8F0008093C0002F5F3F4F2931310579F70F9486
:10E90000DCF10F5F1F4F0530110519F020E030E0FA
:10E91000E5CF10920A0210920B0210920C02109294
:10E920000D02109206021092070210920802109235
:10E930000902109202021092030210920402109235
:10E9400005028FEE90EE60E00F94F5F180E191EE1C
:10E9500060E00F94C2F18091C00087FFFCCF9091DE
:10E96000C600903608F09F759032B8F09093C600BC
:10E970008091C00086FFFCCF8091C00080648093AE
:10E98000C000A0E2A093C6008091C00086FFFCCF2B
:10E990008091C00080648093C000983409F4D7C18E
:10E9A0009934B8F4923409F459C1933458F490333B
:10E9B00019F1903308F4E3C59F33A1F1903409F0C5
:10E9C000DEC5BDC0953409F470C1963409F0D7C5D1
:10E9D00098C1923509F42BC2933538F49C3409F46C
:10E9E000F5C1913509F0CBC518C2963509F445C279
:10E9F000993509F0C4C567C483E792EE62E00F94CD
:10EA0000F5F110920602109207021092080210927D
:10EA1000090210920A0210920B0210920C0210923C
:10EA20000D0213C18FE792EE62E00F94F5F18FEEC5
:10EA300090EE60E00F94F5F181E291EE60E00F94CA
:10EA4000C2F187EB91EE60E00F94F5F180E391EE77
:10EA500060E00F94C2F184EE90EE60E00F94F5F167
:10EA60008FE391EE60E00F94C2F186E090E061E008
:10EA700070E00F9434F20F94DCF18DE591EE60E0DC
:10EA80000F94C2F189EC91EE60E00F94F5F18EE401
:10EA900091EE60E00F94C2F183EC91EE60E00F9490
:10EAA000F5F18CE691EE60E00F94C2F18EE10F94E7
:10EAB0000DF288E90F940DF281E00F940DF20F949E
:10EAC000DCF18BE791EE60E00F94C2F119E0E0E039
:10EAD000F0E010935700E4918E2F0F940DF20F94F5
:10EAE000DCF18AE891EE60E00F94C2F1E3E0F0E03F
:10EAF00010935700E4918E2F0F940DF20F94DCF1D8
:10EB000089E991EE60E00F94C2F1E2E0F0E0109349
:10EB10005700E4918E2F0F940DF20F94DCF188EAE8
:10EB200091EE60E00F94C2F1E1E0F0E01093570045
:10EB30001491812F0F940DF20F94DCF107CF8BE825
:10EB400092EE62E00F94F5F18BE492EE60E00F94A8
:10EB5000F5F10F94DCF100E010E019C0C8016F2D51
:10EB60000F947FFEFF2031F489E492EE60E00F9471
:10EB7000C2F10BC0F092C6008091C00086FFFCCFAE
:10EB80008091C00080648093C0000F5F1F4FC80158
:10EB900081519F41A0E0B0E0ABBFFC01F790BAE229
:10EBA000FB1621F0E2E000301E07C1F60F94DCF105
:10EBB0000F94DCF187E592EE60E00F94F5F10F948D
:10EBC000DCF1CC24DD2400E010E01EC0C8010F946D
:10EBD00077FEF82E882331F489E492EE60E00F94FA
:10EBE000C2F10BC08093C6008091C00086FFFCCFAD
:10EBF0008091C00080648093C000FE1419F00894D6
:10EC0000C11CD11C0F5F1F4FC80181519F41A0E063
:10EC1000B0E0ABBFFC01E790FAE2EF1621F022E092
:10EC20000030120799F60F94DCF10F94DCF182E6C4
:10EC300092EE60E00F94C2F1C60161E070E00F94C3
:10EC400034F20F94DCF10F94DCF110920202109276
:10EC50000302109204021092050278CE89E992EE26
:10EC600062E00F94F5F1279A2F9A16C02F9880E052
:10EC700090E0E0EDF7E03197F1F7019684369105E9
:10EC8000C1F72F9A80E090E0E0EDF7E03197F1F7DF
:10EC9000019684369105C1F78091C00087FFE6CFC9
:10ECA0008091C00087FFFCCF64C485EA92EE62E0E9
:10ECB0000F94F5F140910202509103026091040219
:10ECC0007091050281E020E10F9491F2809102029F
:10ECD00090910302A0910402B091050280509F4FD1
:10ECE000AF4FBF4F8093020290930302A0930402A0
:10ECF000B093050280509041A040B04008F426CE69
:10ED0000A4CF83EB92EE62E00F94F5F140910602FE
:10ED100050910702609108027091090280E020E1A1
:10ED20000F9491F28091060290910702A09108023F
:10ED3000B091090280509F4FAF4FBF4F80930602A2
:10ED400090930702A0930802B0930902FFCD80ECD4
:10ED500092EE62E00F94F5F183E792EE60E00F949B
:10ED6000F5F18FE792EE60E00F94F5F18BE892EE0B
:10ED700060E00F94F5F189E992EE60E00F94F5F10F
:10ED800085EA92EE60E00F94F5F183EB92EE60E09D
:10ED90000F94F5F180EC92EE60E00F94F5F187ECC2
:10EDA00092EE60E00F94F5F188ED92EE60E00F9442
:10EDB000F5F18FED92EE60E00F94F5F18AEE92EEB0
:10EDC00060E00F94F5F183E093EEBDCD87EC92EE19
:10EDD00062E00F94F5F181E40F947BF282E40F94EA
:10EDE0007BF283E40F947BF284E40F947BF285E45E
:10EDF0000F947BF286E40F947BF287E40F947BF20E
:10EE000088E40F947BF28AE40F947BF28BE40F94F6
:10EE10007BF28CE40F947BF299CD88ED92EE62E068
:10EE20000F94F5F1772473948824992409C48FED05
:10EE300092EE62E00F94F5F140910A0250910B02BC
:10EE400060910C0270910D0282E020E10F9491F22A
:10EE500080910A0290910B02A0910C02B0910D02D8
:10EE600080509F4FAF4FBF4F80930A0290930B0289
:10EE7000A0930C02B0930D0269CD8AEE92EE62E08F
:10EE80000F94F5F184EE90EE60E00F94F5F18FECC5
:10EE900091EE60E00F94F5F1662477244301CC5D98
:10EEA000DE4F19821882C452D140D401C301B695F5
:10EEB000A79597958795CA5DDE4F88839983AA8326
:10EEC000BB83C652D140CC5DDE4FA881B981C4520C
:10EED000D1401196CC5DDE4FB983A883C452D14096
:10EEE000CD0162E070E00F9434F2B0E2B093C6005E
:10EEF0008091C00086FFFCCF8091C0008064809329
:10EF0000C000EDE2E093C6008091C00086FFFCCF18
:10EF10008091C00080648093C000F0E2F093C6004E
:10EF20008091C00086FFFCCF8091C00080648093F8
:10EF3000C000CA5DDE4FE880F9800A811B81C6529D
:10EF4000D140BB27A12F902F8F2D0F940DF2CA5DBA
:10EF5000DE4F8881C652D1400F940DF2B0E2FB2EF5
:10EF6000F092C6008091C00086FFFCCF8091C00067
:10EF700080648093C0000DE30093C6008091C000C0
:10EF800086FFFCCF8091C00080648093C00010E2B7
:10EF90001093C6008091C00086FFFCCF8091C00016
:10EFA00080648093C0008BBEF3012791C65DDE4F65
:10EFB0002883CA52D140A22EBB24CC24DD2408943D
:10EFC000611C711C811C911C8BBEF3018791282E42
:10EFD0003324442455240894611C711C811C911C09
:10EFE0008BBEF3013791C55DDE4F3883CB52D140E4
:10EFF0000894611C711C811C911C8BBEF30147910C
:10F00000C45DDE4F4883CC52D140ADEFEA2EAFEF66
:10F01000FA2EAFEF0A2FAFEF1A2F6E0C7F1C801E57
:10F02000911E142D032DF22CEE24EA0CFB1C0C1D5A
:10F030001D1D0F940DF220E22093C6008091C000A8
:10F0400086FFFCCF8091C00080648093C000C65DC5
:10F05000DE4F8881CA52D1400F940DF230E23093D6
:10F06000C6008091C00086FFFCCF8091C000806404
:10F070008093C000C45DDE4F8881CC52D1400F9494
:10F080000DF240E24093C6008091C00086FFFCCFA5
:10F090008091C00080648093C000C55DDE4F888190
:10F0A000CB52D1400F940DF250E25093C6008091A4
:10F0B000C00086FFFCCF8091C00080648093C000B8
:10F0C0008FEFE8168FEFF80680E0080780E018075A
:10F0D00031F484E092EE60E00F94C2F1DFC0D80119
:10F0E000C7018070907CA070B0708050904CA040A0
:10F0F000B040D1F52FEF3FE340E050E0E222F322B1
:10F1000004231523CA5DDE4FA880B980CA80DB8046
:10F11000C652D140AE0CBF1CC01ED11EAA0CBB1CD7
:10F12000CC1CDD1C8EE092EE60E00F94C2F1BB2798
:10F13000A12F902F8F2D0F940DF28E2D0F940DF285
:10F1400030E23093C6008091C00086FFFCCF8091F2
:10F15000C00080648093C0004EE34093C60080915D
:10F16000C00086FFFCCF87C08EE09EEFA0E0B0E03D
:10F17000E822F9220A231B239CE0E91694E9F90608
:10F1800090E0090790E0190709F088C0C45DDE4FE0
:10F19000A881CC52D140EA2EFF2400E010E0102FCD
:10F1A0000F2DFE2CEE24C55DDE4FB881CB52D14031
:10F1B000EB0EF11C011D111DD601C501817090706F
:10F1C000A070B070DC0199278827E80EF91E0A1F8D
:10F1D0001B1F20EF30E040E050E0A222B322C42207
:10F1E000D52241E1AA0CBB1CCC1CDD1C4A95D1F7F1
:10F1F000EA0CFB1C0C1D1D1D81E090E0A0E0B0E0BE
:10F20000282239224A225B2235E1220C331C441C7D
:10F21000551C3A95D1F7E20CF31C041D151D57013E
:10F220006801AA0CBB1CCC1CDD1C85E192EE60E0E1
:10F230000F94C2F1C801AA27BB270F940DF2BB2778
:10F24000A12F902F8F2D0F940DF28E2D0F940DF274
:10F2500090E29093C6008091C00086FFFCCF809121
:10F26000C00080648093C000AEE3A093C60080918C
:10F27000C00086FFFCCF8091C00080648093C000F6
:10F28000C601AA27BB270F940DF2BB27AD2D9C2DDD
:10F290008B2D0F940DF28A2D0F940DF20F94DCF14B
:10F2A000CC5DDE4FE881F981C452D140F99709F471
:10F2B0004DCBF4E0EF2EF12C012D112D6E0C7F1CA7
:10F2C000801E911EF2CD83E093EE62E00F94F5F183
:10F2D0008AE192EE60E00F94C2F18091C00087FF56
:10F2E000FCCF1091C6001F751093C6008091C0001E
:10F2F00086FFFCCF8091C00080648093C0000F9493
:10F30000DCF1812F81548A3108F036C1163409F4BA
:10F3100095C0173490F4133409F44EC0143430F40B
:10F320001134F1F0123409F01DC130C0143409F465
:10F3300059C0153409F016C16BC01A3409F4C4C0A1
:10F340001B3438F4173409F48FC0183409F00AC19B
:10F35000A1C01B3409F4D2C01C3409F003C1E8C0B9
:10F360008FEF81B90DC082B1809582B980E090E0C5
:10F37000E0EDF7E03197F1F70196883C9105C1F790
:10F380008091C00087FFEFCF12B8EFC08FEF84B934
:10F390000DC085B1809585B980E090E0E0EDF7E0A3
:10F3A0003197F1F70196883C9105C1F78091C00033
:10F3B00087FFEFCF15B8D9C08FEF87B90DC088B1DF
:10F3C000809588B980E090E0E0EDF7E03197F1F7C3
:10F3D0000196883C9105C1F78091C00087FFEFCF6F
:10F3E00018B8C3C08FEF8AB90DC08BB180958BB9A7
:10F3F00080E090E0E0EDF7E03197F1F70196883C8E
:10F400009105C1F78091C00087FFEFCF1BB8ADC059
:10F410008FEF8DB90DC08EB180958EB980E090E0F0
:10F42000E0EDF7E03197F1F70196883C9105C1F7DF
:10F430008091C00087FFEFCF1EB897C08FEF80BBD1
:10F440000DC081B3809581BB80E090E0E0EDF7E0F6
:10F450003197F1F70196883C9105C1F78091C00082
:10F4600087FFEFCF11BA81C08FEF83BB0DC084B38C
:10F47000809584BB80E090E0E0EDF7E03197F1F714
:10F480000196883C9105C1F78091C00087FFEFCFBE
:10F4900014BA6BC08FEF809301010FC080910201FD
:10F4A00080958093020180E090E0E0EDF7E03197F5
:10F4B000F1F70196883C9105C1F78091C00087FF64
:10F4C000EDCF1092020151C08FEF809304010FC065
:10F4D0008091050180958093050180E090E0E0ED4A
:10F4E000F7E03197F1F70196883C9105C1F78091DB
:10F4F000C00087FFEDCF1092050137C08FEF8093DA
:10F5000007010FC08091080180958093080180E079
:10F5100090E0E0EDF7E03197F1F70196883C910536
:10F52000C1F78091C00087FFEDCF109208011DC088
:10F530008FEF80930A010FC080910B01809580931B
:10F540000B0180E090E0E0EDF7E03197F1F70196F4
:10F55000883C9105C1F78091C00087FFEDCF1092E4
:10F560000B0103C085E292EEEEC98091C00087FFD7
:10F57000FCCF8091C600EAC988E392EEE4C98CE131
:10F5800091EEE1C988249924933011F1943028F444
:10F59000913089F09230B8F408C0953061F195301F
:10F5A000F0F0963009F048C043C02B3109F042C951
:10F5B00091E06BE13FC96227C15DDE4F2883CF52E6
:10F5C000D14092E037C9B22FA0E0622793E032C960
:10F5D000822F90E0A82BB92B622794E02BC92E3004
:10F5E00009F039C3622795E0C05DDE4F19821882A9
:10F5F000C053D1401FC9E1E0F0E0EC0FFD1FC05D3A
:10F60000DE4F08811981C053D140E00FF11F2083E4
:10F610000F5F1F4FC05DDE4F19830883C053D14079
:10F6200062270A171B0709F005C9D80196E002C92D
:10F63000261709F010C303C0973009F0FBC87724E0
:10F640009981933109F412C19431C8F4963009F4C8
:10F65000D8C0973050F4923009F406C1933009F4C1
:10F660006DC0913009F059C253C0913109F477C08F
:10F67000923108F0BBC0903109F04FC2F5C098310B
:10F6800009F487C0993150F4953109F4EFC09531F0
:10F6900008F4C6C1963109F040C2C2C19A3109F4DA
:10F6A0006CC09A3108F491C09B3109F45BC09D3164
:10F6B00009F033C29D81903359F48F81882311F46E
:10F6C0009EE11CC0813011F091E018C098E916C08D
:10F6D000892F807591F0903539F4E0E0F0E089E011
:10F6E0008093570094910AC0983539F4E3E0F0E034
:10F6F00089E080935700949101C090E01A821B82A8
:10F700008D818C831D829E831F8227E030E009C299
:10F710001A8288E08B8381E48C8386E58D8382E581
:10F720008E8389E48F8383E5888780E589878FE5E9
:10F730008A8782E38B872BE030E0F3C18A818139AD
:10F7400041F0823941F0803911F48FE005C080E04A
:10F7500003C082E001C08AE01A828B8344C0772410
:10F76000739482C08D81882311F48EE12CC0813086
:10F7700011F081E028C088E926C01A82E1E0F0E0BB
:10F7800089E08093570084918B831C8224E030E0D1
:10F79000C8C18B81803589F48C81883039F4E2E0EE
:10F7A000F0E089E08093570084910DC0E0E0F0E044
:10F7B00089E080935700849106C0E3E0F0E089E09F
:10F7C0008093570084911A82DFCF8D81836C99E0FA
:10F7D000E1E0F0E0082E90935700E89507B600FCB2
:10F7E000FDCF1A821B8223E030E09BC180EC8A832C
:10F7F000CE5CDE4F188219821A821B82C253D1401E
:10F800008EC18A8190E0A0E0B0E0582F44273327D2
:10F8100022278B8190E0A0E0B0E0DC0199278827C7
:10F82000282B392B4A2B5B2B8D8190E0A0E0B0E098
:10F83000282B392B4A2B5B2B8C8190E0A0E0B0E089
:10F84000BA2FA92F982F8827282B392B4A2B5B2BCF
:10F85000220F331F441F551FC05EDE4F288339839C
:10F860004A835B83C052D1401A8259C13A81C95C34
:10F87000DE4F3883C753D140CA5CDE4F1882C6536F
:10F88000D1408B81C82EDD24CA5CDE4F488159816E
:10F89000C653D140C42AD52A933109F082C0CE5C28
:10F8A000DE4F88819981AA81BB81C253D1408050AB
:10F8B000904CA340B04030F583E0CE5CDE4FE88052
:10F8C000F9800A811B81C253D140F70100935B008C
:10F8D00080935700E89507B600FCFDCFCE5CDE4F65
:10F8E000088119812A813B81C253D14000501F4FAA
:10F8F0002F4F3F4FCE5CDE4F088319832A833B8313
:10F90000C253D140C05EDE4F488159816A817B81FC
:10F91000C052D140DE011B9631E08C9111962C91A2
:10F9200011971296C75CDE4F2883C953D140C85C3B
:10F93000DE4F1882C853D14090E0C85CDE4FE881AA
:10F94000F981C853D1408E2B9F2B0C01FA01609393
:10F950005B0030935700E89511244E5F5F4F6F4F67
:10F960007F4F0EEFE02E0FEFF02ECE0CDF1CC114F8
:10F97000D10499F685E0C05EDE4F088119812A81A5
:10F980003B81C052D140F80120935B008093570027
:10F99000E89507B600FCFDCF81E180935700E8951C
:10F9A00035C0C05EDE4F88819981AA81BB81C0527B
:10F9B000D140B695A795979587957C018601ABE0D8
:10F9C000AA2EB12CAC0EBD1E0BC0D5016D915D01F0
:10F9D000C7010F947FFE0894E11CF11C01501040F8
:10F9E0000115110591F7A60160E070E0440F551F65
:10F9F000661F771FC05EDE4FE880F9800A811B8199
:10FA0000C052D1404E0D5F1D601F711F1A82C05E33
:10FA1000DE4F488359836A837B83C052D1407FC0C5
:10FA2000FA80C55CDE4FF882CB53D140C65CDE4F16
:10FA30001882CA53D1408B81C82EDD24C65CDE4FAC
:10FA400008811981CA53D140C02AD12A1A828981DA
:10FA5000BE016D5F7F4F843121F59601C05EDE4FA0
:10FA6000E880F9800A811B81C052D1400BBFF701A9
:10FA700087919691DB018C9311969C936E5F7F4FDB
:10FA8000D801C7010296A11DB11DC05EDE4F88835B
:10FA90009983AA83BB83C052D14022503040F1F6F3
:10FAA00036C0C05EDE4F288139814A815B81C052F9
:10FAB000D1400894C108D108760100E010E0089414
:10FAC000C11CD11C0894E11CF11C011D111DE20E8A
:10FAD000F31E041F151F21BDBB27A52F942F832FB5
:10FAE00082BD2F5F3F4F4F4F5F4FF89A80B5DB01CC
:10FAF0008D93BD012E153F054007510761F7C05E8C
:10FB0000DE4F288339834A835B83C052D1409601FC
:10FB10002D5F3F4FFB01108204C080EC8A8322E0FE
:10FB200030E08BE18093C6008091C00086FFFCCF5F
:10FB30008091C00080648093C000C15DDE4FF88179
:10FB4000CF52D140F093C6008091C00086FFFCCF19
:10FB50008091C00080648093C000432F3093C60022
:10FB60008091C00086FFFCCF8091C00080648093AC
:10FB7000C000922F2093C6008091C00086FFFCCF6A
:10FB80008091C00080648093C0008EE08093C600A6
:10FB90008091C00086FFFCCF8091C000806480937C
:10FBA000C00065E1C15DDE4FE880CF52D1406E25D7
:10FBB00069276427FE01319610C090819093C6009A
:10FBC0008091C00086FFFCCF31968091C000806498
:10FBD0008093C0006927215030402115310569F715
:10FBE0006093C6008091C00086FFFCCF8091C0006A
:10FBF00080648093C00085B1805885B9772081F4F6
:10FC0000C15DDE4F0881CF52D1400F5FC15DDE4F35
:10FC10000883CF52D14090E0A0E0B0E00D941AF4F8
:10FC200027982F9880E090E020ED37E0F901319798
:10FC3000F1F7019684369105C9F700008091C00064
:10FC40008D7F8093C00081E180935700E895EE2777
:10FC5000FF270994FFCF90E00D941AF497FB092E2B
:10FC600007260AD077FD04D02ED006D000201AF443
:10FC7000709561957F4F0895F6F7909581959F4F08
:10FC80000895A1E21A2EAA1BBB1BFD010DC0AA1FDD
:10FC9000BB1FEE1FFF1FA217B307E407F50720F0F5
:10FCA000A21BB30BE40BF50B661F771F881F991F70
:10FCB0001A9469F760957095809590959B01AC01B9
:10FCC000BD01CF010895AA1BBB1B51E107C0AA1FAC
:10FCD000BB1FA617B70710F0A61BB70B881F991FED
:10FCE0005A95A9F780959095BC01CD010895F99991
:10FCF000FECF92BD81BDF89A992780B50895262F31
:10FD0000F999FECF1FBA92BD81BD20BD0FB6F89400
:0EFD1000FA9AF99A0FBE01960895F894FFCF63
:040000033000E000E9
:00000001FF
